:020000040000FA
:1000000000800020A511000001400020AF11000079
:1000100000000000000000000000000000000000E0
:10002000000000000000000000000000AF11000010
:100030000000000000000000B1110000B31100003A
:10004000B5110000B5110000B5110000B511000098
:10005000B51100008F1C0000B5110000B5110000A3
:10006000B5110000B5110000B5110000B511000078
:10007000351D0000B5110000B5110000B5110000DC
:10008000B5110000B5110000B5110000B511000058
:100090000348854601F02AFF004800477503000029
:1000A000008000207CB5844D0C462878090408D5D2
:1000B00013F0D4FD002801D013F0A8FD0120C003E7
:1000C00032E0E10701D001202EE061070BD5FF21CE
:1000D000F53100910822019000231146688803F051
:1000E00041FE042020E0A00720D56A78FF2665366F
:1000F000642A08D30021FF32334608467B3200F0E1
:10010000C9F8002068706A783346FF320021012068
:100110007B3200F0BFF868786422001D687002210D
:10012000287813F077FF022060407CBD00207CBD62
:1001300030B585B0614809F08FFE5F4D012428700D
:1001400069460C706A4621465D4803F0B3FF5C487F
:100150002A1D0721401C03F0ADFF59482A461432DE
:100160001A21801C03F0A6FF564A1521002005F035
:10017000B1FC0020694600900C71087203200873DE
:100180000C746A460421504803F072FB012101AA55
:10019000880203F06DFB4C4802AA0121801F03F086
:1001A00067FB494803AA0121401F03F061FB464851
:1001B00004AA0121801E03F05BFB0620694608703B
:1001C00001216A46084600F036F900F0EDFE2946A6
:1001D00030310846243800F00EFC0121287813F055
:1001E000C7FD05B030BD1CB5030009F0D7FF072ED1
:1001F00005101F121D2F2E00C1206946800003F03C
:1002000029FD6946012004F02BF930A01FE033A03E
:100210001DE02948498941801922D2010421007832
:1002200013F0F8FE31A012E034A010E08878042822
:1002300005D0062805D0052807D137A007E03CA047
:1002400005E0897941A009F081FF1CBD46A009F0B5
:100250007DFF1CBDF8B50024069E079D002B04D031
:10026000012B07D0022B0BD011E00095337800F062
:10027000D3FE03E03346009500F0E1FE044606E0BD
:100280000D48FF22F5320221007813F0C3FE20460C
:10029000F8BD70471CB56C4620706170A270100AE2
:1002A000E0702371180A607101216B46062208462E
:1002B00000F0BFFB1CBD000020420020A500000094
:1002C000050300009041010007040000496E6974B5
:1002D00069616C697A65642E2E0A00004164766556
:1002E00072746973696E672E2E0A0000436F6E6E1A
:1002F00065637465642E2E0A00000000436F6E6E05
:100300006563746564204164766572746973696EAF
:10031000672E2E0A000000004164766572746973CE
:10032000696E672074696D656F75742E2E0A000002
:1003300057616974696E6720666F722061647665C3
:1003400072746973696E672E2E0A000044697363C4
:100350006F6E6E65637465642E2E20526561736FD7
:100360006E3A25780A0000004572726F722E2E0ACE
:10037000000000000D498A6A481502438A62032181
:1003800001F088F901F08DFB09490AA009F0DEFEB1
:1003900001F0EDFB01F06BFC03F074FD00F004FBD9
:1003A000FFF7C6FE09F076FDFCE700008010004074
:1003B000B442010025730A0010B58F498F4804F03C
:1003C000B9FC8F4B102218460521503804F084FEEA
:1003D00010BD8B496839486170473EB504460079C5
:1003E000C00727D06088844904F068FEC00721D088
:1003F000002000906088002301221B2105F072FA82
:100400000290002816D07E4869465038408D88807A
:100410000120C8807A48029968380078087060889E
:10042000002201A905F044F8002803D01B2101A8EF
:1004300005F09EFA3EBD10B50024012802D002242A
:10044000204610BD6E4811786838417000788842A7
:10045000F6D26C480FF0B6F8F2E7694B10B50022FF
:10046000683B002809D0012809D01833022809D098
:1004700003280AD00222104610BD187800E05878F0
:100480000870F8E758890880F5E75D486238047815
:100490000C7140784871588D0880588F4880012031
:1004A0008871E8E770B5564D683DA868002800D00F
:1004B0008047FF24E8682D34002800D08047A988B1
:1004C000A14201D8642070BD6888A04201D30020F9
:1004D00070BD2A69002A02D02046904770BD091AD3
:1004E000491C0904201A1922890C50434018401E47
:1004F00001F058FCC0B270BD10B5FFF7D3FF404902
:1005000068390A78904203D208703E480FF05AF8D2
:10051000002010BD30B53A48049D6838039C4180E6
:100520008280083038C030BD70B5049800241D4664
:100530001646002801D00B2070BD48684278037829
:100540001002314A184390420CD1FFF7ABFF2C49FF
:1005500068390A78904200D2087001202880087813
:1005600030700BE0294A904207D1022028800246D1
:10057000C968304613F054FA00E00A24204670BDE2
:100580007CB54C6815466278247812022243204CD0
:10059000069EE24208D10122019200962A4604F00A
:1005A0002FFC040003D000E00A2420467CBD6878BC
:1005B0002978000208431249683949690029F4D0B2
:1005C000002802D001208847EFE70220FBE710B5A2
:1005D00004460A48401E84420DD0012907D0022952
:1005E00009D1012120460FF055F8002803D1024916
:1005F000204604F09FFB10BDE4680020FFFF0000D0
:10060000C8420020DB030000192A0000082900006E
:10061000FED6FFFF10B56E4B102213216D4804F07B
:100620005BFD10BD10B500241346002802D0022443
:10063000204610BD67480A461946093813F0F0F9FC
:10064000F6E770B50D460024030009F0A7FD090682
:100650000A1014181C2024282C005E49082209398D
:1006600001E05D490D22284613F0DAF91CE05A49F1
:100670000E220D31F7E7584912221B31F3E7564994
:1006800012222D31EFE7544912223F31EBE7524954
:1006900012225131E7E750490E226331E3E74D4919
:1006A00007221039DFE70224204670BDF8B54968FB
:1006B00094464A78097817020F430698474A112151
:1006C0000025079CBE1A091A974244D009DC444A07
:1006D000BA1813D0012A1DD0022A26D0032A08D125
:1006E0002FE0012E41D0022E49D0032E51D0292EC9
:1006F0005BD0002018800A252846F8BD082856D26D
:100700000821091AA14200D80C463249A2B21A8027
:10071000093957E00C284AD20C21091AA14200D805
:100720000C46A2B21A802C494CE00D283FD20D2174
:10073000091AA14200D80C462749A2B21A800D31ED
:1007400040E0112833D2A14200D80C462249A2B27F
:100750001A801B3136E0112829D2A14200D80C465C
:100760001D49A2B21A802D312CE011281FD2A142BE
:1007700000D80C461849A2B21A803F3122E0112855
:1007800015D2A14200D80C461349A2B21A805131A9
:1007900018E00E280BD20E21091AA14200D80C46EF
:1007A0000D49A2B21A8063310CE0072801D3072556
:1007B000A2E70721091AA14200D80C460549A2B2B6
:1007C0001A8010390918604613F02AF994E70000DE
:1007D00018440020E8420020D0410100272A0000F0
:1007E000DDD5FFFF704710B5FE4B012806D002286B
:1007F00003D10221987913F06BFC10BD18780428FE
:10080000FBD1F94A0221987913F004FC10BDFEB522
:10081000064600201746F34C0D4603460A46009054
:100820001B21208905F05EF80290002813D068464D
:100830008680C5802A463946029813F0F1F80022D6
:1008400001A9208904F034FE040005D01B2101A871
:1008500005F08EF800E013242046FEBD30B5E14AD5
:100860000446E24BD068D2791B780BE00579A542AB
:1008700005D145798D4202D185799D4205D0521E20
:10088000D2B20830002AF1D1002030BDFFB581B0CE
:1008900015460E460746FFF7E1FF04001CD06088AE
:1008A000694604F0EBFC002816D0C168CD480089E9
:1008B00004F004FCC0070FD020882946049AFFF7F3
:1008C000A6FF002808D1CA482A46077046708570DE
:1008D000C01C049913F0A4F805B0F0BD70B5C14D6B
:1008E0000C4608040AD5A87913F0B8F9002801D0FD
:1008F00013F08CF901212046C9030AE0E0070AD071
:10090000B84AA87920321146083903F09FFB2046E7
:100910000121484070BDB348610700780CD5042818
:1009200008D1B4A009F012FCA878002802D12889C7
:1009300003F086FC04200BE0A1070BD5042806D1A8
:10094000FFF7DAFDA84A0221A87913F063FB022021
:10095000604070BD200725D56878082126464E40A6
:1009600000281BD028796979884201D1002309E049
:100970000B21401C01F000FA29710B2041439C48D7
:100980000B300B18002B05D09A7859781878DB1C9F
:10099000FFF77CFF28796979884201D1304670BD24
:1009A000204670BD002070BD38B5974809F054FA54
:1009B0008C4C6946A0710120087001466A46934834
:1009C00002F056FF0025ED43284604F0D9FF2846E3
:1009D00004F068F9FFF71EFEFFF7EEFC00F04AFB9B
:1009E0008B48FFF7F6FC8B4800F051FB0121A07902
:1009F00013F0BEF938BD7B4A116150617047794AE6
:100A0000D160D071704708B53021032004F06CF834
:100A10005021042004F068F83C21012004F064F81F
:100A200001206946087001466A467B4803F042FB94
:100A300008BDF8B50E466B49074608781C461546B2
:100A400004281AD0022826D000F062FA002820D00C
:100A50002021032004F048F83021042004F044F859
:100A60000521012004F040F8012069460870014684
:100A70006A46694803F01EFB0DE0487800280AD05A
:100A800008794979884206D131463846FFF7FEFE9B
:100A9000F8BDFFF7B8FF23462A463146384600F036
:100AA00042FAF8BD08B54F480178042908D0002063
:100AB000694608706A460121574803F0FBFA08BDF1
:100AC000008903F0BDFB08BDF8B50024002802D062
:100AD00002242046F8BD002901D01824F9E7444F2C
:100AE00079783878FFF7BAFE05001CD0BA78F91C7F
:100AF0000023082A09D8002004E00E5C9E4204D19D
:100B0000401CC0B29042F8D308E00021F81C13F05A
:100B100061F8B9782888FA1CFFF779FE0B220021CA
:100B2000334813F057F82F4D2878042802D128892C
:100B300003F086FB002068712871024601464120BF
:100B4000000102F095FEC4E7022070470A46014604
:100B500010B52448008902F071FC10BD10B5214980
:100B60000246224BC868C9791B7808E00488944281
:100B700002D184799C4205D0491EC9B208300029AF
:100B8000F4D1002010BDFEB517464A681D465478C2
:100B90001278089824020026099B1443002804D0E8
:100BA0001E4A944201D00B20FEBD1C4A921C944266
:100BB0000AD01A4A293A944206D0184A193A94425D
:100BC00002D0521C944232D14889FFF7C7FF002857
:100BD0002AD001970095034A4179126900790123CF
:100BE00015681DE02C440020983A00006244002063
:100BF000F46800206869642069646C652065766526
:100C00006E742E2E0A000000DD080000140400009F
:100C1000E7070000E5070000050300004B2A00007D
:100C20002246A847064635E00020288032E0D54A13
:100C300094420ED1D44A1288904201D3072629E06B
:100C4000121A9A4200DD1A4692B22A80C96809181F
:100C50001DE0CC48401E844204D104202880C9688D
:100C6000024614E0C94A022094420DD0C54AD21C63
:100C7000944205D101202880C8680078387009E0C6
:100C8000C24A521E944205D12880C96802223846C1
:100C900012F0C6FE3046FEBDFFB583B084460C9808
:100CA000002416460F46002802D00B2007B0F0BDE6
:100CB00079684A78097815020D43B249891C8D423A
:100CC00003D0B04919398D4211D17889FFF746FF19
:100CD000002856D006A901960091AD4A41791269C3
:100CE0000079146800232A46A047044649E0A54934
:100CF0006A46491C138B8D420AD1012B40D13078B2
:100D0000002801D0012843D1002849D0012047E024
:100D10009E49891F8D422DD10121019100903246BB
:100D20003946604604F06CF804002AD170783178B6
:100D300002020A4396497B89C868C97905E0478859
:100D40009F4205D0491EC9B208300029F7D10020C2
:100D5000002816D006A901960091012A08D0032385
:100D60008B4A41791269007916682A46B04708E033
:100D70000223F5E78348C01C854202D1012B02D033
:100D80000D24204692E73078002803D0012801D0B6
:100D90008024F6E7F96808703078002805D0032031
:100DA0007B49096949688847EBE70220F8E7F8B50D
:100DB000774E0421B07913F08BF901213089FFF7C8
:100DC00006FC0121308900F0CDF937897148F568BA
:100DD000874212D0F4790EE06888002808D069466E
:100DE00004F04CFA002803D0C168384603F0A2FF93
:100DF000641EE4B20835002CEED100206649707004
:100E000001240C70B07001460B22644812F0E2FE1F
:100E100000F07EF8002816D070690079800712D59E
:100E2000A021032003F060FEA021042003F05CFE5B
:100E30000021012003F058FE684604706A46012133
:100E4000574803F037F9F8BDF8B50027504D0E4666
:100E50000446042803D0287804280BD012E07089B7
:100E600028816F70684607706A4601214C4803F07C
:100E700021F907E0FFF79BFFE878042802D1FFF78C
:100E8000C2FDEF702869002805D0C268002A02D090
:100E90003146204690472C70F8BD10B501203C4CDF
:100EA000002904D0012904D0022909D00EE0A07045
:100EB0000CE00021A170002A00D16070E27005E012
:100EC000002A03D16070208900F0F6F8207961795A
:100ED000884206D06078002803D00821A07912F05B
:100EE00047FF10BD38B50D4629490969002905D0CD
:100EF0008C68002C02D02946A04738BD6946294895
:100F000002F0ECF800212846009A02F097FA38BD6A
:100F100008B500206946087022480E3002F0DEF85D
:100F20006946087808BDFFB581B016460746FFF749
:100F3000EFFF002824D0164C0B216079401C00F0F4
:100F40001BFF617120790D46814204D10B21401CA9
:100F500000F012FF21710B204543104832460B3040
:100F600047552818029941708670C01C049912F0E8
:100F700057FD6078002803D00821A07912F0F8FE10
:100F8000AAE400004B2A0000584400200829000071
:100F90002C440020FEFF000062440020F468002082
:100FA000050300000704000010B52D492D4803F08B
:100FB000C1FE2D4B102212212C4804F08DF804465E
:100FC0002A48C1690220FFF748FA28482449C01F6F
:100FD000027818390A71244A40784871603A508979
:100FE0000880508B488001208871C53A13780B73B4
:100FF00052784A731C4A203A52890A8100224A8157
:10100000887310310320FFF728FA15490320183997
:10101000FFF7F5FC204610BD30B5154D0020039CB0
:10102000EA4202D1032901D00A2030BD012B01D0B0
:101030000D2030BD0D4A2178083A117030BD0C48A2
:1010400010B512180020029C002A06D1032904D1F1
:10105000064808380078207001201880002010BD54
:1010600090690020FFFF00008C4500206C440020A8
:10107000B3D5FFFF10B54649464803F05BFE464B2B
:10108000102218460621603804F026F810BD4249A7
:10109000683908607047022070473F4B02460020C5
:1010A000643B002A03D0012A03D0022070471A882B
:1010B00000E05A880A8070473EB50446344903F080
:1010C000FDFFC0071ED000252B4601221B21204614
:1010D000009504F007FC0290002813D02E486946C2
:1010E0002038408B88800120C8800298002205703B
:1010F00001A9204604F0DCF9002803D01B2101A837
:1011000004F036FC3EBD00207047FEB5089E00246A
:101110001546002E01D00B20FEBD4F687A783F782F
:1011200012023A431D4FBA420ED1042B01D00D24B6
:1011300016E0C8681A46294612F072FC16490120CA
:101140006839096888470BE0154CA24207D1012293
:10115000019200962A4603F053FE044600E00A245A
:101160002046FEBD10B504460A48401E84420DD0FC
:10117000012907D0022909D1012120460EF08AFA5F
:10118000002803D10249204603F0D4FD10BD000021
:10119000A0690020FFFF0000084600204F2A000041
:1011A000022900000448804704480047FEE7FEE7A4
:1011B000FEE7FEE7FEE70000C1110000910000001D
:1011C00010B5FA4857210170A8210170F74A88210B
:1011D000403A1181002101700A2000F025FC012015
:1011E00000F06FFB10BDF0B5F04EF04D0427572214
:1011F000A824203E403DED49030008F0CFFF0D0834
:101200000E161B1F24282C32373C41462F000A7033
:101210000C70F07BFB22104003E00A700C70F07B36
:101220003843F073C820288118E00A700C705120F0
:10123000C000F8E70A700C70DD48F4E70A700C7023
:1012400081208000EFE70A700C708820EBE70A70BD
:101250000C700220E7E70A700C702F8100200870E4
:10126000F0BD0A700C7093208000DCE70A700C70EF
:10127000CF484D30D7E70A700C7095208000D2E738
:101280000A700C704B20C000CDE70A700C70C84883
:101290005C30C8E7C54810B540380089C1B20B06BC
:1012A0009A0FC448022A05D0012A04D09A0F06D00A
:1012B0007D20000210BDC906C90EBF4801E0C90665
:1012C000C90E00F059FD10BDB84A57211170A82170
:1012D0001170B64940394B150028088904D01843CD
:1012E00008810020107070479843F9E7AF4A5721F2
:1012F0001170A8211170AD4920390028C87B05D094
:1013000004231843C873002010707047FB23184053
:10131000F8E7A6498A7B800792089200800F024373
:1013200057200870A82008708A7300200870704742
:101330009E498A7B8F231A40000102435720087080
:10134000A82008708A73002008707047974A203AD6
:10135000917B800789088900800F014393485723B8
:101360000370A823037091730021017070478F4AA6
:10137000203A917B0907090F000101438B4857234D
:101380000370A82303709173002101707047FEB5AC
:101390008648002740380089FE1EC0B201068A0F29
:1013A000022A4CD00124A403012A4BD0890F55D026
:1013B0000524002000902005000D01907B48203876
:1013C000848900267949572330460B70A8250D7073
:1013D00001228A74754957220A70A8220A70734A3A
:1013E000203A948100220A708A7C9207FCD50A8AEE
:1013F0008A7C9207FCD48A7C9207FCD5098A019AE0
:101400007F1C891A0DB2FFB2002D35D029467143D9
:1014100005D5012832D0411C30D000282ED02E46D0
:1014200002943046009900F0BDFC00B2211A8CB243
:1014300002998C4247D1002D43DD641C42E05F4C91
:101440000096B8E7C506ED0E29465D4800F094FC0D
:101450000019C40B24202946C04309E0C506ED0E3F
:101460002946584800F088FC0019C40B294630462C
:1014700000F098FC00B29DE70020FEBD002E03DACC
:10148000761EF04306B202E06D1EE84305B2B54297
:101490000FDD464857210170A8210170434A029987
:1014A000203A9181002101707D20C0007043019994
:1014B00003E07D20C0006843114600F073FC80B259
:1014C000FEBD641EA4B2142F84D3FF20FEBD70B5F0
:1014D0000D461446182100F04FFC83B2E120C000F5
:1014E00041431E20454348196108401881B2E00776
:1014F00001D00120C0030A0402432C495720087080
:10150000A8200870294C403C636328482038437C5D
:1015100080252B4343746263427C40231A43427408
:101520000020087070BDF7B5064620480D464038CB
:10153000C06B84041D48A40C2038418B008B012211
:101540004900D203904201D3012000E000200F188F
:10155000E1210901384600F00FFC1822544300191C
:10156000306008463C2100F007FC28803C213846CA
:1015700000F002FC02980180FEBD0C4957220A705F
:10158000A8220A70094A403A506308482038427C31
:1015900040231A43427400200870704703494039C1
:1015A000886B8A6B8242FBD170470000401000407C
:1015B000020200000048E80100389C1C13130000E0
:1015C00000180D8F0068890910B5304A5721117035
:1015D000A82111702D4920394B7CE82423404B74FD
:1015E0004B7C1024204303434B740020107010BD2B
:1015F00000B50346FFF7D2FF2549C018884201D93C
:10160000494240180104090C02D001210904401884
:101610001E4957220A70A8220A701C4A403A506399
:101620001A482038427C20231A4342740020087054
:1016300000BD0021002802D0012802D002E02021B4
:1016400000E01021114857220270A82202700F4AB0
:10165000203A537C8B43537400210170A4E70B495B
:1016600020390028087C02D0402108409CE7C009AE
:10167000C00199E705492039002804D0012893D1F9
:101680001020087490E72020FBE700004010004085
:101690000000C0A800B5524A0B0008F07FFD050409
:1016A000071016191F00516B81430AE0516B8143EB
:1016B0005163116B01431163116A81430DE0516B5A
:1016C00001435163116B8143F5E7516B814301E0A5
:1016D000516B01435163116A0143116200BD404ADD
:1016E00000B540320B0008F059FD0504071016192B
:1016F0001F00516981430AE05169814351611169B9
:1017000001431161116881430DE051690143516149
:1017100011698143F5E75169814301E05169014352
:10172000516111680143116000BD2D4A002906D0A6
:10173000012907D0022908D0032913D10CE0918A8E
:10174000814304E0918A814308E0918A01439182B8
:10175000D16A0143D16205E0918A01439182916A85
:10176000014391629083118A0143118270471C4B9F
:101770001B4A4033002906D0012907D0022908D08E
:10178000032913D10CE0D18A814304E0D18A81433B
:1017900008E0D18A0143D182D9680143D96005E0CC
:1017A000D18A0143D182996801439960D083518ADB
:1017B0000143518270470A4A803A0028108B01D0B9
:1017C000084300E0884310837047054A803A0028A8
:1017D000508B01D0084300E08843508370470000DD
:1017E00080100040F8B5624D5726614CA827203D77
:1017F00000282670277028880ED0211508432880DD
:101800000A2000F011F92670277028886115084316
:10181000288000202070F8BD032149028843F7E7A3
:10182000F0B5534C57261C228B07514DA8270A4070
:101830009B0F403C00282E702F7010D0080603D557
:10184000E07BFD210840E073A07A1043A072484875
:101850002038C17B1943C17300202870F0BD0806F1
:1018600003D5E07B02210843E073A07A9043A07285
:101870003F482038C17B9943EDE730B53C4C5723B6
:101880003B4AA825403C002813701570E06804D03E
:101890008843E0600020107030BD0843F9E730B5A0
:1018A000334C5723324AA825403C0028137015704A
:1018B000A07B04D00843A0730020107030BD884383
:1018C000F9E7F8B52A4D5726294C0021A827203DD5
:1018D0000028267027700ED0012068712871002022
:1018E0002070012000F0A0F8267027700D202871CC
:1018F00000202070F8BD29712170F8BD1D480169D4
:1019000004229143016130BF7047194B57241C706A
:10191000A8251D7016494039887B0822104388731A
:101920000920134E0003203E308000271F70886B73
:101930008A6B8242FBD1104A0A30904201D952424E
:1019400080180204120C02D00122120480183022E6
:1019500032741C701D7048632F2070741F701C70CF
:101960001D70052008811F7040BF20BF20BFFEE70B
:101970004010004000ED00E00000C0A83C490628EF
:1019800005D0497901228240114008467047087805
:10199000082108407047364857210170A82101707E
:1019A0008179012211438171002101707047314911
:1019B0000968016000202F49C043803108607047EA
:1019C0002C49086070472C48806970472849572285
:1019D0000A70A8220A700028887905D004221043D2
:1019E0008871002008707047FB221040F8E72049FA
:1019F00057220A70A8220A700028887905D002228E
:101A000010438871002008707047FD221040F8E7ED
:101A1000174857210170A8210170817910221143C4
:101A2000817100210170704700220AE0022101E06B
:101A300000BF00BF0B46491E89B2002BF8D1521CD3
:101A400092B28242F2D3704770B500247D260546DB
:101A5000F60004E03046FFF7E7FF641CA4B2AC4296
:101A6000F8D370BD0549CA7A082AFCD008727047BD
:101A70004010004000E100E000E000E000340040E1
:101A800010B50446FFF706FC0A214843C00821466A
:101A900000F072F90A21401D00F06EF92249888198
:101AA00010BD10B5E1204002FFF7EAFF1E48872174
:101AB00081700321C170402141700121817310BDEB
:101AC00019498A789206920E800102438A70704703
:101AD000154A0028507806D0084350701078082125
:101AE0000843107070478843507070470E4980203B
:101AF000487070470C4A07E0D37A082B04D003786B
:101B00001372491E89B2401C0029F5D17047014665
:101B10000020054A04E0137A401C0B7080B2491C77
:101B2000937A002BF7D170470034004010B5FFF7CF
:101B30002EFC022801D9FFF72AFC10BD30B556490A
:101B4000CC7E0B7E4A7EC87E80252843C8760F2037
:101B5000087621204876887E012528438876887E6D
:101B6000C007FCD1888BCC760B764A7630BD30B579
:101B70008DB0122249A14E4811F044FF002841D0F7
:101B8000454857210170A82101705121424AC900DE
:101B9000403A1181002101704748464A4261474A54
:101BA0000724D3691B021B0A45042B43D3618161BF
:101BB00004610169022291430161342200216846D7
:101BC00012F008F83E4800900120400369468880E2
:101BD0001B20C873052008740120487415208874E0
:101BE000FB20800202900D20087736480890364886
:101BF0000A90084601F036F9010007D033A008F03A
:101C0000A5FAFEE739A008F0A1FAFEE70DB030BD55
:101C100070B50C4609040AD512F020F8002801D04E
:101C200011F0F4FF01212046C903484070BDE007D0
:101C300002D00120604070BD314DA00405D501F0F7
:101C40007DF901262F4A760308E060040DD52EA009
:101C500008F07CFA7D22D2010126B60331462878AD
:101C600012F0D8F92046704070BD002070BD10B54C
:101C7000264808F0F1F8224C207000F063F862B6B4
:101C8000204A01214903207812F0C4F910BD10B593
:101C900001F03EF810BD00004010004043483537C9
:101CA000785F424C455F4C49425F56312E3600000A
:101CB000B4420100FEFFFF0000E000E004ED00E0A0
:101CC000E4480020C71900003D1B00004C49422099
:101CD000696E6974206572726F7220636F64653A11
:101CE000202578202E2E2E0A0000000068656164F1
:101CF0002066696C65206572726F722E2E2E0A0046
:101D00001546002000EE02002A200000111C0000F1
:101D10000104090C02D0012109044018144957227A
:101D20000A70A8220A7012494039486311490020FC
:101D3000086070470E493020203908740D49012091
:101D40000860704710B50A4857210170A82101703A
:101D500007492039CA7B07231A43CA73002101703F
:101D60000A460846FFF7B3FB002008F0A5F910BDAE
:101D7000401000401846002030B50B4601460020B8
:101D80002022012409E00D46D5409D4205D31D4681
:101D90009540491B2546954040191546521E002D79
:101DA000F1DC30BD70B500242546002801DA01249D
:101DB0004042002901DA01254942FFF7DDFFAC422C
:101DC00000D04042002C00D0494270BDF0B51FB495
:101DD00086B000200090019002900698069980B28B
:101DE00004900798090C020400141143079000277F
:101DF000089D099806913E463C4603900398A9B277
:101E00000204000C039004982D0C15434843002154
:101E1000224600F018F8C719714110340E46402CC4
:101E2000ECDB3846029A00F00EF8009A019B80180D
:101E30000090594102980191103002904028CCDB6B
:101E400000980BB0F0BD10B5202A04DB0146203A03
:101E50009140002010BD914020239C1A0346E3408E
:101E60001943904010BD03460B439B0703D009E084
:101E700008C9121F08C0042AFAD203E00B780370C5
:101E8000401C491C521EF9D27047F0B51FB40646DB
:101E9000002082B005464024019100901BE001998A
:101EA00022460F46304600F033F8049A059B801A0C
:101EB000994110D3104619462246FFF7C4FF361A3F
:101EC0008F410197224601200021009FFFF7BBFFB1
:101ED00038184D4100902046641E0028DFDC019B2D
:101EE00000982946324607B0F0BD0000064C012597
:101EF000064E05E0E36807CC2B430C3C98471034B2
:101F0000B442F7D3FEF7C8F8AC460100DC46010046
:101F100010B5202A04DB0846203AD040002110BD2D
:101F20000B46D340D0402024A21A914008431946C2
:101F300010BD70B58C180578401C6B075B0F01D184
:101F40000378401C2A1106D10278401C03E0067871
:101F50000E70401C491C5B1EF9D12B0705D40023D1
:101F6000521E0DD40B70491CFAE70378401CCB1AA3
:101F7000921C03E01D780D70491C5B1C521EF9D5A4
:101F8000A142D8D3002070BD70B50D46014614465D
:101F9000104600F0F5FF0E4830C004F073F9002041
:101FA00000F00EFE012407F0C3FE07F0A3FE06F0CA
:101FB00009FD204600F004FE641CE4B20A2CF2D3B2
:101FC00007F0B6FE07F096FE0A2000F0F9FD70BD9E
:101FD000D848002010B5124C2068C0051FD503203A
:101FE000206000200821401C2268C0B20A43226001
:101FF0000EE02268920510D4222807D90948026B06
:10200000002A0AD001210320904706E0401CC0B2FC
:102010002268D205EDD50028E5D10020206010BD52
:1020200080C30040CC690020F8B514460D46064632
:10203000FFF7D0FF504F3B681868062188431860AF
:102040007178307809024018B178F27809041206E4
:102050008918401898627179307909024018B1796D
:10206000F2790904120689184018D862717A307A18
:1020700009024018B17AF27A090412068918401848
:102080001863717B307B09024018B17BF27B090435
:102090001206891840185863697828780902401890
:1020A000A978EA78090412068918401898616979B4
:1020B000287909024018A979EA79090412068918D1
:1020C0004018D861697A287A09024018A97AEA7A10
:1020D00009041206891840181862697B287B0902D6
:1020E0004018A97BEA7B0904120689184018586237
:1020F00058680221884358605A68012002435A6098
:102100001A6802431A6058688007FCD558688843EB
:1021100058609869207038688069000A6070386873
:102120008069000CA07038688069000EE070386823
:10213000C1692171C169090A6171C169090CA17183
:10214000C169090EE171016A2172016A090A6172AD
:10215000016A090CA172016A090EE172416A2173D8
:10216000416A090A6173416A090CA173406A000E51
:10217000E0730020F8BD00005848002070B50C4600
:102180000546FFF727FF284802681068202188438A
:10219000E907890E084310608034A06C1061E06C80
:1021A0005061A0699061E069D061206A1062606A44
:1021B0005062A06A9062E06AD062206B1063606B2C
:1021C0005063A06B9060E06BD060D168E36B174800
:1021D000994204D0026B002A1ED0202107E0916AA8
:1021E000A36A994206D0026B002A15D02121032050
:1021F000904711E0D169E369994204D0026B002A4B
:102200000AD02221F3E71169A36C994206D0026B30
:10221000002A01D02321EAE7012070BD1068402187
:1022200008431060002070BD58480020CC69002091
:1022300070B50C460546FFF7CDFE284802681068C9
:1022400020218843E907890E084310608034206C00
:102250001061606C5061A0699061E069D061206A92
:102260001062606A5062A06A9062E06AD062206B7D
:102270001063606B5063A06B9060E06BD060D168BE
:10228000E36B1748994204D0026B002A1ED010213C
:1022900007E0916AA36A994206D0026B002A15D022
:1022A00011210320904711E0D169E369994204D0DC
:1022B000026B002A0AD01221F3E71169236C9942BC
:1022C00006D0026B002A01D01321EAE7012070BD7D
:1022D0001068402108431060002070BD584800205D
:1022E000CC69002010B504F0AFFE024903F041FCB8
:1022F000002010BD0604000010B50EF05BF910BD03
:1023000008B5002808D0002906D0002A04D010887B
:10231000002801D0002008BD1220694608706A46D6
:102320000121034803F021FC6946087808BD00003C
:10233000350C000008B504F0C1F9694608706A461A
:102340000121034803F011FC6946087808BD00002C
:102350002720000008B504F0FBF9694608706A46BA
:102360000121034803F001FC6946087808BD00001C
:102370001120000008B504F033FB694608706A4676
:102380000121034803F0F1FB6946087808BD00000D
:102390002920000008B504F029FB694608706A4648
:1023A0000121034803F0E1FB6946087808BD0000FD
:1023B00010200000FEB508AF70CF6F4670C704F064
:1023C0003BFB0446024903F0D4FB2046FEBD00005F
:1023D0001320000008B504F027FE694608706A461D
:1023E0000121024803F0C1FB002008BD0E200000BF
:1023F00038B5044605F030F8694608704C70200A7C
:1024000088706A460321024803F0AFFB002038BD04
:102410001B20000038B5044605F036F86946087000
:102420004C70200A88706A460321024803F09DFB25
:10243000002038BD1A2000000EB500A8013005F0BC
:1024400074FB694608706A460921024803F08DFB57
:1024500000200EBD1820000008B500A8013004F0CF
:1024600083FF694608706A460421034803F07DFB38
:102470006946087808BD00000220000038B504460F
:1024800005F0AEFB694608704C70200A88706A46F9
:102490000321024803F069FB002038BD2120000021
:1024A0007FB5044608A861C80090029601952046B1
:1024B00005F0AEFB694608734C73200A887303AAC3
:1024C0000321034803F051FB002004B070BD00005D
:1024D0002020000008B505F09BFE694608706A469A
:1024E0000121034803F041FB6946087808BD00005C
:1024F0002D20000008B505F029FF694608706A46DE
:102500000121034803F031FB6946087808BD00004B
:102510000820000008B505F0A1FE694608706A466B
:102520000121034803F021FB6946087808BD00003B
:102530000A200000F0B585B00AACF0CC03976F46D6
:1025400070C705F023FF6946087404AA01210348F7
:1025500003F00BFB6946087C05B0F0BD06200000C7
:1025600008B505F069FF694608706A46012103480D
:1025700003F0FBFA6946087808BD0000052000005A
:1025800008B505F097FF694608706A4601210348BF
:1025900003F0EBFA6946087808BD00002E20000021
:1025A00008B505F09DFF694608706A460121034899
:1025B00003F0DBFA6946087808BD00000C20000033
:1025C00008B505F0D1FF694608706A460121034845
:1025D00003F0CBFA6946087808BD00000920000026
:1025E00010B506F028F8024903F0C3FA002010BD28
:1025F0001920000010B504F087FF10BD1CB500A81D
:10260000013005F0A1FA694608706A4607210348BF
:1026100003F0ABFA694608781CBD00000910000001
:1026200010B505F04DFD10BD0A7802708A78427031
:102630004A88120A82700979C170042070470A78AA
:1026400002700988090A41700220704708888004D6
:10265000000C70478A78027088780128088804D0B6
:1026600012214843401C80B270478000FAE70A7884
:1026700002700A88120A42704888801C80B2704733
:102680000A7802700A88120A42708A7882704A8830
:10269000120AC2708888001D80B27047088870478F
:1026A0008A780270088849884843401C80B2704785
:1026B0008A780270088849884843401C80B2704775
:1026C00008887047088870477FB515460446022978
:1026D00001D0102903D1022B04D0102B02D00020EE
:1026E00004B070BD994202D10A46294607E010297C
:1026F000694607D000F00EF810226946284611F00E
:1027000081F9EDE7104600F005F8102269462046F1
:10271000F5E7000070B50C4605000CD0002C0AD07F
:1027200010220649204611F07BF92878207368783A
:102730006073012070BD002070BD00005C4301008B
:1027400008B500220B4600920122024907F0F4FE70
:1027500008BD00002926000008B50A88172A07D3FB
:1027600000220B4600920322024907F0E5FE08BD55
:10277000022008BD3F26000008B500210B461922A3
:10278000009107F0D9FE08BD38B5054608880C460B
:1027900000280DD0606800280AD0012111F0EEF861
:1027A0000090234607220349284607F0C5FE38BD9E
:1027B000022038BD4D26000038B5054688780C4605
:1027C000012801D0022810D1208800280DD060688F
:1027D00000280AD0022111F0D1F8009023460522EA
:1027E0000349284607F0A8FE38BD022038BD000086
:1027F00055260000064910B5884202D103F0D2FDEB
:1028000010BD0CF097FE0028FAD1172010BD000073
:10281000FEFF000038B505464A6800200C46002A35
:1028200003D00321104611F0A9F8009023461D2281
:102830000249284607F03CFE38BD00006F26000024
:1028400038B505464A6800200C46002A03D003210B
:10285000104611F093F8009023461B2202492846A7
:1028600007F026FE38BD00006F2600000248002158
:1028700001604160704700007C4800200098022BF6
:1028800001D0042070475178127809021143018069
:10289000002070470098012B01D004207047117868
:1028A00001700020704770B5049C1E461546062B2B
:1028B0001BD368782978000208432080E878A9783B
:1028C000000208436080022020710246291D601D1D
:1028D00011F0A6F8B01F2081062E03D0AD1DE560D3
:1028E000002070BD0020E060FAE7042070BD009871
:1028F000042B01D004207047517813780902194342
:102900000180D178927809021143418000207047FC
:10291000F8B584890D46002C2BD0866837783906A7
:1029200001D4002010E00D2C23D30C3CA4B23119AB
:102930000091408823463246012107F063F90028C0
:1029400001D0022000E0012079062870C90FBA06E4
:102950006970920EAA70641E2204120CAA8002D022
:10296000761CAE6001E00022AA60022803D1002993
:1029700001D00120F8BD0020F8BD10B50298042B4D
:1029800014D351781478090221430180D1789478C6
:10299000090221434180191F8180042B02D0121D9E
:1029A000826001E000218160002010BD042010BD84
:1029B0000098042B01D00420704751781378090245
:1029C00019430180D1789278090211434180002097
:1029D000704710B502981146062B03D0142B03D074
:1029E000042010BD022200E0102202714A780B7808
:1029F00012021A430280CA788B7812021A4342806C
:102A00000279401D091D11F00BF8002010BD00983F
:102A1000D90706D1022B04D059088180026000201A
:102A20007047042070470098022B01D004207047A3
:102A3000517812780902114301800020704710B5C7
:102A4000029C022B11D3207261725078117800021F
:102A500008432080981E6080022B02D0921C626086
:102A600001E000206060002010BD042010BD0000C7
:102A700038B5054688680C46002802D0052110F0BC
:102A80007DFF0090234617220249284607F054FD97
:102A900038BD00008126000038B5054648680C4660
:102AA000002802D0012110F069FF009023460D227A
:102AB0000249284607F040FD38BD00009D26000071
:102AC00038B5054608880C4600280DD060680028F7
:102AD0000AD0022110F052FF009023461122034930
:102AE000284607F029FD38BD022038BDA126000088
:102AF00038B5054608880C4600280DD060680028C7
:102B00000AD0022110F03AFF00902346092203491F
:102B1000284607F011FD38BD022038BDB12600005F
:102B200038B5054648680C4600280AD0012110F047
:102B300025FF009023460F220349284607F0FCFC9E
:102B400038BD022038BD0000C126000038B505465A
:102B50004A6800200C46002A03D00121104610F0DC
:102B60000DFF009023460B220249284607F0E4FCA3
:102B700038BD0000C526000001490860704700000C
:102B80007C48002070B5054608480C46854205D0B3
:102B9000172C03D303F006FCA04201D2012070BD24
:102BA000214628460CF086FD70BD0000FEFF0000A7
:102BB00008B500210B461322009107F0BDFC08BDAB
:102BC000F0B50D4A002180000C4D1668844662461F
:102BD0005218930000208A0092191F18145CEF5DB0
:102BE0007C401454401CC0B20428F6D3491CC9B21E
:102BF0000429ECD3F0BD0000D8480020C06C0020B0
:102C000004480349006801600349C162704700003D
:102C1000A52208015C480020784E010070B52B49C0
:102C2000002008602A4800892A4CC0B28109022984
:102C300004D0012908D0810916D026E0D020A08038
:102C40000820E080E8201FE0C506ED0E2D20294673
:102C50008001FFF791F8A08029467820FFF78CF8D3
:102C6000E08029461C480DE0C506ED0E2946C0202F
:102C7000FFF782F8A08029460820FFF77DF8E08062
:102C80002946E820FFF778F82081154913480860A5
:102C90001549144808601649144808601649154833
:102CA000086017491548174C086017492068012229
:102CB000D202C8608018086100F040F9607D0028E9
:102CC00002D112492020086070BD00003C4600205F
:102CD00000100040006A0020980D000000C0004075
:102CE0006048002000C300405848002000C2004057
:102CF0003846002000D000406448002000C1004059
:102D00005C480020CC690020206A002000E100E03F
:102D1000F0B54F48006881680026C9054D4C012771
:102D20004D4D002923DA81683A0291438160217870
:102D3000490605D5494B996BA1609A6B9142FAD12E
:102D40002178394321706670E179062901D05D212F
:102D50000165286800280AD001690A6840690243B1
:102D60000A60286801680A68806802430A60384B74
:102D700018688168890521D5816801225202914332
:102D80008160A0783843A070E67035480068C16A59
:102D900089088900891CC1620168D204114301605D
:102DA000286800280AD041680A68806802430A60DF
:102DB0002968C868026849690A430260186881681E
:102DC000890715D58168022291438160E770A6705A
:102DD0005D210165286800280AD001690A684069F8
:102DE00002430A6029680868026889680A43026029
:102DF00018688168C90713D0816849084900816053
:102E000026706770286800280AD041680A688068C0
:102E100002430A602868C1680A68406902430A6080
:102E200018688168C90603D58168102291438160C2
:102E30008168490703D581680422914381608168D4
:102E4000090703D58168082291438160F0BD000025
:102E500038460020206A00203C4600200010004038
:102E60005C48002010B504460068002823D00121EA
:102E7000000C490388421ED1A08800281BD02046A0
:102E80000622FF21163010F0AEFD012815D0A288D1
:102E90000021206810F09EFE34220021264810F008
:102EA00099FE34222146244810F0BAFD2248818937
:102EB000002904D006E0022010BD032010BD01212E
:102EC00049028181827B0121002A00D18173C27B6A
:102ED000002A01D11B22C273027C002A01D10522E3
:102EE0000274427C002A00D14174817C002901D106
:102EF00015218174817F002901D128218177C17C2E
:102F0000002908D0827FE17C52088918C174617F52
:102F1000002904D005E0817F49085031F6E70421FB
:102F20004177806A002803D08047034934314881C3
:102F300006F04CFF002010BDCC69002010B500F059
:102F40006BF803F09DFB05F07FFDFFF759FE0A4C7F
:102F50005D202168086505F041FE06F0FFFB05F0E5
:102F600005FE05F0D7FD2168002008650349C871FA
:102F7000FFF730F810BD000038460020206A00201E
:102F800000228B5C8354521CD2B2102AF9D37047B2
:102F900070B50E4B00209989002901D10C49998107
:102FA0000E210124A4039A8915462540CD405204E0
:102FB000120C0543E8B25604D50BF60F75401543C5
:102FC000491EC9B29D810629EDD870BD006C002054
:102FD000FF7F000070B50E4B00205989002901D1F8
:102FE0000C49598108214C015A8915462540CD408C
:102FF00005435200E8B2550A56097540ED07ED0F3A
:103000001543491E09065D81090EEDD170BD000012
:10301000006C0020FF0100000A4809490068CA68E6
:103020000261CA68426109698161C16182680121E6
:1030300049030A438260C2680A43C26070470000C5
:10304000206A00206048002030B5104A0346517ABB
:10305000FD20842454720E4CA568002D07D0A57B5A
:10306000002D04D0A489E51FFF3DFA3D02D0517226
:10307000FF2030BD7D24E402A34205D35360A62087
:103080001072907A40235840517230BD00180040B1
:10309000CC690020F8B500240F4E274613E0F06BF2
:1030A000250128180622FF2110F094FDF06B06225E
:1030B0002818FF21801D10F08DFDF06B28188781E6
:1030C000641C8773E4B2307E8442E8D3002010F0A1
:1030D00061FE307E7076F8BDB447002070B50C46B6
:1030E0000146012080020A1A00252B48130007F030
:1030F00055F820111316181A1D1F21232527292BD7
:1031000032343648393B3D3F4348484848484848B0
:1031100048464148007800E04078207039E08078E7
:10312000FBE7C078F9E710221C4910E00079F4E7CA
:103130004079F2E7006A13E08079EEE7C079ECE7C6
:10314000007AEAE7407AE8E7144910221031204675
:1031500010F066FC1DE0807ADFE7C07ADDE7406AA8
:10316000206016E0007BD8E7407BD6E7807BD4E781
:10317000407CD2E7807CD0E707F044FFCDE7807D3C
:10318000CBE7192904D2084601F056FA208000E066
:103190000225284670BD0000B4470020346B002093
:1031A00010B5044600F0D4F80248C47508F064F87D
:1031B00010BD0000B4470020FFB58FB006460020C8
:1031C0000C900D901F460CAA304600F0B5FA454D04
:1031D0000446287E84425AD2204608F02DF806463E
:1031E000042F04D0A879022803D0002002E0287818
:1031F000F9E7012000903B4632462146119807F03E
:10320000D9FE1422002101A810F0E4FC204606217A
:10321000484300902430C0B201AA102110F018FEDB
:10322000002813D11022FF2101A810F0DCFB002898
:103230000CD1009805AA2530C0B2042110F008FE78
:10324000F107C90F01AA119801F068FC7034E0B2CF
:1032500006AA182110F0FCFD002811D106A807F0DD
:10326000FDFF0024A10006A808180188002903D04A
:103270008278119801F08EFF641CE4B2062CF1D321
:10328000B00706D5E97D119801F072FF01E0082F23
:1032900002D0042F13D021E0A87902281ED10022E9
:1032A0003146119807F0C0FDA86A002816D043687F
:1032B000002B13D000221146119898470EE0287871
:1032C00002280BD129791198002900D001216A78B0
:1032D000002A00D00422114301F0E6FB002013B0C5
:1032E000F0BD0000B4470020F8B501F039FA00281D
:1032F0002BD1164D0026E87C012801D000241CE0CB
:1033000007F0CCFEEE7400202A7EE96B04E0030196
:103310005B18401C9E73C0B29042F8D310E0E86B7B
:1033200027013818807B012805D1204607F0C8FE08
:10333000E86B38188673641CE4B2287E8442EED3AE
:10334000502010F049FD07F097FFF8BDB44700206A
:10335000F8B5354EFF20F07500273776334CF7630C
:10336000A07B30214843422110F076FBF063002817
:1033700025D02046807B410040183076002413E0A1
:10338000F06B250128180622FF2110F023FCF06BBA
:1033900006222818FF21801D10F01CFCF06B281855
:1033A0008781641C8773E4B2307E8442E8D31F486F
:1033B0008068002801D0B77601E08020B076307EAA
:1033C00070760124776334707770B770F7701022CD
:1033D0000021174810F0FEFB3771772575713762B1
:1033E000B471F771124837727772102200211030D1
:1033F00010F0F0FBB772F5727762377305207073C7
:103400001020B073F77302203074B762F76237632D
:103410007774F774347504487475B4750549483089
:10342000016005494160F8BDB4470020CC69002027
:10343000346B002089B5000051B5000070B5002440
:10344000054600290BD108491046FEF795FC0846B1
:10345000294601F0E1F9040003D00121284601F0DA
:1034600085FB204670BD000040420F0010B50649A4
:103470000C46483CA162E062E17D182001F034FB7B
:10348000E07D01F023FE10BDFC47002070B5264D05
:103490000C4608040FD5E87D10F0E0FB050006D0CF
:1034A00007F090FF002802D0284610F0AFFB012063
:1034B000C003604070BDA0070BD50021084607F08F
:1034C00015FC02214C40002825D1E87D10F050FC6D
:1034D0001FE0E00721D0686B808807F0A5FF01217D
:1034E0004C40002817D0A86A00280DD04368002B54
:1034F0000AD0686B002280889847A96A686B00220E
:103500004B68808803219847287D10F081FC07F0E4
:10351000DFFB204670BD0121D7E7600702D50420FC
:10352000484070BD002070BDB44700207FB5044600
:1035300080787F4D801F030006F030FE0AF4F7F715
:10354000A41306F0F778B9F7A96A2046002907D036
:103550000C68002CFBD0437B027B4189C01CA04738
:10356000E3E060780026002847D1A079C00744D066
:10357000686B002841D110220021684610F02AFB18
:103580006169002903D006226846103107E0A0884F
:103590000BF0FCFE0028E3D0811D0622684610F0E7
:1035A0003FFA69468889A1794907C90F08436946E6
:1035B000888107F027FD297E88420BD1A87D00284D
:1035C00001D0FFF767FD5B48026B002A02D00121A2
:1035D0000820904707F016FD297E8842A87E02D178
:1035E0000121084301E040084000A87621466846D2
:1035F00007F07CFB002812D01526A86A002855D0B9
:103600004368002B52D06278A08801219847002E91
:103610004CD0A96AA0884B683246032173E002218E
:10362000E87D10F0A5FB002004B070BD607806288E
:1036300017D1A0880BF0AAFE060012D0287C012822
:1036400004D0022808D003280BD114E07179A08897
:10365000002207F0E9FB04E0A1883078052201F0A0
:1036600095FAA86A002860D04368002B5DD0627884
:10367000A088022147E0002241201146000100F00D
:10368000F7F8E9E7E0780022211D00F055F8297EDF
:1036900088424AD20621484325302246C0B20C3225
:1036A000042110F019FC287D10F0B2FB3DE0287BCE
:1036B000002802D0A088697B28E028780028A0880C
:1036C00023D00BF063FE06002FD0A07AC0070BD0EA
:1036D0007079002808D0A189890505D46A46B11DF2
:1036E00000F02AF8002814D022467179A088083208
:1036F00007F09AFBA86A002817D04368002B14D063
:103700000022A088114698470FE0052101F02EFA0B
:103710000BE0A0880321F9E700E003E0A08800F0B7
:1037200031FA02E0A088FFF7DFFD01207CE700000E
:10373000B4470020CC690020F0B52E4E85B0347E11
:1037400015460F46002806D0012804D0022811D0C3
:1037500003284BD121E0084607F026FD317E0446C0
:10376000884243D2002D41D006223946284610F027
:1037700057F93BE000240BE0F16B200140180622D2
:103780003946801D10F03EF9002826D1641CE4B2B1
:10379000307E8442F0D3C4B21FE0002419E02046FA
:1037A000062148432330C0B26A46102110F050FB76
:1037B00000280CD11022FF21684610F014F90028CF
:1037C00005D13946684601F03DF9002805D0641C52
:1037D000E4B2307E8442E2D3DDE7307E844205D21B
:1037E000002D03D02946204607F006FD204605B0EF
:1037F000F0BD0000B4470020F8B50E461949152564
:10380000194F884214D1002409E032460221204693
:1038100007F012FC002800D00025641CE4B2387EBA
:103820008442F2D3002E1BD010480BF0CBFE17E0E1
:103830000BF0ACFD040012D060790022A11DFFF74F
:103840007BFF397E884204D23246022107F0F4FB26
:103850000025002E04D0204607F050FD00E014257E
:103860002846F8BDFFFF0000B4470020FDB200006D
:10387000F0B50746012080021546381A89B00024A9
:10388000BC4ABD4E030006F089FC2011181F262DEE
:10389000333A3F464D545B626970757CEFEEEDEC58
:1038A000EBEA89E9E8AAAAF3F6E5E4EB012971D18C
:1038B000287802286ED8307059E10129F7D128788C
:1038C0000128F7D8707052E10129F0D12878042836
:1038D000F0D8B0704BE10129E9D128780128E9D866
:1038E000F07044E11029E2D110222946A348ADE04E
:1038F0000129DCD128780128DCD8307137E1012991
:10390000D5D12878707132E10429D0D1286890424D
:10391000D0D830622BE10129C9D128780228C9D832
:10392000B07124E10129C2D128780128C2D8F071F0
:103930001DE10129BBD128780428BBD8307216E1DB
:103940000129B4D128780128B4D870720FE1102968
:10395000ADD18A4810222946103077E00129A6D13E
:1039600028780128A6D8B07201E101299FD12878D2
:10397000F072FCE004290DD1286890420AD87062E8
:10398000F5E0002906D100F0EBFE002803D001206D
:10399000F074ECE074E007F081FB1CE007296FD1C4
:1039A0000622691C684610F03BF828780022694618
:1039B000FFF7C2FE0546307E854239D200F0D0FEC8
:1039C000002805D0F26B0120290189188873CEE008
:1039D000284607F075FB502010F0FEF996E0072905
:1039E0004ED10622691C07A810F01AF82878002288
:1039F00007A9FFF7A1FE317E88421BD2062148436A
:103A000005462135E8B26A461C2110F021FA00284B
:103A10000ED15B48874201D1012000E0FF206946BA
:103A2000C876E8B26A461C2110F056FA307D4BE0A9
:103A300002249CE0B07E0028FAD05148874214D17D
:103A40000120F0764C480722294640300FF0E8FF6D
:103A50008DE05EE07AE00EE00AE075E06FE067E09E
:103A60007BE04AE041E039E031E00020F0767EE0A2
:103A7000002070757BE00027012070753D461BE03B
:103A800066E028460621484306462136F0B26A46DB
:103A90001C2110F0DDF900280CD16846C07EFF28FB
:103AA00008D0FF206946C8760127F0B26A461C217B
:103AB00010F012FA6D1CEDB22F48007E8542E0D363
:103AC000002F54D02C48007D10F0A2F94FE00129BE
:103AD0003ED1287801283BD8307348E0012937D1FE
:103AE0002878092834D8707341E0012930D128782A
:103AF000C11F09292CD8B07339E0012928D1717C64
:103B000028787074002932D1012830D107F0B4FB35
:103B10002DE001291CD1B17C2878B074002903D193
:103B2000012801D107F0A8FBB07C02F0AEF81EE03E
:103B300001290DD1287803280AD8307417E001290B
:103B400006D12878307512E00120BDE7012901D0A7
:103B500018240CE02878B07509E0192F00D367E726
:103B60000229FCD12988384600F0BEFF04462046D1
:103B700009B0F0BD3F420F00B4470020346B002075
:103B80001A040000FEB5064600200190029030465F
:103B90000BF0FCFB040017D0144FB879022813D0A7
:103BA000607901AAA11DFFF7C7FD0546387E854251
:103BB0000BD2284607F040FB024601200090082364
:103BC0002946304607F0F6F9FEBDB879002807D03F
:103BD0000128F9D161790022304607F025F9FEBDB0
:103BE0000521304600F0C2FFFEBD0000B4470020B2
:103BF000F7B516491525164E174688420FD10024F1
:103C000009E03A462046019907F082FB002800D0DF
:103C10000025641CE4B2307E8442F2D313E00BF042
:103C2000B5FB00280ED04379811D00221846FFF70E
:103C300083FD317E884206D23A46019907F068FB3F
:103C4000002500E014252846FEBD0000FFFF00000F
:103C5000B447002070B50C460146032000020A1A42
:103C600000252548130006F099FA130B0D10171ABA
:103C70001E2125292B2D3133393B3D3D35373D0064
:103C8000407811E010221D4902E01C491022103139
:103C900020460FF0C5FE2DE0406920602AE016495D
:103CA00006221E31F4E7C078207023E012498278A2
:103CB0002431EDE7114902791F39E9E7407AF3E74A
:103CC000807AF1E70C4906221831E1E7C07AEBE788
:103CD000007BE9E7C0890AE0008A08E0007AE3E7B0
:103CE0004079E1E7192904D2084600F0A5FC2080BC
:103CF00000E00225284670BD08480020936B002094
:103D0000F8B5164CFF202070002565700320A070C8
:103D10000126E670062765611920E781C00120822F
:103D200020461F22294624300FF054FF204602214E
:103D3000243001704670877025711F2200210848C9
:103D40000FF048FF20460622002118300FF042FFF6
:103D50006571A571FF20E071F8BD000008480020E2
:103D6000746B0020FFB583B01C4615460E460C9FB1
:103D700003980BF00BFB002817D0C189B14207D381
:103D8000A94205D8018AA14202D1408AB8420ED088
:103D90006846068045808480C78069460D9A0398EE
:103DA00002F0D2FA002007B0F0BD1420FBE7182083
:103DB000F9E7000010B52548007F800744D0244C67
:103DC0002078FF2840D1234806F046F82070FF28CD
:103DD0003AD0214900240C602049214A0C7004216A
:103DE000117000F029FE102200211E480FF0F2FE93
:103DF000102200211C480FF0EDFE1C481E490460F3
:103E00001B48184A04701B480470072008701B48A0
:103E100010210470022010F01BF8134A1021032017
:103E200010F016F810220F4915480FF0F9FD14484C
:103E300010220D4910300FF0F3FD04210B4A084603
:103E400010F006F8002010BD182010BDCC6900202D
:103E500008480020E53E00000448002010480020EB
:103E600009480020936B0020A36B00201C48002011
:103E70001148002012480020134800201448002058
:103E8000546B002010B504F08DFB104805F0E4FFE2
:103E900002F09AFA0E4805F0DFFF00F0D9FB0D485A
:103EA00005F0DAFF01F0C6FA0B4805F0D5FF05F082
:103EB00029FD0A4805F0D0FFFFF772F9084805F020
:103EC000CBFF00F005FFFFF775FF10BD1D6500007B
:103ED0005549000041550000159A00008D3400003E
:103EE0004D4E0000FEB54A4C0D46080448D52078DA
:103EF0000FF0B4FE040040D046480078002808D0F7
:103F00002078454ED02808D0A22802D0912821D070
:103F100014E0204608F0D8FB2CE0A07800280DD053
:103F2000052807D0082809D006280BD00728F0D18B
:103F3000A0881BE0608919E0007B04E0204608F0BF
:103F4000C3FB02E0E0790828E3D1214630780FF086
:103F5000BDFE12E060780E28F0D1A0882F4988427B
:103F6000ECD1A06881784278080210430BF00EFA79
:103F70000028E1D120460FF049FE0120C00345E0B2
:103F800068040BD50421264A08460FF0A5FF2548F2
:103F900000780FF03DFF0120800337E0E80736D0BE
:103FA00021480078002830D00BF024FB1F49097FFE
:103FB0008907890F884203D30320694608700CE003
:103FC0001B486946007808701A4806220078487035
:103FD00000A8194902300FF023FD184869460078FF
:103FE0000872174800784872207800F04DFB0028CE
:103FF0000BD014490620087013490968002904D021
:104000000A68002A01D00021904701206840FEBDC7
:10401000084800200E4800200F480020051400002A
:104020001C480020C84700200B480020CC69002015
:10403000114800201248002020480020134800208A
:104040001448002010480020044800207CB5144685
:104050000D4601F0EFFA002D02D02846FFF706FAD0
:104060000C480078002801D011207CBD002C01D024
:10407000094804600A48009008490B4801910278F9
:104080000A48084B01780A48007800F057FA0020E7
:104090007CBD000010480020044800201C4800207F
:1040A000A36B0020936B00200D48002009480020DE
:1040B00008480020F8B50C465E49164642181921FA
:1040C0000025C9015C4F130006F068F8120A1017AA
:1040D000A81C3E526970778188A8A3A8A88F98A8C9
:1040E000102C73D11022314654486CE0102C6DD145
:1040F000524810223146103065E0042C66D13068F9
:10410000786190E0012C61D1F97830784A4AF870F2
:10411000127800290AD0002807D1387A022801D065
:10412000052802D1104600F05DFA7CE000287AD024
:10413000387A012803D0032801D0042873D1012143
:1041400010460FF015FE6EE01F2C60D83A481F2273
:10415000002124300FF03EFD3748224631462430FE
:104160000FF05EFC344BBC7024332246012112E078
:104170001F2C4CD831481F2200211F380FF02AFD78
:104180002E48224631461F380FF04AFC2B4B3C711B
:104190001F3B22460021387800F03CFD48E0012C0E
:1041A00035D13078042832D878723CE0012C2ED1F9
:1041B000307803282BD8B87235E0062C27D11E485A
:1041C0000622314618300FF02BFC2CE01FE0012CAA
:1041D0001DD1307807281AD8F87224E0012C16D1A6
:1041E0003078032813D838731DE03088022C0ED1A4
:1041F00006280CD388420AD8F88114E03088022CB3
:1042000005D1062803D3884201D838820BE018254F
:1042100009E0012CFBD13078787104E0192801D233
:10422000022C02D002252846F8BD318800F05CFC43
:104230000546F8E7FFFCFFFF08480020936B0020CD
:1042400010B504460BF0A2F8002805D00078132220
:10425000214600F09BFC10BD122010BDF8B50E46A3
:10426000070048D038880BF091F8050041D0234A68
:10427000A96BD078022806D0012804D0287B082812
:1042800003D1002E01D0122436E0002901D01124E0
:1042900032E047212C200FF0DFFB0446A86320000A
:1042A00025D02C2200210FF095FC388860801C223C
:1042B000391D201D0FF0B4FB022020700F483A88F2
:1042C0000178287B082810D00020231D05F04FFC22
:1042D0000446002E03D0314628460EF0A3F9002CE8
:1042E0000AD0284607F07CFA06E00120EDE7132407
:1042F00002E0142400E002242046F8BD72480020A9
:10430000FFB51F4881B0C0781E4617460D460228EB
:1043100018D0012816D0002F30D001980BF036F8B5
:10432000040029D0E06A002801D00FF0D9FB1C213D
:1043300038460FF081FBE062011E1BD0207B08286D
:1043400003D00DE0122005B0F0BD002E08D0887E0D
:1043500000900B4612330A8A01980EF0ABFC00E085
:1043600000202179002D01D0062200E00422114313
:104370002171E8E71320E6E71420E4E70220E2E7F2
:104380007248002010B50548C078000701D50448E0
:1043900000E0002008F0A0F810BD000072480020E6
:1043A0009048002070B51A4C05460121207807F08E
:1043B0003DFA1848C1780A20014223D025701648DA
:1043C00008F084F8606800281AD1207800281DD0F1
:1043D000000107210FF040FB6060002810D0217819
:1043E0000A0100210FF0F6FB0020FF21626803E0C4
:1043F0000301401CD154C0B223789842F8D305E0A1
:10440000132070BD0020207008F060F8002070BDFF
:104410008448002072480020B46B00200949002025
:104420000870486088600948074901600849416090
:1044300008498160034808490C3001600749416020
:1044400070470000844800202DB70000B46B0020A6
:1044500051C00000ADBF00000DB6000045B6000021
:10446000F3B5334F0025BE7883B0044603282DD81A
:104470003878032802D0102005B0F0BD012C04D0FC
:10448000022C02D0032C29D02DE0049800280CD057
:104490000622002168460FF09DFB0622694604981B
:1044A0000FF0B0FA002811D104E0062168460DF0A3
:1044B000ABFE18E00622FF2168460FF08BFB0622B8
:1044C000694604980FF09EFA002801D00220D3E735
:1044D0000622684604990FF0A3FA04E06946F868DA
:1044E00005F09DF905461348BC70007804210FF0D3
:1044F000EFFD00207871002D01D0BE7015E0002C7A
:1045000013D0684607F0D4FC0500F6D1032C0CD17B
:10451000112000F091F80006000E787105D00548D2
:10452000054A007804210FF063FD2846A4E7000047
:10453000546A00207248002000770100F8B5022478
:10454000079F1D461646042919D004DC012907D00F
:10455000022945D10BE008291BD00C2940D129E0C4
:1045600000F03EF904003BD100F092F938E000F091
:1045700037F9040034D13046FFF714FF30E000F083
:104580002FF904002CD13A462846069900F05EFA2D
:1045900020E000F025F9040022D13A462846069989
:1045A00000F054FA3046FFF7FDFEFFF7EBFE05F092
:1045B000BBF915E000F014F9040011D13A46284681
:1045C000069900F043FA3046FFF7ECFEFFF7DAFEFB
:1045D00005F0AAF900F05CF900F042F905F07EFA66
:1045E0002046F8BD70B5104C2168002919D0097813
:1045F000814214D10D4D022128780FF069FD0C483D
:1046000000264680287804210FF062FD0948467193
:10461000216803204870002001F03FFB70BD03209B
:1046200070BD122070BD000054460020724800206A
:104630006C460020546A0020192801D302487047B4
:1046400002494000085A7047FFFF0000746A0020CA
:1046500010B5044600F088F800F05CF9FFF7DEFEC4
:10466000FFF74EFB0649FF23CB7000228A700A71C8
:104670000448052143700470204601F097FF10BDE7
:10468000546A002072480020F3B5304E0024306890
:1046900083B0002802D0112005B0F0BD2C4D0521BB
:1046A000E878084201D11220F6E72A494968002932
:1046B00005D00978002902D0C00702D008E01020F8
:1046C000EAE700F04DF807460AF076FF874207D385
:1046D00004980078022803D0032801D0122432E085
:1046E00047210C200FF0B8F9306000282AD0039938
:1046F0000170002141700A22801C04990FF090F98A
:10470000154EB078032806D008F080F904001AD0BE
:1047100007F05AF817E007F0DFF8694605F07FF870
:10472000684607F0C5FB012030711120FFF784FFB8
:104730000006000E707106D02878084A04210FF098
:1047400057FC00E013242046A6E700005446002052
:10475000724800206C460020546A00200077010057
:1047600010B50AF013FF10BD1A4800210170417006
:1047700041608160C1600161416181611648B4227C
:1047800001804280012292038280A022C2800281A5
:104790001022428182815023C3810382428282821D
:1047A000C2827D2302831B0143838183C1830184F1
:1047B0000F234384094B83840723C384028501228A
:1047C00042857E22D2438285C1850186491E41866B
:1047D0007047000040460020746A002080BB000043
:1047E00070B50E4605462022002109480FF0F2F967
:1047F000074C0848E570C67001F07EFA002803D027
:1048000000202070122070BD0121217070BD0000B9
:10481000546A0020724800207FB504460D460846C1
:104820000AF0B4FD002817D00C48844212D210229E
:10483000002168460FF0CEF969460C70200A4870D6
:10484000200C8870200EC8702946684605F0A0F834
:1048500004B070BD0220FBE71220F9E740420F00D0
:1048600010B50848C078400707D5074807F040FE54
:1048700000200649C043C88010BD002007F038FE64
:1048800010BD0000724800207C460020546A0020C1
:10489000F8B51D4C00256068002802D00FF020F903
:1048A0006560E068002802D00FF01AF9E560174E45
:1048B0000527F078384223D0154807F013FEF0782A
:1048C00038421BD0472120200FF0C6F86060002836
:1048D00014D0202200210FF07DF9472120200FF075
:1048E000BBF8E060002805D0202200210FF072F90B
:1048F0000020F8BD60680FF0F3F865601320F8BD84
:10490000002007F0EFFDF3E76C460020724800201E
:10491000A86A00200948FF21017000214180416000
:104920008160C16007480649016007494160074945
:104930008160024906481031086070476C460020CB
:104940004DBB0000A86A0020DDBB00000DCA0000BE
:10495000BDBA0000FEB5354F354D0C4608041FD5D5
:1049600038780FF07BF9061E17D03078A22806D0D1
:104970007D78304607F0B0FC00280AD102E02C48D0
:10498000C578F6E7FF2D04D0314628460FF09EF992
:10499000E6E730460FF03AF9E2E70120C00341E0D4
:1049A000E0070126234900280AD04868002804D0DF
:1049B0004168002901D00020884720467040FEBD94
:1049C000A00709D5C868002804D04168002901D093
:1049D00001208847022025E0600725D56879002856
:1049E0001FD0401E0006000E68711AD148690028C9
:1049F00008D02E71C868002804D04168002901D071
:104A0000012088476946E86804F009FF684607F016
:104A10004FFA1120FFF710FE6871387804210FF06B
:104A200057FB04206040FEBD0020FEBD7248002000
:104A3000546A002040460020014948707047000039
:104A40007248002010B505F023F810BD70B5154C64
:104A50000E46626121610546E0601022FF2130466A
:104A60000EF0C1FF012806D01022002130460EF0C2
:104A7000BAFF012803D1102120690DF0C5FB1022D7
:104A8000FF2128460EF0AFFF012806D0102200219A
:104A900028460EF0A8FF012803D11021E0680DF090
:104AA000B3FB70BD546A00207FB50C4605460AF082
:104AB0006DFC002814D0826B007B042802D01220E9
:104AC00004B070BD002A00D0947D684621460EF0E7
:104AD0002DF9044B6A46022128460EF0A9F8EFE7AB
:104AE0001420EDE71F32010070B50C460546192869
:104AF00002D20848844201D1022070BD112D04D198
:104B00003C20604380B201F0DBF8034968000C529E
:104B1000002070BDFFFF0000746A002070B50E46D3
:104B200011491546CB78022B17D0012B15D0002D3B
:104B300017D00AF02BFC040011D0002E03D02079EE
:104B400002210843207120461022294618300EF019
:104B500067FF2869A062002070BD122070BD14207C
:104B600070BD022070BD00007248002038B50C46B0
:104B700005460AF00BFC002806D06846047069461A
:104B800028460EF043F838BD142038BDF7B5054669
:104B90001E4812261E4F0C46814208D1B8680028D4
:104BA00032D00268002A2FD028469047FEBD174811
:104BB000401C844219D1B868002806D00268002A37
:104BC00003D028469047002806D02846029906F0D0
:104BD00055F8060005D017E07D7002983870002067
:104BE000FEBD7D70029838700EE008460AF0CEFBDC
:104BF000002809D00078A84201D00320FEBD20463D
:104C0000029900F0BEFFFEBD3046FEBDFEFF000073
:104C10004046002070B51446024620481E46C07823
:104C20000523184224D01E4D00296B68E86802D085
:104C3000002B1DD001E000281AD0202C2CD2002CF3
:104C400001D0002E28D02A70002913D01F22002165
:104C5000581C0EF0BFFF686822463146401C0EF01B
:104C6000DFFE696820460C70491C01F012F870BD27
:104C7000122070BD1F220021401C0EF0ABFFE8681F
:104C800022463146401C0EF0CBFEE96820460C70EF
:104C9000491C01F01DF870BD022070BD7248002053
:104CA0006C46002010B5094A014613790020002BFC
:104CB0000BD101231371C90707D01346643318467B
:104CC00010220421403800F007FA10BD3C470020B4
:104CD000F8B5044600F06AFE00F044F8114F134E98
:104CE000FC701149304600F025F84721C0200EF035
:104CF000B3FE00221346B861940106530021241824
:104D00000C254D436519AB80491CEB600529F7DB89
:104D1000521C032AF0DBF878787005480AF086FC0C
:104D2000F8BD00003C470020F66A0020FFFF0000AD
:104D3000DDD0000070B50A4C0025A04208D100204B
:104D400082008C525218401C95700328F8DB70BD0D
:104D500008F095F90028FAD00480857070BD000035
:104D6000FFFF0000F0B51E4920200870FF204870AA
:104D70008870C8700126CE8000200881C860086154
:104D80000B4602241C3348611C70164A5A600A46BE
:104D9000087124321470144D556016725081D3601E
:104DA0001474124F15466F612E766883E9612021D5
:104DB000545413460E4D59185D6208725885D862D6
:104DC000302154540B4C0323511854630B725087F9
:104DD000094ACA600249094A643105C10860F0BD48
:104DE0003C47002032430100344301003A430100B4
:104DF0005243010040430100F66A00209DDB0000A1
:104E0000F8B50E460746069900240798002902D0F7
:104E10000B242046F8BD022B01D00D24F9E7517870
:104E200012780D0215432946814301D08024F0E712
:104E30003846F16800F042F9A842EAD02A463846DE
:104E4000F16800F0EFF90446E3E7000070B50D46A5
:104E500008041AD50E48C0780EF000FF04000FD0E9
:104E60002078B02809D1204608F0CEFA002804D0D6
:104E700020462179083000F07BFD20460EF0C6FE6A
:104E800001212846C903484070BD002070BD0000C4
:104E90003C470020FFB585B000200F9F0090087AA6
:104EA0000E9D1C460E46C0060BD5079808F0E0F88C
:104EB00003007DD00A2231460598984700900028CB
:104EC00016D13078022815D0079808F0F7F8002896
:104ED000EFD0006884460028EBD011991098224644
:104EE0000097029101902B46314664460598A047F1
:104EF00009B0F0BD706829224178007809020143A9
:104F00001202881A91427CD00BDC6948081A13D02F
:104F1000012811D0022817D00328D5D1002F53D053
:104F20009BE001287ED002286DD0032877D004288A
:104F3000CAD1002F68D090E0002F6FD1F0680178BF
:104F400029800278416884E0002F67D1F0684178B9
:104F500000780F02074304202880F06804A9007835
:104F60002070F06840786070384600F087F90600DD
:104F700022D06846028A03AB4E493046F76800F0FB
:104F8000DBF900280AD1337802214B487268FDF71B
:104F90009BFB002802D1474869468881387802285F
:104FA0000CD10222201D79680EF03AFD288800E01D
:104FB0007CE0801C288001E0684687816846808903
:104FC000A070000AE0706FE001202880F0680021E6
:104FD000007820707089401C80B200F04FF90028E2
:104FE00013D0298802788918891C2980817A6170F8
:104FF0004189090AA17002784168E01C0EF010FD99
:1050000052E00CE00EE026E03BE028880422001D80
:1050100028800021601C0EF0DDFD45E01DE0002F22
:1050200027D01AE0F0680FF066F880B2B84201D2DB
:1050300007205DE7874201D1002006E01099C919D9
:10504000814201D3C01B00E01098288082B2F06832
:10505000C1192046D2E7002F01D00B2048E7F168A4
:10506000059800F02BF8022129802070000A60705A
:105070001AE002202880F06800782070F0684078FC
:10508000F5E70721F0682980017821704178617087
:105090008178A1704188090AE170017921718179D3
:1050A0006171C088000AA071009821E70E201FE7F7
:1050B00000280000FFFF00003643010010B507F094
:1050C000DEFF002800D0807810BD00000149887004
:1050D000704700003C4700207CB51E4605001CD0F0
:1050E000684601808270019500F0AAFA04001FD181
:1050F000002E1DD0688900280FD047210C200EF00B
:10510000ABFC002813D00021016069898180094A25
:1051100086601169002903D107E002207CBD114699
:105120000A68002AFBD1086002E0106100E0132445
:1051300020467CBD3C470020F8B50C4C0746A078C3
:1051400015460E46FF280FD00A200EF04BFD010039
:105150000AD0B12008704F80002048700871CE80BE
:105160000D81A0780EF0B2FDF8BD00003C47002094
:1051700070B50C4605460649FFF7A0FF800704D529
:105180002146284600F0B6FA70BD012070BD00002F
:10519000F66A00200EB56B461A81FE2300220193A9
:1051A0000092022302AA00F001F80EBDFFB583B001
:1051B000174602A90D9E049800F060F804002AD05A
:1051C0006846008907F07AFF002822D04568002D44
:1051D0001FD00C98019600903A462146069B0398F2
:1051E000A847050018D1FE2E16D02078022813D12A
:1051F00060684178027808020949104388420BD15F
:105200007878397802020A4304990398FFF794FFEB
:1052100002E00E2500E00125284607B0F0BD0000A1
:105220000229000070B514460E46054607F027FF18
:10523000002806D13146054807F021FF002803D099
:1052400005808470002070BD112070BDFFFF00003C
:1052500010B50178B0290BD14178002908D1017926
:10526000122906D01B2903D14088012101F0A0F8A2
:1052700010BD417C0129F7D010BD0000F0B5104AE7
:10528000536919E09C686589A84214D39E887219F5
:10529000824210D900220CE017013F197F89874212
:1052A00005D1002900D00D8010010019F0BD521C5D
:1052B00092B2B242F0D31B68002BE3D10020F0BDC4
:1052C0003C470020FFB51B4883B0002345692DE013
:1052D000AE68002470890190A888009016E0210132
:1052E00088194289039FBA420ED3049FBA420BD851
:1052F000069A002A0FD01346715C4068059AFDF7A4
:10530000E3F9002807D10023641CA4B2009884426A
:10531000E5D3002B09D00C98002802D00C990198F5
:1053200008802001801907B0F0BD2D68002DCFD175
:105330000020F8E73C470020FEB5174600256A46E6
:105340009580044640891D4A1E46904208D001AA15
:105350000092401C237880B26268FFF7B3FF0546D5
:105360002378022116486268FDF7AEF9002807D1BC
:105370002378022113486268FDF7A6F9002801D0BE
:1053800060890EE0237802210F486268FDF79CF9DE
:1053900000280DD0002D03D068468088B84203D085
:1053A000384608F01FFD04E06889401E80B200E026
:1053B0006089002E00D030802846FEBDFFFF00002F
:1053C00034430100364301003A430100FFB583B086
:1053D0000E461D46174601A9039807F06DFC040010
:1053E00022D1002F0FD0694608803088FFF746FF92
:1053F0006946088800F0BAF901460122039809F0CD
:1054000099FF002811D131460398FDF703FA0400F3
:105410000AD1FF2D08D0019B1E22194604489B1C6F
:1054200008F0EBFC0198C570204607B0F0BD000005
:105430004DDC000010B50446FDF718FA0749FF20BF
:10544000087048700020486088608C7004212046F5
:1054500001F0ACF800F004F810BD00003047002067
:1054600070B500200D4D0E4B0446FF22062141432E
:105470005D52C918CA708A70401C0C710328F5DB94
:105480000120C0431880074807F0A8FD0648FDF733
:1054900073FB06480AF0CAF8002070BDFFFF000049
:1054A000E46A002095DC000077DC0000CDDB000022
:1054B0007CB516460C460546FCF71EFF11490978D7
:1054C000884201D316207CBD01A9284607F0F4FBD1
:1054D0001728F8D0002E10D00020694608802088B8
:1054E000FFF7CCFE6946088800F040F9014601222A
:1054F000284609F01FFF0028E5D121462846FDF780
:105500009FF97CBD99480020F8B51C4615460E460B
:10551000074609F03BFF00280DD0017B074808290A
:105520002B4632463946009403D0007807F0DAFB68
:10553000F8BD4078FAE70120F8BD000030470020B0
:10554000F0B587B00F46080470D5394EB0780EF02C
:1055500085FB040064D02078A0285ED10120694634
:1055600008732046FDF7D4F9050041D168468078DC
:1055700000280BD0142809D0152807D01A2805D0E8
:105580001C2803D001461F3920290BD8B1680029F7
:105590002ED06946497800292AD169460874062028
:1055A00008751FE0C0070AD07368002B05D060881B
:1055B00003AA6946984705461AE0062518E0B3682D
:1055C000002B06D0608803AA69469847050001D1E0
:1055D0000EE0062568464078002809D1694688789B
:1055E00008740D7500204882608804A9FDF7A8F8AA
:1055F0006846007B002804D0A068002801D00EF087
:105600006FFA002D05D168468078122805D01B2836
:1056100003D16088012100F0CBFE20460EF0F6FA9F
:105620000120C003784007B0F0BDFFE70020FAE793
:1056300030470020014908707047000030470020C3
:1056400070B504464568008800284AD02B780221AE
:1056500025486A68FDF738F8002807D12B78022121
:1056600022486A68FDF730F800283AD0A078C01FB9
:10567000092834D81E4EF08800282ED0218808181A
:1056800001210904884228D847210C200EF0E4F9B2
:10569000050020D0002207E011016368F0880A317C
:1056A0005852401CF080521C20889042F4DC0020AC
:1056B000286008222146281D0EF0B2F970690028E2
:1056C00001D105E0084601680029FBD1056000E032
:1056D0007561002070BD132070BD012070BD1820C1
:1056E00070BD022070BD000034430100364301004C
:1056F0003C470020FEB50E46074600250223194A06
:10570000194901200095FFF7DDFD040027D0232073
:105710000090002304221D21384600F0E3F8029097
:1057200000281AD06089694688800420C8800299C0
:10573000012008700298334645700299FF20887056
:1057400002990022C87001A93846FFF73FFE040005
:1057500006D002980EF0C4F902E0152400E00124FE
:105760002046FEBD52430100FFFF000000B507F0D8
:105770005FFA002801D0807800BD102000BD00B580
:1057800007F056FA002800D0008800BD7CB50D4611
:10579000044609F0FBFD29462046FDF7F3F90028F1
:1057A00012D168468580204609F0F0FD00280BD014
:1057B000027B01A90748082A009106D07F23002216
:1057C0002146007807F08EFA7CBD7F230022214617
:1057D0004078F7E73047002010B504460B468806AE
:1057E0000DD51046FFF7C2FF01460122204609F001
:1057F000A1FD052801D00F2800D1082010BD882068
:1058000003420CD01046FFF7B1FF0146180701D53F
:10581000012200E00022204609F08CFD10BD88071F
:1058200001D5002010BD032010BD10B50346C806E9
:105830000DD51046FFF79AFF01460122184609F0E0
:1058400079FD052801D00F2800D1082010BD480798
:1058500005D51046FFF78AFF0146012206E04806FB
:1058600008D51046FFF782FF01460022184609F0CE
:1058700061FD10BDC80701D0002010BD022010BD81
:1058800070B51D4603460C4688060DD51046FFF739
:105890006DFF01460122184609F04CFD052801D094
:1058A0000F2800D1082070BD8820044214D0104673
:1058B000FFF75CFF0146200701D5012200E000222E
:1058C000184609F037FD002808D0697A0029EAD087
:1058D000297A002902D170BD880701D5002070BD4A
:1058E000032070BDF8B5069F1E461546162928D020
:1058F0000CDC09291FD004DC05291CD0062911D194
:105900001BE0112917D012290CD118E01D2916D03F
:1059100004DC172915D01B2904D110E052290ED020
:10592000D2290CD00124114A95420CD1FCF762FF18
:10593000001B85B20BE00224F5E70724F3E70324FC
:10594000F1E70524EFE7D22901D10C35ADB260199A
:1059500080B2394600F086FE002805D0002E00D027
:10596000358061420EF00AF8F8BD0000FFFF00002C
:1059700010B507F06DF9002801D00EF0B1F810BD98
:1059800010B5094A014653790020002B0BD10123A1
:105990005371C90707D01346A433184610220921B2
:1059A0009038FFF799FB10BD80460020F0B500212C
:1059B0003D4C0222A1603D4D227008462954401CF6
:1059C00080B21628FAD36270374BE180A270502063
:1059D0000C331880A0205880184681807D20C0009C
:1059E000D880E27001233048237161711430027055
:1059F0002F4C4460037241812E4CC46006460274F1
:105A00002D4F77613446337671831034143EE6604F
:105A1000202402550646294F341977622372718576
:105A2000F562302402550546234E6E632C1923720D
:105A30006987133DE560402402550546204E6E649B
:105A40002C19237261810E3DE560502402550546F4
:105A5000194E2C196E6523726181123DE560602438
:105A600002550546174E6E662C1923726181083D5A
:105A7000E5607024025505460F4E2C196E6723729F
:105A80006181113DE560802402550F4A80304260FB
:105A9000037241816A1CC2600C48A03210600C483D
:105AA000506010468160F0BD80460020B46A00203E
:105AB00034430100C84201003A4301004843010059
:105AC0004A430100504301005A430100C1DE000077
:105AD00009E0000070B51646214A0D461146002423
:105AE0001431030004F05AFB0A0613383818382121
:105AF00028383138152D2AD81622002119480EF0E1
:105B000069F82A46314617480DF08AFF25E0022D34
:105B10001DD13088D08020E0082D18D110480822EF
:105B200031460C30FCF79FF917E0012D0FD1CA69FF
:105B30000B4930783C3105E0012D08D1CA6B08498A
:105B400030785C3108F028FA07E0012D01D01824E4
:105B500003E03078107100E00224204670BD0000A0
:105B600080460020B46A0020704710B500F0FAF8B3
:105B700010BD10B500F016F910BD10B500F02AF9EF
:105B800010BD10B5FCF7AEFB10BD10B500F036F936
:105B900010BD10B500F04AF910BD10B500F060F965
:105BA00010BD10B5FCF7ACFB002010BD10B5FCF724
:105BB000C1FB10BD10B5FCF7CDFB10BD10B5FCF757
:105BC000D9FB10BD10B5FCF7E5FB10BDFEB508AF65
:105BD00070CF6F4670C7FCF7EDFBFEBDF0B585B02A
:105BE00084460AA8F1C804976F4671C7604600F062
:105BF0004DF905B0F0BD38B5049C009400F07EF975
:105C000038BD10B5FCF7E6FB10BD38B5049C009418
:105C100000F092F938BDFFB587B094468E4610A8C3
:105C2000F7C806976F4677C762467146079800F037
:105C3000A1F90BB0F0BD10B500F0EEF910BD10B534
:105C4000FCF7D6FB10BD10B5FCF7E4FB10BD10B59A
:105C5000FCF7F2FB10BD10B5FCF7FEFB10BD10B554
:105C600000F0F8F910BD10B5FCF708FC10BDFEB54A
:105C700008AF70CF6F4670C7FCF712FCFEBD38B599
:105C8000049C009400F004FA38BD10B5FCF722FC27
:105C900010BD10B5FCF72EFC10BD10B5FCF73AFC9A
:105CA00010BDF0B585B00AACF0CC03976F4670C755
:105CB000FCF740FC05B0F0BD10B5FCF751FC10BD81
:105CC00010B5FCF75DFC10BD10B5FCF769FC10BD0C
:105CD00010B5FCF775FC10BD70B55478157822022C
:105CE0002A43FCF77DFC70BD10B5FCF783FC10BDAA
:105CF00010B500F0EBF910BD10B5FCF77FFC10BD3E
:105D000038B5049C009400F0F9F938BD38B5049C0E
:105D1000009400F09FFA38BD10B500F00BFA10BDEA
:105D200010B5FCF77DFC10BD10B505280ED90C4C44
:105D3000A0420BD2A14209D2814207D3FF20F53005
:105D4000824203D2092B01D9A34201D3002010BD06
:105D5000521C4A43D8008242F8DA012010BD0000EC
:105D6000810C0000F8B50746084616460D460C3073
:105D70000DF038FF040011D0912020700E206070CB
:105D8000A5702046A7800C302A463146A0600DF051
:105D900047FE0348214600780DF098FFF8BD00004B
:105DA0007248002070B505460C4606200DF01AFF1B
:105DB00001000BD0912008700F2048708D700120D9
:105DC000C87003488C8000780DF080FF70BD000023
:105DD0007248002010B5044603200DF003FF0100B7
:105DE00008D0912008701A20487003488C70007801
:105DF0000DF06CFF10BD00007248002070B5064623
:105E000014460D4608200DF0EDFE01000AD0912049
:105E10000870052048708E708D8003488C71007862
:105E20000DF054FF70BD00007248002070B50646AA
:105E300014460D4608200DF0D5FE01000CD092202E
:105E400008703E204870082088708D808E7103484D
:105E5000CC7180780DF03AFF70BD000072480020D0
:105E600070B505460C4606200DF0BCFE010009D0B9
:105E700091200870302048708D7003488C80007825
:105E80000DF024FF70BD000072480020FFB50746EA
:105E900081B01D46164616200DF0A4FE040029D040
:105EA000912020703E2060700120A070002F08D04B
:105EB0003120E07020460622002108300DF08AFED5
:105EC00007E00020E0702046062208300A990DF015
:105ED000A7FD0298A080A671E5710B98E0810C984F
:105EE00020820D9860820E98207503482146007824
:105EF0000DF0ECFE05B0F0BD72480020F8B5074685
:105F00001C4615460E460C200DF06CFE01000FD00D
:105F1000912008703E20487003208870CF708E80DA
:105F2000CD800C8106984881024800780DF0CEFEA5
:105F3000F8BD000072480020F8B507461C4615461B
:105F40000E460E200DF04EFE01000FD0912008707D
:105F50003E204870072088708F80CE800D814C8154
:105F600006988881024800780DF0B0FEF8BD000068
:105F700072480020FFB581B01D4616460F4622200C
:105F80000DF030FE040042D0912020703E20607061
:105F90000A20A0700198002814D03120E07020461B
:105FA0000622002108300DF015FE204606220021B1
:105FB0000E300DF00FFE20460622002114300DF0A9
:105FC00009FE13E00020E0702046062208300A99FE
:105FD0000DF026FD204606220E300B990DF020FD17
:105FE0002046062214300C990DF01AFDA780A671E8
:105FF000E5710D9860830E98A0830F98E0832021AF
:10600000109808550348214600780DF05FFE05B052
:10601000F0BD000072480020F8B5064615460F4650
:1060200010200DF0DFFD040011D0922020703E20E2
:1060300060700520A070A68008223946A01D0DF0D2
:10604000EFFC0348E581807821460DF03FFEF8BD66
:1060500072480020F8B5064617460D460E200DF092
:10606000C1FD040011D0922020703E2060700420F9
:10607000A070E670A58008223946A01D0DF0D0FC66
:106080000248214600780DF021FEF8BD724800203C
:10609000F8B507461C4615460E460E200DF0A2FD2B
:1060A00001000FD0912008703E20487006208870B3
:1060B0008F80CE800D814C810698888102480078BF
:1060C0000DF004FEF8BD00007248002070B51446C3
:1060D0000D4608200DF086FD01000BD090200870C1
:1060E00013204870012088708D800348CC80007890
:1060F0000DF0ECFD70BD00009F480020F8B507468C
:106100001C4615460E460C200DF06CFD01000DD00E
:10611000912008700C2048708F708E808D710C81DA
:1061200006984881024800780DF0D0FDF8BD0000C7
:1061300072480020FFB581B0444E02990025F068F6
:10614000174602292ED0B18800297CD07288CB193D
:10615000121D934271D840183A4604990DF060FC24
:10616000B088C01980B2B0807188091D88426AD198
:106170000C200DF037FD01005ED090200870FF204C
:1061800048700198488002200871B088C880F06883
:1061900088602F4800780DF099FDB580357000209B
:1061A00005B0F0BD04994A780B78110219433A1FE3
:1061B0007180914222D10C200DF014FD040039D0E1
:1061C00090202070FF2060700198608002982071FC
:1061D000E780482138460DF03FFCA060002809D038
:1061E0003A4604990DF01CFC1948214600780DF040
:1061F0006DFDD4E720460DF073FC1BE0914219DDE4
:106200003178002903D0002801D00DF069FC708896
:106210004821001D80B20DF01FFCF060002812D054
:106220003A4604990DF0FCFBB78001203070B6E7C8
:1062300009E002E0B58006E0F068002801D00DF02A
:106240004FFCB58035700120AAE700006C480020A3
:106250009F480020FFB583B01C4615460E460C9F94
:10626000039809F093F8002809D068460680458015
:106270008480C780FF226946039800F065F807B064
:10628000F0BD0000F8B52649264B4C68002081007F
:10629000625C5A540A19C91855784D7095788D70FA
:1062A000D278401CCA700428F1D336E00022810065
:1062B0006C460E1FB5185D5DA554521C042AF9D317
:1062C000820714D1224656789578D778164A2478D2
:1062D000965DB446565D6D466E70D65DAE70125DCD
:1062E000EA70124C8208A25C664656402E70CC18AA
:1062F0002246203A6E46157C367875405D546E46CF
:10630000517C757869406170917CB5786940A17065
:10631000D17CF2785140E170401C2C28C6D3F8BDE6
:10632000D8480020C06C0020AC430100AC450100FF
:1063300008B51346034A00920A46012108F0C8FD39
:1063400008BD0000BDE100003EB500230192042419
:1063500002930A460094024B122108F0C5FE3EBD8E
:1063600063E2000008B51346034A00920A4613216F
:1063700008F0AEFD08BD00008FE200001FB56946C1
:10638000C8810022FF2103206C4607C4034B03AAE7
:106390000621034808F0A8FE04B010BD33E2000057
:1063A000FFFF000001480089704700009848002066
:1063B00013B504480079012803D101AA6946FFF703
:1063C000F0FB1CBD9848002070B500252A4C3022F7
:1063D00025706570A570E57025716571A5712581C1
:1063E000E560E071294625480DF0F4FB09F072F8EC
:1063F00026460A36307800280ED000014C210DF0D8
:106400002BFB2061002807D07178E1703178A170F2
:106410000A0100210DF0DEFB1948E17800784018F0
:10642000C0B2207000014C210DF016FBE060002886
:1064300011D021780A0100210DF0CCFB0020FF21B2
:1064400005E0E3680201D218401C5172C0B2227804
:106450009042F6D301E02570E570084A002017212C
:10646000103A4300401CC0B2D1520828F9D3054865
:1064700009F0DCF870BD000098480020D06B0020C7
:10648000AC47002001E600000A2A01D00120704735
:106490004A780B7812021A430280CA788B7812026B
:1064A0001A4342804A790B7912021A438280CA79D0
:1064B0008B7912021A43C2804A7A0B7A110219436D
:1064C000018100207047042A01D0012070474A78DA
:1064D0000B7812021A430280CA788B781102194392
:1064E000418000207047082A01D0012070474A7877
:1064F0000B7812021A430280CA788B7812021A4370
:1065000042804A790B7912021A438280CA798B79C8
:1065100011021943C180002070470000F8B5214ED8
:106520000D4608042ED5F0790DF098FB04000BD031
:106530002078902805D16078132808D0204608F0EC
:10654000C7FB20460DF062FB0120C00328E016497E
:106550000020097CA7780BE0420012199279737829
:10656000D218D2B27270914200D27170401CC0B287
:106570008742F1D870780028E3D00121F0790DF03E
:10658000F7FBDEE7E8070CD008F08EFD002806D008
:106590007078002803D00121F0790DF0E9FB01208B
:1065A0006840F8BD98480020CC690020042907D035
:1065B000052905D0062903D0072901D002207047FC
:1065C0000C22044B4A43D218403A118290740020A6
:1065D00070470000D06B002070B50C460988054656
:1065E000042905D0052903D0062901D0072929D17E
:1065F0006068002826D00121284609F04BF80028C1
:106600001ED0284608F096FF0F498D420BD0002877
:1066100009D12189002906D9208806280ED10B48E6
:10662000008881420AD20A480078002804D0214616
:10663000284607F08FFE70BD162070BD1B2070BD70
:10664000142070BD022070BDFEFF0000A048002095
:1066500099480020024A001F1081517070470000C5
:106660009848002010B5001D80B24C210DF0F4F9BF
:10667000002803D00321C9430DF080F910BD0000AC
:106680000C480B4A0068918841610A21C16141624E
:106690003223C3624163C36393884364C164118935
:1066A000816541681F22114341600349C160704701
:1066B000006A0020384600201F03000070B5154610
:1066C0001C46214A0B46916B90B0002902D0097BF1
:1066D000002934D1116C002902D0497C00292ED127
:1066E000916C002902D0C979002928D1164940317E
:1066F0008E8E16498988890A8E4202D3072010B0EF
:1067000070BD11496031097F490618D56946C870C6
:106710000622194601A80DF083F90AA8102229467D
:1067200002300DF07DF906A81022214602300DF04E
:1067300077F9684601F006FB801B012801D00C2088
:10674000DDE70020DBE70000006C0020CC690020C2
:106750001CB51B4B9A6B002A05D0147B002C02D071
:10676000D27A002A11D11A6C002A05D0547C002C50
:1067700002D0927CD20708D19A6C002A07D0D37934
:10678000002B04D0D27B002A01D012201CBD0C4A61
:106790000C4B40329B88928D9B0A9A420BD26A46E0
:1067A000507000A8062202300DF03AF9684602F057
:1067B0009FF8012801D007201CBD00201CBD00004F
:1067C000006C0020CC690020F0B51F4C89B00D464C
:1067D00006462146002003F0F2FE0028F9D0A04230
:1067E000F7D0002104460120800527460743009189
:1067F00001910291039104910591069107916A46D6
:10680000D773390A9173390C5173304604AA69461B
:106810000AF00EF96A46907F517F00020904401881
:10682000D17F40182870010A6970000CA8700121FE
:10683000200A89030843EF702871200C4021084387
:10684000687109B0F0BD0000FFFF3F00F8B5444992
:106850000D468035C86A2877020A6A77000CA87747
:10686000886AE877010A2C4620342170000C607099
:106870003C49002003F094FE00260746711E304676
:1068800003F09DFE30433A460AE0002003F088FE04
:1068900000270646791E384603F091FE38433246FB
:1068A000930430499B0C0343EFD0D643C3430E40BF
:1068B0003343EAD0FF231B02034020721B0A63729A
:1068C000FF231B0403401B0CA372000EE072227313
:1068D000100AC0221043607301200090214900205B
:1068E00003F05EFE00270646791E384603F067FE79
:1068F0000146394330460A460243EFD0194BCA439A
:1069000043401A43EAD0FF230A461B021A40130AE7
:106910000A46FF273F043A40CEB2A673C7B2E373DC
:10692000120C2274090E61748004A774800EBC4698
:10693000E0742F7FBE4211D16E7FB3420ED1AB7F88
:106940009A420BD1EA7F914208D12278944505D131
:106950006178884202D100980028BFD1F8BD0000BC
:10696000006C0020FF3F000010B500F01DF88222EF
:106970008021002001F0D0F910BD000010B50648BC
:10698000C078002804D1054803F066FA00F054FCF2
:1069900004490348C86310BD006A002081750000E7
:1069A00025F70000006C002010B50B48846B03F045
:1069B000D1FE00202073A0722071084C0121E078E4
:1069C0000DF086FBE07802210DF082FBE0780421D7
:1069D0000DF07EFB10BD0000006C0020006A00205E
:1069E00010B501F047FA002010BD000010B51149A4
:1069F000886B002805D0027B002A02D0C07A0028CC
:106A000011D1086C002805D0427C002A02D0807C7D
:106A1000C00708D1886C002807D0C179002904D0AC
:106A2000C07B002801D0122010BD01F099FF00208A
:106A300010BD0000006C0020FFB581B00D4600F0D5
:106A40006DFA040022D01920C00185421ED8062DFF
:106A50001CD30399814219D8A94217D3FF22049964
:106A6000F432914212D80A9981420FD80498C90091
:106A7000401C6843814209DDA07BC00706D1264641
:106A800080367168480701D4880702D5122005B006
:106A9000F0BD20464030C585039A02860B9A428697
:106AA0000C9A8286049A82820A9AC2820746E27906
:106AB0000220002AA27E02D0002A30D039E0002A2B
:106AC00037D1E022125D920702D50143716024E0C4
:106AD000039885420BD028184108284603F060FD32
:106AE000788221465231039809F08EFF00E07D82C2
:106AF00009F060FD401C042801D9042002E009F0DF
:106B000059FD401CF873204609F028FF208F04210E
:106B10000A303883706808437060122008E0E02271
:106B2000125D920701D41A20B1E70143132071606E
:106B3000A0760020ABE7017A4A07D30FEC22125867
:106B400012781207D20F934204D1042251400172ED
:106B50000020704701207047017A0A07D30FEC220A
:106B6000125812785207D20F934204D00822514093
:106B700001720020704701207047000038B50546BB
:106B80000021084603F07EF90C4C2068002811D043
:106B90000B48006E01280DD1684600F0AFFA094895
:106BA0000099807F4008081A7D21C9004843216868
:106BB00040098847B020287338BD0000D448002021
:106BC000006C0020CC690020014680318A6C521C88
:106BD0008A64CA6C01D1521CCA64120603D5012210
:106BE0008A640022CA642030C1784A0602D5202275
:106BF0001143C1707047000070B50546FF200002C8
:106C00002C468034216F05E04A8902434A81216F76
:106C1000C96821670029F7D1A16F002906D04A89E8
:106C200002434A81A16FC968A167F6E7A06E0028F8
:106C300001D00CF055FF2C4620346078FF2801D09D
:106C40000DF022FA2078FF2801D00DF01DFAA0786F
:106C5000FF2801D00DF018FAA88800F0D9F80848EC
:106C6000806800280BD00748006E002807D1064C2A
:106C7000E069002803D00CF033FF0020E06170BD14
:106C8000CC690020006C0020006A002070B504462A
:106C90001C480E46C16D0025A14200D1C565F820F3
:106CA0000059002804D0A0880022802101F034F887
:106CB000E08F002804D0A0881322812101F02CF855
:106CC000A0880522812101F027F8A57165734E2067
:106CD0000655E079002807D109F072FC012803D895
:106CE0000121002003F0CEF8E079012807D109F056
:106CF00075FC012803D80221002003F0C3F800200E
:106D000070BD0000006C0020014680310A6C521CEE
:106D10000A644A6C01D1521C4A64120603D501224E
:106D20000A6400224A642322125C520609D5028FAB
:106D300040304388D2180280012248689202904372
:106D40004860704770B5044618206072E82000590A
:106D500000282BD00F21817021464031CA8DC2708E
:106D6000120A02710A8E4271120AC31C82711D46F8
:106D70008A8A2A71120A6A71CA8A4272120A827255
:106D80008A7FC272098C0173090A417321460C2261
:106D900062310E300CF044FE20462030C1780422CF
:106DA0001143C17092206073002070BD012070BD3E
:106DB00070B5054618206872E8204059002825D093
:106DC00010212C4681704034E18DC170090A017197
:106DD000218E4171090AC31C81711A46A18A117161
:106DE000090A5171E18A4172090A8172A17FC17257
:106DF000218C0173090A417329460C2262310E303D
:106E00000CF00EFE97206873002070BD012070BD4D
:106E100070B5164C0346206D002102460D461CE05D
:106E2000FF265936365A9E4215D1002904D0626D8C
:106E3000824204D1616504E01168216501E00268C5
:106E40000A600CF04DFE606D0560206E002809D0D0
:106E5000401E206604E0014600680028E0D1206E54
:106E6000002802D100F004F8256570BD006C0020F8
:106E700070B5064D6C6B03E020460CF031FEE46803
:106E8000002CF9D10020686370BD0000006C002068
:106E9000F8B51F4E706B002838D1348C1D48213452
:106EA00004401D4D2146287C1031801C484380B28F
:106EB0001B210CF0D1FD002828D07063297C154ED1
:106EC00009010A1800218C3E0F4620321AE00229DF
:106ED00002D2104B8E3B05E0042901D2468102E02C
:106EE0000C4B1F334381026007812B7C5B1C8B4260
:106EF00003D903461033C36000E0C760491C121970
:106F000089B210302B7C9B1C8B42E0D8F8BD00006E
:106F1000006C0020E0FF0000CC690020014606481C
:106F2000006D05E0FF225932125A8A4202D00068F1
:106F30000028F7D170470000006C002030B50C4AE3
:106F400004460948137C0021406B084D9B1C07E058
:106F50004289A24207D0AA4205D0491CC9B21030CA
:106F60008B42F5D8002030BD006C0020FFFF0000F0
:106F7000CC69002010B51422002102480CF02AFE32
:106F800010BD0000506C002070B5FF255D3510214C
:106F900028460CF061FD04462A4600210CF01AFE3A
:106FA000002C0FD01F4D01232A6D002A0CD0686DD4
:106FB000FF304130018B491C89B2080400D5012102
:106FC000104609E0002070BD19460AE0FF26593638
:106FD000365A8E4203D000680028F7D101E000281D
:106FE000E9D12646FF3641363183002910D0002AE8
:106FF00012D0686D04606C65286E401C2866696D4F
:1070000000200860318BA180A0712073A08870BD22
:1070100020460CF065FDF9E72C656C652B66FFF7E3
:1070200037FFECE7006C002010B50648806C0028A4
:1070300006D0C079002803D000F074F9002010BDFC
:107040000C2010BD006C002010B50C46FFF766FF49
:1070500000280FD08179102901D0022010BD4E21C7
:107060000C54C179002903D031214173002010BD97
:107070003021FAE7122010BD70B504460D20607271
:10708000E8200059002815D0054604202146A870A4
:10709000FF3108222931E81C0CF0C2FC2146FF31E7
:1070A0002846042231310B300CF0BAFC44206073C6
:1070B000002070BD012070BD0B4610B5014618467A
:1070C000FAF762FF002010BD10B509230146437294
:1070D00080318A6E002A0FD09370C2798B6E002A9D
:1070E00006D008225831D81C0CF09AFC002010BDA4
:1070F00008220146D031F6E7012010BD38B504461C
:107100001948C1780020C043002928D0002C26D07F
:107110001649096D002922D0154D942253580A8E24
:10712000934201D39A1A01E09A1A5219904200D957
:10713000104609680029F0D10E498A6B00928A6BCB
:10714000009B9A42F9D11946834201D8C11A05E041
:10715000814205D58842F9D2C11A4919216038BD4A
:1071600000202060084638BD006A0020006C002026
:107170000000C0A800100040F1B5002582B02C46E8
:107180000420029A290E121824020C43FF3229020D
:1071900001321578401E0D4340B20028F1DA029802
:1071A000C17C203040790818C7B2252F01D3253F74
:1071B000FFB202983A46C77401200021FAF743FE55
:1071C00028402140084302D002988774FEBD002069
:1071D00006460090324601200021FAF734FE28408E
:1071E0002140084303D00098401CC0B20090761C98
:1071F00076B2252EEEDB38460099FAF7BDFD002762
:107200003E460091324601200021FAF71CFE28403C
:107210002140084307D00098874202D10298867423
:10722000FEBD7F1C7FB2761C76B2252EEADBFEBD4A
:107230000021C1747047000070B505463048002435
:1072400004603048C022046021462F480CF0C2FC84
:107250002E480622C5702E48002105460CF0C3FBBF
:10726000012804D12B49062228460CF0D9FB284AD4
:10727000294D163AD07D117E000209044018917DF7
:1072800041182148C162917ED37E09021B04C918AE
:10729000537EC91881620821C18105821F4B438238
:1072A0000175C3824175058343830146FF23603125
:1072B0000B774C778C77CC7720310C704C708C70BE
:1072C000CC7020318B76CB760B774B771F238B7767
:1072D000D17B0184CA00703242848184C2841B2124
:1072E0008183FF214931C1830D490163FBF796FC7E
:1072F000FFF740FE01F046FB00F0D4FD70BD00003A
:1073000068480020D4480020006C0020006A00205B
:10731000E269002008060400D70700006081000031
:1073200000F9150070B50E48846C03F013FA0D4D8A
:10733000FF21E87801310CF0CBFE0121E878490209
:107340000CF0C6FE0321002002F09CFD0020E0713D
:107350002071A0718122802100F0DEFC70BD000050
:10736000006C0020006A00200449098C0170002193
:1073700041700349097C817000207047006C002037
:10738000CC69002070B509214172E8210958002913
:1073900030D014228A700246FF3224321346547DC4
:1073A000127D25021543CA1C1446CD7002462D0AD3
:1073B000FF320D712232557E167E2D0235434D71FE
:1073C0002D0A8D715D7E1E7E2B02334323711B0AB5
:1073D0006371537F147F1A0222434A72120A8A721F
:1073E00001462031CA7804231A43CA70B22141737E
:1073F000002070BD012070BD30B509214172E82127
:107400000958002926D015228A700246FF322432FC
:107410001346547D127D24021443CC70CA1C240AE6
:10742000FF300C712230447E057E24022C434C71C7
:10743000240A8C715C7E1D7E23022B43CB711B0AB8
:107440005371427F037F100218434872000A88720A
:10745000002030BD012030BD10B5FFF75FFD0028D2
:1074600005D0C179012902D1417B462901D00220F2
:1074700010BD0146062220310A7147224273487826
:107480000CF002FE002010BD70B50C46FFF746FD63
:10749000002802D0C179012901D0012070BD417BB3
:1074A00046292FD1A27BE17B12028918627B237BC4
:1074B00012041B06D2188A18014680318A62A37A08
:1074C000E27A1B02D218637A257A1B042D065B1917
:1074D000D218CA62A379E2791B02D218637925799E
:1074E0001B042D065B19D2180A63A378E2781B02ED
:1074F000D218637824781B0424061B19D2184A6317
:1075000050214173002070BD70B50D46FFF706FD98
:10751000040006D02946FFF7B9FB20342071002073
:1075200070BD122070BD01214172E8210958002967
:1075300005D00B228A70742141730020704701200E
:10754000704701214172E821095800290AD012220E
:107550008A70A22141732030C17804221143C17086
:107560000020704701207047012141728030806EF9
:10757000002803D01321817000207047012070473C
:1075800070B50C460146200412D508460CF066FB87
:1075900005000AD02878802801D0812802D1284609
:1075A00000F070F828460CF031FB0120C00361E0C8
:1075B0003249E207886B8030002A05D00068002835
:1075C00000D08047012055E0A20705D5406800287B
:1075D00000D0804702204DE0600703D5FFF7C4F9D3
:1075E000042047E02548A206006C05D5006D002860
:1075F00000D0804720203DE0E20605D5C06C002881
:1076000000D08047102035E01C48A205806C06D5CC
:10761000006E002800D08047012040022AE0E205E9
:1076200006D5C06D002800D08047FF20013021E042
:10763000124AE004157913D511484278D2070DD0CB
:10764000006903234278521D1A43805CC00602D4AD
:107650000889401C0881284600F086FA204670BD43
:10766000A00409D5CB798A794979284601F0A0F898
:1076700001204003604070BD002070BD006C002000
:10768000206A0020F0B5017800248DB0802902D056
:1076900081297DD0D3E1FC4E4178354680350629DD
:1076A00077D006DC0B0002F079FD060D3EEFEEED23
:1076B000ECEF07296ED081296DD082296CD0862904
:1076C000E8D178E14088FFF729FC05007ED02E46FE
:1076D000AC758036B06F002823D0036882790179B9
:1076E000A8889B1CFEF718FB00280DD1B06FFF2265
:1076F0004189120211434181B06FC068B067A88F01
:10770000002801D0401EA887B06F002809D0A888A3
:107710000022802100F000FB002801D10120A87583
:1077200001E2AC87FFE14088FFF7F8FB0700CDD00E
:10773000F879012834D0B66C002EC7D0687D800758
:1077400072D53420805D02286FD00622002107A860
:107750000CF040FA35464035287902287FD00622C1
:10776000002109A80CF036FA0622A91D0BA80CF07E
:1077700057F9F98DB88D7A8D039204AB13C309AA1A
:1077800007A90BA86B4607C3B9886B79203704E0BB
:1077900042E1FAE01FE189E09AE038790022A8E0AE
:1077A000B46B002C92D0687D80073FD525466035AC
:1077B0002879022814D00622002107A80CF00AFA22
:1077C000687D022813D30622214600E0F0E07631DE
:1077D00009A80CF025F9216E06220BA8091D0FE05F
:1077E0002146062207A866310CF01AF9E8E70622BE
:1077F000002109A80CF0EEF92146062276310BA8EB
:107800000CF00EF938462030798D8479FB8DBA8DD5
:1078100003AE1EC609AB07AA0BA96C460EC46B7D4E
:10782000B9880079012264E02FE011E03846203069
:10783000798D8579FB8DBA8D01AE2EC621467631C4
:1078400000916034637DB9880079012260E006E030
:1078500031460622363107A80CF0E2F87AE73146C5
:107860000622463109A80CF0DBF8716D06220BA840
:10787000091D0CF0D5F8706D0221C07808436871BD
:1078800077E76FE058E046E0D9E0F88DB98D7A8D62
:1078900003903046463004940192029100904036A5
:1078A000B988203773793879002231E0B06C00282C
:1078B0007ED0C28A818AC38C02AD019316C501466F
:1078C00046310091403000224379114602201FE0EA
:1078D000B06B0028ECD0697D89070DD5059406941E
:1078E00000230394049400940194012219463C203F
:1078F0000294FEF790F916E101466E310091019471
:107900000294039460300494437B012200213C20C4
:10791000FEF764F907E14088FFF700FB0028C7D0B5
:1079200001464031CA8A00928B8A4A8A8188203077
:107930000079FEF760F9F6E04088FFF7EFFA0028DB
:10794000B6D0C1790129818807D02422135C024670
:10795000D8321846FEF783F9E5E02422135C02468C
:10796000D032F6E74088FFF7D9FA002820D0C11DB1
:10797000FC314A7D097D12020A4301468388FF31AA
:1079800010311846FEF757F9CDE04088FFF7C6FAE8
:1079900004000DD020464030C18A0091838A028EB7
:1079A000C18DA088FEF76BF9A07B0421084300E09D
:1079B00077E0A073B7E04088FFF7B0FA002870D0F6
:1079C00001464031CA8A00928B8A0A8EC98D80880E
:1079D000FEF79CF9A7E04088FFF7A0FA002860D0E6
:1079E0000146FF3144314B7B0A460C7B190221438F
:1079F00000910146FF3142314B7B0C7B1B0223433C
:107A0000547C157C22022A434C7C0D7C21022943A4
:107A10008088FEF7FAF886E041781A2968D008DCF9
:107A200005290FD0082931D00C2942D0132906D1BD
:107A300050E0302966D0572972D0FF2973D0012039
:107A40000DB0F0BD4088FFF769FA050066D0F02060
:107A5000405900280DD0E98FC068491CE9870028EB
:107A6000F9D10A04120C04D0A9880120FEF740F9CC
:107A7000EC874E20425D2420A988405DFEF785F802
:107A80002846FFF7B9F84EE0006C00204088FFF769
:107A900045FA002842D04621095C002902D0012283
:107AA00001E03BE00022818820300079FEF771F888
:107AB00039E04088FFF732FA00282FD001464031E4
:107AC0008A8900924B894A7A818820300079FEF7B2
:107AD00017F928E04088FFF721FA05001ED0EA8F49
:107AE000002A20D0A9880120FEF702F9EC871AE0CD
:107AF0004088FFF713FA002810D020300079FEF7F5
:107B00003CF810E04088FFF709FA002806D0818889
:107B100020300079FEF741F805E001E002208FE710
:107B20004088FEF721F800208AE770B5054600245A
:107B3000FF21012002F051FD2855641CE4B2082CFD
:107B4000F6D3002070BD0000064A00215318803390
:107B50001B7F0370491CC9B2401C0629F6D30020C4
:107B600070470000006C002010B5002803D00B28DF
:107B700003D8401E06E025200CE00C2804D026285F
:107B800004D8801EC0B205E0262003E0272801D0DB
:107B9000122010BD02F0A8FD002010BD022141728C
:107BA000014680310A46896E002907D00D238B706B
:107BB0002030916E0079C870002070470120704716
:107BC00003224272E8221258002A07D01123937030
:107BD000D17020300079107100207047012070476B
:107BE00010B50C46FFF79AF900280FD024210C5449
:107BF000817B4A070AD5FB22114081738030012224
:107C00004168920311434160002010BD122010BD55
:107C1000FFB581B016460F46FFF780F904463C4990
:107C2000B81F884271D2481D86426ED8BE426CD3BE
:107C3000FF220499F432914267D80A99814264D8AC
:107C40000498C900401C7043400081425DDD002C57
:107C50005BD0A07B41074BD5FB2108402546A07394
:107C60004035EF852E86E079002808D02046803008
:107C700001224168520311434160102037E0688CB3
:107C80002449884204D0B74202D12882608D09E09D
:107C9000E88B0090002807D001463046FAF76CF8D0
:107CA0000099484368820AE0B8194108384602F052
:107CB00077FC688221465231304608F0A5FE08F074
:107CC00079FC401C042801D9042002E008F072FC71
:107CD000401CE873204608F041FE208F04220A3041
:107CE0002883204680304168114341601120A076EE
:107CF00040340B9860860C98A0860498A0820A985D
:107D0000E082002005B0F0BDFFE71220FAE7000096
:107D10007B0C0000FFFF000070B5064614460D46C0
:107D200004200BF05FFF010007D00D704C70044879
:107D30004E80C0780BF0CAFF70BD042070BD0000FB
:107D4000006A0020F0B5002787B005463848009744
:107D50000197029703973E46846F0CE0E078E9783C
:107D6000884206D11022291D201D0BF04BFE012850
:107D700042D02646E46B002CF0D11A2140200BF0B3
:107D80006BFE040038D0E878E0700622291D201D23
:107D90000BF046FE20461A30294610221A31059073
:107DA00004900BF0DBFF1022694604980BF02AFECA
:107DB000002823D0A772294620462A3010222A31D3
:107DC00005460BF0CBFF1022694628460BF01AFE41
:107DD00000281FD0A774164D2046296B08F016FF07
:107DE000002E23D0F4631249E7634031888E401C93
:107DF00080B2888607B0F0BD0020FBE70120A072AA
:107E0000E07802210843E07221460C310598FEF724
:107E1000DBFCD0E70120A074E07802210843E07485
:107E2000214614312846FEF7CFFCD4E7AC67DAE7E9
:107E3000006C0020F7B50E4815466E46846F0CE0C6
:107E400068464078E178884206D10622211DB01CA0
:107E50000BF0D8FD012804D0E46B002CF0D10020F9
:107E6000FEBD204629462A3008F082FEFEBD0000F5
:107E7000006C002070B50A4DFF26AC6F07E020783B
:107E80000CF002F926702046E46B0BF029FE002C62
:107E9000F5D100200249A8674031888670BD0000F6
:107EA000006C002010B5044900208886403988679E
:107EB000FEF7CCFC10BD0000406C002070B50546FC
:107EC0000B48846F0DE06878E178C007C00F8842E6
:107ED00006D10622211DA81C0BF094FD012804D018
:107EE000E46B002CEFD1002070BD204670BD000077
:107EF000006C002070B505460848846F07E02046F6
:107F0000A91C2A3008F034FE012804D0E46B002CB0
:107F1000F5D1002070BD204670BD0000006C00202F
:107F2000F8B504468030C16EC81C0A798446CB7807
:107F3000100218432E4B821F9A4225D28B794D791D
:107F40001B0219264A1C2B43F601B3421CD883425C
:107F50001AD365466F792D793F022F43FF25F435FB
:107F6000BE46AF4210D8557A177A2D023D43B5422E
:107F70000AD87646761C4643EF00BE4204DACE7A33
:107F8000002E03D09E4201D91E20F8BD668D002729
:107F9000864208D19E4206D1A38D734503D1E38D5D
:107FA000AB4200D1012723464033D885507915795B
:107FB0000002284318866046457906792802304336
:107FC0009882507A127A00021043D882C87AD883F5
:107FD000487B0A7B00021043188420460C22623042
:107FE0000E310BF01DFD0420A0763846F8BD0000D0
:107FF0007B0C000070B5EC210B58DA1C1979144683
:108000000A02DD780146FF312A4341314A805A1C79
:108010009B7915791B022B438B80637924791B0292
:108020002343CB80537A147A1A0222430A8108F040
:108030006CF970BDEC2109584030CA7842724A7917
:108040000B7912021A434281CA798B7911021943C2
:108050008181704770B50F48046C02F07BFB0025EE
:1080600025730421284601F00DFF0B49282088774D
:108070006574A571606A0BF033FD25846562A562A5
:10808000064C1021E0780CF023F8E07820210CF069
:108090001FF870BD006C0020CC690020006A002031
:1080A00000214172017A012289088900114301727D
:1080B0008030806E002801D000207047012070477A
:1080C000FFB581B01F461546FEF728FF06000BD00E
:1080D0003046FF3042300090417C027C0802104361
:1080E000A84204D2C4B203E0022005B0F0BDECB255
:1080F0001C48FEF723FF010026D0887A48813046CD
:108100008030026F002A1DD0426FD1604167426FFC
:108110000021D160416FCC80426F01211181426FFB
:1081200002991171406F224600683946801C0BF09D
:1081300077FC281B05042D0C0FD03F19012002905D
:108140000098C9E70167E1E70748026B002A02D0FF
:108150000649022090470720C7E738460BF0C0FCCD
:108160000020C2E754FF0000CC690020AA5500009F
:1081700030B5C37D0146027A8031002B09D00B6FE8
:108180001B681A700B6F427A1B685A70096F096876
:1081900005E08B6E1A708B6E427A5A70896E1A4C9B
:1081A000437AE26841339B090D6815604D6855605C
:1081B0008D689560CD68D5600D6915614D69556113
:1081C0008D699561CD69D5610D6A15624D6A5562FB
:1081D0008D6A9562CD6AD5620D6B15634D6B5563E3
:1081E0008D6B9563CD6BD563403140325B1E1B06B2
:1081F0001B0ED9D1407A0549401D8008E268897C70
:108200008000115030BD0000206A0020CC690020A1
:10821000114A916B002902D0097B00290BD1116C06
:10822000002902D0497C002905D1916C002904D095
:10823000C979002901D0122070475070064A803257
:10824000517D002802D00620014301E0F9200140C1
:108250005175002070470000006C002070B538494F
:10826000C96B00296AD0364A0028946B02D00128D5
:1082700009D063E0002C61D0207B00285ED0FEF79F
:1082800093FB002070BD01260025F602002C10D1C2
:108290008847040018D026826682A5760720E076FB
:1082A000652005552649204606229C3166300BF094
:1082B000B7FB207B012841D0A07E010706D0000734
:1082C000000F012802D009E0032070BD08F086F9F4
:1082D0001C49097F8907890F88422FD0A07E01079A
:1082E000090FA17101280AD0208A628A80184008EB
:1082F00001229203A08290420BD9A28214E00620B0
:10830000A0821148E582C078324604210BF082FE3B
:108310000FE0022904D0062902D020280CD302E065
:10832000A02800D2A020A0821021002002F038F95D
:10833000E082E06F804770BD2020F4E7122070BD1E
:10834000006C0020CC690020006A002070B5044653
:108350000D480D46C26B002A03D0806B002802D066
:1083600004E0122070BD904700280AD0E206D20E29
:108370000277002C03D029461E300BF051FB002061
:1083800070BD032070BD0000006C0020FFB52949BE
:1083900081B0C86B0B9D1E461746002803D08C6B1E
:1083A000002C03D005E0122005B0F0BD804704008A
:1083B00015D0019820820298012100226082012FAD
:1083C0000FD0022F0FD0032F0FD0042F0FD0A27683
:1083D0002046603046712B78002B1AD10AE003202A
:1083E000E2E7A176F4E7062002E0022000E0112097
:1083F000A076EDE76B78002B0BD1AB78002B08D182
:10840000EB78002B05D12B79002B02D16B79002B57
:1084100009D001730A9941732046062229466E301D
:108420000BF0FEFA00E002730C98E0760D98E07213
:108430000020B9E7006C002010B5040024D01C49CE
:108440008A6B002A02D0107B00280BD1086C002810
:1084500002D0407C002805D1886C002804D0C07967
:10846000002801D00C2010BD012088701048062281
:108470002146A2300BF0D4FA62799309032B05D080
:10848000900908D0012B0BD0122010BD08480622FD
:108490002146A83008E0064806222146AE3003E017
:1084A000034806222146B4300BF0BAFA002010BD72
:1084B000006C002070B51921084D890148432863DC
:1084C000AC6F06E02078FF2802D0296B0BF01CFE71
:1084D000E46B002CF6D1002070BD0000006C002081
:1084E00010B50C461F494B6C002B05D00A6C0028B8
:1084F00004D0012807D00EE00C2010BD002A0AD0BD
:10850000FFF7A8FD2BE0002A07D01046417C012987
:1085100001D000290ED0122010BD9847002807D0A6
:10852000002101741022028342832D221154EDE7B1
:10853000032010BD028B012189038A4200D90183E7
:10854000428B018B8A4200D94183418B5522514392
:10855000090A8183017C01728475806C8047002048
:1085600010BD0000006C002070B505460C480C469C
:10857000C26B002A03D0806B002802D004E01220D6
:1085800070BD9047002808D0EA06D20E42772146F7
:108590003E300BF045FA002070BD032070BD000096
:1085A000006C002010B5FEF7E9F904480249416665
:1085B0000349816610BD000049F90000006C0020ED
:1085C000EDF9000010B504460920214660728031A3
:1085D000886E002811D00E228270886E08225831D1
:1085E000C01C0BF01DFA20462030C1780422114334
:1085F000C17062206073002010BD012010BD0121F8
:108600004172E8210958002905D005228A705221BB
:108610004173002070470120704701214172E82119
:108620000958002905D006228A7054214173002080
:10863000704701207047F8B51C4616460F46FEF7F6
:108640006DFC050002D0E879002801D00220F8BDB9
:108650002846FF300822394610300BF0E1F9E81DBA
:10866000FC300675310A4175A17BE07B0902411897
:10867000607B227B0004120680182E460818803684
:10868000B062A17AE07A09024018617A227A09047C
:10869000120689184018F062A179E07909024018A1
:1086A0006179227909041206891840183063A1788B
:1086B000E0780902401861782278090412068918C6
:1086C00040187063284640308179002904D0012188
:1086D000C1712021706850E00BF024FB024600209D
:1086E000C3001146D9402B18FF330133401C597683
:1086F0000428F5D30BF016FB02460020C3001146F8
:10870000D9402B18FF330133401C59770428F5D387
:10871000E81DF930C27E017F12028918827E437EF5
:1087200012041B06D2188918044671622034C27FD5
:10873000217812028918827F407F120400061018E7
:10874000081830620BF0EEFA02460020C300114612
:10875000D9402B18FF332133401C59700428F5D31E
:10876000A178607809024018E1782279090412069C
:1087700089184018B0637068402108437060002079
:10878000F8BD02224272E821095800290DD08A70F2
:108790004E22125CCA7001462031CA7808231A435F
:1087A000CA703221417300207047072070470000D3
:1087B000FFB50500364881B0C468164603D00B2DBE
:1087C00003D86D1E06E025250AE00C2D04D0262DC9
:1087D00004D8AD1EEDB203E0262501E0272D0FD110
:1087E000002E10D0012E19D0022E1AD0032E1BD02D
:1087F000042E24D0052E25D0062E26D0072E27D0D5
:10880000122005B0F0BD002704E0FAF7E3FBE11900
:1088100088707F1C02988742F7DB1EE0F021029AE5
:1088200018E0AA21029A15E0002704E0FAF7B0FB4D
:10883000E11988707F1C02988742F7DB0DE0FF2169
:10884000029A07E00021029A04E00F21029A01E057
:10885000029A5521A01C0BF0BDF93007000F2070C3
:10886000029860700498029A000601D5012100E088
:108870000021284602F0F4F8054800E000BFC17866
:108880000029FBD003490889401C08810020B8E773
:10889000206A0020006C0020022242728030826E2A
:1088A000002A05D007239370806EC17000207047A6
:1088B0000120704706214172E8210958002912D091
:1088C0000C220A4B8A709A7BCA701A8A0A71120AA1
:1088D0004A715A8A8A71120ACA71C17E4906490EC2
:1088E000C17600207047072070470000006C002010
:1088F000F8B51A4F054600263C6F0CE060786978A1
:10890000884206D10622A91CA01C0BF07BF8012886
:108910001ED02646A468002CF0D119210C200BF0A3
:108920009BF8040015D0687860700622A91CA01C72
:108930000BF076F8386F00280DD0002E00D0B46010
:108940000020A06005484030818D491C81850120B0
:10895000F8BD0020F8BD3C67F2E70000006C002085
:1089600070B5074D2C6F03E02046A4680BF0B8F8F3
:10897000002CF9D10020024928674031888570BD5C
:10898000006C00200249002008674031888570474C
:10899000006C002073B50A486D46046F0CE0694610
:1089A00060784978884206D10622A91CA01C0BF0E9
:1089B00029F8012803D0A468002CF0D100207CBD48
:1089C000006C0020F8B51F4F00263A68B400115D16
:1089D000A21808460091517848409178D27805460F
:1089E00051404D400BF0CDFB014638686940025DB7
:1089F0004A40025521184878897848400BF0C1FB5D
:108A00003968684061184A7842404A708878C97865
:108A100048400BF0B6FB3968684061188A784240DC
:108A20008A70C878009948400BF0ABFB3968684001
:108A30006118CA78761C4240F6B2CA70042EC4D3BC
:108A4000F8BD0000D848002070B531480921006801
:108A5000C9018162826C0721090703238A435B07EE
:108A6000D2188264836C0F2212030324934364039D
:108A70001B198364836CCC0023438364C36C0C1583
:108A8000A343C364436D802423434365C36B934373
:108A900022029A18C263C36B0A119343A4041B19E0
:108AA000C363C36BDC000123E4089B07E418C463C1
:108AB000C46D0C43C465C56D0C122543C565C56DF9
:108AC0000E133543C565C56D9543C565C56AA54398
:108AD0005C122C19C462C46A944305221206A218BF
:108AE000C262C26A032424032243C262C26A24010E
:108AF0002243C262026B120912010263026BF0246C
:108B0000A2430263026B8A43D118016370BD000067
:108B10006448002014480068C268FF2101318A437C
:108B2000C260826D0B029A43826542681A434260BA
:108B300082681A438260C2680A43C260014680317B
:108B4000CA68D205FCD500BF00BF00BFC968426833
:108B500009079A434260826D0F23DB019A43490D56
:108B60000A438265704700006448002010B51A4827
:108B70000068016D01231B049943016581685C0154
:108B800021438160C26810210A43C260C2688A43DF
:108B9000C26000BF00BF00BFC2680A43C260416834
:108BA000012212031143416001468031CA69D20596
:108BB000FCD500BF00BF00BFC969026DC906C90E60
:108BC0001A430265026D520952010A430265816827
:108BD000A143816010BD000064480020F0B5FF484B
:108BE00087B005686868FF21013188436860A86A1A
:108BF00009018843A862E86A10218843E862A868EE
:108C00004A031043A86068680843686068684008C1
:108C100040006860A86BF24A0321104089034018A5
:108C2000A86368680123184368602C468034206973
:108C30004001C10F20698001C00F0029F7D0002832
:108C4000F5D0206986066069B60EC003400E01901B
:108C50006868400840006860A86BE721104009027E
:108C60004018A86368681843686020694001C10F14
:108C700020698001C00F0029F7D00028F5D02069B5
:108C80008006800E04906069C003400E06906868FC
:108C9000400840006860A86BD321104009024018CA
:108CA000A86368681843686020694001C10F2069A3
:108CB0008001C00F0029F7D00028F5D02069800678
:108CC000800E039060692721C003400E0290039834
:108CD000301A06464843F9F765F80007216A000F85
:108CE0000909090108432062262070432721F9F76A
:108CF00059F80007226A000EF0218A4310432062CF
:108D0000252070432721F9F74DF80007226A000D4E
:108D10000F2109028A431043206224207043272137
:108D2000F9F740F80007226A000C0F2109038A4373
:108D300010432062232070432721F9F733F80007FE
:108D4000226A000B0F2109048A431043206222206B
:108D500070432721F9F726F80007226A000A0F213D
:108D600009058A4310432062700130182721F9F762
:108D700019F80007216A00090F273F06B943084385
:108D8000206270012721F9F70DF8216A0007090117
:108D90000909084320627001801B2721F9F702F8B6
:108DA0000007616A000F09090901084360621E207B
:108DB00070432721F8F7F6FF0007616A000EF022E2
:108DC0009143084360621D2070432721F8F7EAFFB2
:108DD0000007616A000D3A149143084360621C2049
:108DE00070432721F8F7DEFF0007616A000C3A1391
:108DF0009143084360621B2070432721F8F7D2FF9C
:108E00000007616A000B3A129143084360623046E2
:108E10001A2148432721F8F7C5FF0007616A000AB5
:108E20003A11914308436062304619214843272193
:108E3000F8F7B8FF0007616A0009B94308436062A8
:108E40003046182148432721F8F7ACFF616A000734
:108E50000901090908436062304617214843272168
:108E6000F8F7A0FF0007A16A000F090909010843EC
:108E7000A062162070432721F8F794FF0007A16A2B
:108E8000000EF02291430843A06215207043272171
:108E9000F8F788FF0007A16A000D3A1491430843D0
:108EA000A062142070432721F8F77CFF0007A16A15
:108EB000000C3A1391430843A0621320704327210A
:108EC000F8F770FF0007A16A000B3A1291430843BC
:108ED000A062122070432721F8F764FF0007A16AFF
:108EE000000A3A1191430843A0623001301827214B
:108EF000F8F758FF0007A16A0009B9430843A062C8
:108F000030012721F8F74EFFA16A0007090109097E
:108F10000843A0623001801B2721F8F743FF0007B8
:108F2000E16A000F090909010843E06230460E2199
:108F300048432721F8F736FF0007E26A000EF021C8
:108F40008A431043E06230460D2148432721F8F759
:108F500029FF0007E26A000D39148A431043E062DA
:108F600030460C2148432721F8F71CFF0007E26A2E
:108F7000000C39138A431043E06230460B2148430A
:108F80002721F8F70FFF0007E26A000B39128A4326
:108F90001043E06230460A2148432721F8F702FFD8
:108FA0000007E26A000A39118A431043E062F000C8
:108FB00030182721F8F7F6FE0007E16A00093A4663
:108FC00091430843E062F0002721F8F7EBFEE16AE5
:108FD0000007090109090843E06203E06448002032
:108FE000FF00FEFFF000801B2721F8F7DBFE0007E3
:108FF000216B000F0909090108432063304606214F
:1090000048432721F8F7CEFE0007010E206BF0221F
:10901000904301432163B00030182721F8F7C2FEC6
:109020000007226B000D39148A4310432063B000FF
:109030002721F8F7B7FE0007226B000C39138A438B
:1090400010432063700030182721F8F7ABFE0007AB
:10905000010B206B3A1290430143216370002721DA
:10906000F8F7A0FE0007226B010A38118243114372
:10907000216330462721F8F795FE0007226B00098F
:1090800039468A4310432063206B000100092063A6
:1090900004990398471A28213846F8F783FE0007F9
:1090A000616B000F090909010843606378002821FA
:1090B000F8F778FE0007616B000EF0229143084339
:1090C0006063780038182821F8F76CFE0007616BA0
:1090D000000D0F221202914308436063B80028215B
:1090E000F8F760FE0007616B000C0F22120391433A
:1090F00008436063B80038182821F8F753FE0007CA
:10910000616B000B0F221204914308436063062039
:1091100078432821F8F746FE0007616B000A0F220A
:109120001205914308436063F800C01B2821F8F73B
:1091300039FE0007626B00090F2109068A431043BC
:109140006063F8002821F8F72DFE616B0007090124
:10915000090908436063F80038182821F8F722FE4F
:109160000007A16B000F090909010843A0633846F5
:109170000A2148432821F8F715FE0007A26B000ECC
:10918000F0218A431043A06338460B21484328212D
:10919000F8F708FE0007A26B010D0F2000028243C2
:1091A0001143A16338460C2148432821F8F7FAFD02
:1091B0000007A26B010C0F20000382431143A1633F
:1091C00038460D2148432821F8F7ECFD0007A26B33
:1091D000000B0F2109048A431043A06338460E2177
:1091E00048432821F8F7DEFD0007A26B010A0F2093
:1091F000000582431143A1633801C01B2821F8F701
:10920000D1FD0007A26B00090F2109068A43104314
:10921000A06338012821F8F7C5FDA16B00070901FB
:1092200009090843A063380138182821F8F7BAFD66
:109230000007E16B000F090909010843E0633846A4
:10924000122148432821F8F7ADFD0007E26B000E1C
:10925000F0218A431043E063384613214843282114
:10926000F8F7A0FD0007E26B000D0F2109028A4309
:109270001043E0633846142148432821F8F792FD53
:109280000007E26B010C0F20000382431143E163EE
:109290003846152148432821F8F784FD0007E26B82
:1092A000010B0F20000482431143E163384616216D
:1092B00048432821F8F776FD0007E26B000A0F21EA
:1092C00009058A431043E0633846172148432821A3
:1092D000F8F768FD0007E26B00090F2109068A43D1
:1092E0001043E0633846182148432821F8F75AFD17
:1092F000E16B0007090109090843E06338461921B9
:1093000048432821F8F74EFD0007216C000F09099A
:1093100009010843206438461A2148432821F8F7F8
:1093200041FD0007226C000EF0218A4310432064A7
:1093300038461B2148432821F8F734FD0007226CEA
:10934000000D0F2109028A431043206438461C2176
:1093500048432821F8F726FD0007226C000C0F2156
:1093600009038A431043206438461D2148432821BD
:10937000F8F718FD0007226C000B0F2109048A433F
:109380001043206438461E2148432821F8F70AFD7F
:109390000007226C000A0F2109058A43104320644C
:1093A0007801C01B2821F8F7FDFC0007226C00099A
:1093B0000F2109068A431043206478012821F8F719
:1093C000F1FC216C000709010909084320647801B8
:1093D00038182821F8F7E6FC0007616C000F09092E
:1093E0000901084360643846222148432821F8F7E0
:1093F000D9FC0007010E606CF022904301436164C8
:109400003846232148432821F8F7CCFC0007626C3A
:10941000010D0F200002824311436164384624216C
:1094200048432821F8F7BEFC0007626C000C0F21AE
:1094300009038A43104360643846252148432821A4
:10944000F8F7B0FC0007626C000B0F2109048A4397
:10945000104360643846262148432821F8F7A2FCCF
:109460000007626C010A0F2000058243114361640A
:109470003846272148432821F8F794FC0007626CFE
:1094800000090F2109068A431043606438462821E9
:109490004843F8F787FC616C000709010909084394
:1094A00060643846292148432821F8F77BFC0007EF
:1094B000A16C000F090909010843A06438462A215C
:1094C00048432821F8F76EFC0007A26C000EF0213B
:1094D0008A431043A064069A02983946801A0A22E9
:1094E00000905043F8F75EFC082108430007A16C88
:1094F000000D0F22120291430143A16400983946E6
:10950000C2008018F8F74EFC082108430007A16C40
:10951000000C0F22120391430143A16400983946C5
:10952000C000F8F73FFC082108430007A16C000BBE
:109530000F22120491430143A16400983946C200EE
:10954000101AF8F72FFC082108430007A16C000A45
:109550000F22120591430143A16400980622394667
:109560005043F8F71FFC082108430007A16C0009CD
:109570000F22120691430143A164009839468200EC
:109580008018F8F70FFC08210843A16C00070901B7
:1095900009090143A164009839468000F8F702FCEC
:1095A000082108430007E16C000F09090901014384
:1095B000E1640098394642008018F8F7F3FB08216F
:1095C00008430007E16C000EF02291430143E1647F
:1095D000009839464000F8F7E5FB082108430007EA
:1095E000E16C000D0F22120291430143E164394600
:1095F0000098F8F7D7FB082108430007E16C000C3E
:109600000F22120391430143E16431460020F8F731
:10961000C9FB0007E16C000B0F22120491430143C8
:10962000E164029A01983146871A3846F8F7BAFB86
:109630000007E16C000A0F22120591430143E16427
:1096400031467800F8F7AEFB0007E16C00090F2205
:10965000120691430143E164780031463818F8F767
:10966000A1FBE16C0007090109090143E1643146EE
:10967000B800F8F797FB0007216D000F09090901F1
:1096800001432165B80031463818F8F78BFB000715
:10969000216D000EF02291430143216506203146E1
:1096A0007843F8F77FFB0007216D000D0F221202AF
:1096B000914301432165F8003146C01BF8F772FB66
:1096C0000007216D000C0F22120391430143216515
:1096D0003146F800F8F766FB0007216D000B0F22FA
:1096E0001204914301432165F80031463818F8F718
:1096F00059FB0007216D000A0F2212059143014317
:1097000021650A2031467843F8F74CFB0007216DAC
:1097100000090F2212069143014321656968102058
:10972000814369606968490849006960A96A020261
:109730001143A962E96A0143E962A86B81090398B0
:1097400089010143A963A86B7F2109068843029917
:1097500009060843A86307B0F0BD0000034800688D
:109760004168FF2201321143416070476448002084
:10977000FEB51F48816B0091816B009A9142F9D12F
:109780001C4F1D4D397D1926C9071046002905D0EB
:10979000294600F0EBFC8904800B04E0314600F020
:1097A000E5FCC905400A084300900020134C0190D5
:1097B000A0690099884219D0884201D8081A13E09C
:1097C000397D0F48C90705D0294600F0CFFC890430
:1097D000800B04E0314600F0C9FCC905400A08438B
:1097E000A169401A009940180190A1610198FEBD3D
:1097F00000100040CC69002033030000006A002004
:109800000000C0A8002908D0002A02D105E008C83D
:1098100008C2491EFBD200207047FD20704738B5B2
:109820000D46040019D0002D17D00321684608F01A
:10983000EBFC6946887840218006800E0843694623
:1098400088702A46204609F006FB040006D1032250
:109850006946E81C0AF0E4F800E00224204638BD1E
:10986000F7B58CB00C9815460F46002831D0002D66
:109870002FD0381D0A9080B253210AF0EDF8040071
:109880003BD002F035F806463A46201D0C990AF006
:1098900065FAF0B20990E0703004000E0890A070F4
:1098A0003002000E07906070370E277002F01AF831
:1098B0000146102201A80AF051FA082000900A98E7
:1098C00005AB82B2214601A809F032FA060002D0A7
:1098D0000FE0022612E0099828700898687007982F
:1098E000A870EF70082205A9281D0AF037FA02F0C7
:1098F00005F820460AF0F4F800E0132630460FB0D1
:10990000F0BD000010B5024600F01EF80448062124
:1099100082701046FCF74AFE024805F087FE10BD33
:1099200072480020B523010005480649C0780007A9
:1099300002D508460C3000E0002048600020704747
:1099400072480020AC4800200A49002008604860A6
:109950008860084808490C3001600849416008499E
:10996000816008490C300160074941600749816006
:1099700070470000AC48002057320100552201001A
:10998000FD9A0000EF360100F12801007127010067
:1099900070B506460D46084605F0F8FC00280ED0C6
:1099A000446B002C06D0E078022805D0032803D0B1
:1099B000042801D0122070BDA088A84201D0022046
:1099C00070BD10223146E01D0AF02AF820462C30E6
:1099D0001021054608F018FC23461C332A46E11DD9
:1099E000204609F065FA207802210028607803D02B
:1099F000032807D1617009E0042802D0032803D0AE
:109A000000E06170002070BD05206070204608F005
:109A1000CFFB70BDF8B50D46080417D51B4EB078C6
:109A20000AF01CF9040009D008F05EFE002809D1F4
:109A30007078FF2806D021460AF048F90120C003BB
:109A40006840F8BD20460AF0E1F8F7E7E80701278B
:109A5000002804D008F0BEFC28467840F8BD002D50
:109A600012D001240CE03846A04086B2354205D021
:109A7000304609F04FF928467040F8BD641CE4B246
:109A800005F09AFDA042EED80020F8BD72480020F3
:109A90007CB50D46040015D0002D13D00322E91C1F
:109AA000684609F0BDFF6946887840218006800E2F
:109AB00008436946887001AA204609F0CCF90400E1
:109AC00002D009E0022407E00322294601A809F098
:109AD00099FF012800D0012420467CBD0548064995
:109AE000C078400702D50846183000E000208860A2
:109AF0000020704772480020AC480020FFB50F4698
:109B000083B01E4614465321102009F0A5FF05001E
:109B100029D0002F22D069460C72200A48721022E8
:109B2000002128460AF056F8394628460C9A09F0D2
:109B300077FF002E05D008223146684609F070FFF5
:109B400004E00822002168460AF044F82B4602AAE5
:109B500069460398FCF7C0F8044600E00224284652
:109B600009F0BEFF00E01324204607B0F0BDFFB5AA
:109B700081B01F46039805F009FC060005D0706B04
:109B80000025002804D011253AE0022005B0F0BDE0
:109B90001320FAF751FDC4B21420FAF74DFDC1B2FB
:109BA000002F2CD0387EA04229D3884227D85321B9
:109BB000702009F051FF0446706320001DD0702210
:109BC00000210AF007F800206070019921700299C5
:109BD000A1700399A180E765A061E0700198002859
:109BE00003D0204608F0F6FA054601206070002DEB
:109BF00006D0304608F0B4FA02E0132500E0022552
:109C00002846C3E7FFB587B00998109D0E46002887
:109C10001FD0002D1DD0079805F0B8FB04001BD005
:109C20005321102009F018FF019000285FD06978B7
:109C3000287809024018A978EA78090412068918D8
:109C400041180691A06A884208D3401C06D002241D
:109C500049E002200BB0F0BD1420FBE7002E02D03B
:109C6000207980073ED50822002102A809F0B2FF22
:109C70000A9F53213F1DB8B209F0EEFE06002FD017
:109C8000301D0A9A09990AF069F8042229463046DB
:109C90000AF064F821461022183101980AF05EF8A3
:109CA00008200090BAB202AB3146019809F040F8A2
:109CB00004000CD1082202A904A80AF04FF80822D7
:109CC000291D04A809F09EFE012804D00124304675
:109CD00009F006FF07E00699079802F0FBFEF6E799
:109CE000132400E00124019809F0FAFE00E0132497
:109CF0002046AFE70D480068417842794270427AC9
:109D00004271427B427241738178827A82708172A1
:109D10008179827B82718173C178C27BC270C27A81
:109D2000C273C279C272C17170470000D848002066
:109D300030B50948094D046800210020820012193D
:109D4000535C401CEB5CC0B253540428F6D3491C4E
:109D5000C9B20429F1D330BDD8480020AC4301007A
:109D600070B50C46014620040AD5084609F076FF76
:109D7000002801D009F04AFF0120C003604070BDF7
:109D80006004FCD0002632462046D040C00713D0E5
:109D9000002901D00F2000E000200B4980184968FD
:109DA000C00045180120904086B22968686888473D
:109DB00000202860686003E0521CD2B20F2AE3D36F
:109DC0002046704070BD00001C46002070B509F0B0
:109DD000D1FE1C2200211D4809F0FCFE1B48202258
:109DE0000021503009F0F6FE194D0020286168610D
:109DF0001648164C1C30007F50348107890F8008AC
:109E00000818410040180D30C0B2A0700621484328
:109E10002121F03009F020FE6860F030A860A178C0
:109E200089000818E86009F013FF09F0D7FF60788F
:109E3000084A8100A86842506178491CC9B2617023
:109E4000890042506078401C607070BDB06900208D
:109E50001C460020619D000010B508490246487864
:109E60008B78984207D2064C8300A468E2504A7867
:109E7000521C4A7010BDFF2010BD0000006A002077
:109E80001C460020072902D2014A89005050704721
:109E9000B0690020FEB5844D02E0804700F0C0FEAE
:109EA00028680028F9D10124A0002858002807D0EC
:109EB00080477D481C30407D002801D0F8F728FFFE
:109EC0002868002875D1641CE4B2072CECD3764CCA
:109ED000764E50346278F06821784B00C35A002BDC
:109EE00004D1491CC9B221709142F5D3C9B2914243
:109EF00011D24A00815A002383522078B36882002D
:109F00009A5890472178F2684900535A03435352B4
:109F10002078401C207020786178884201D300208E
:109F2000207061480068002843D17069002840D043
:109F3000804700283DD0616905460918616100210C
:109F4000C9435A4821610669002E29D00027B0680C
:109F5000A84201D8002000E0401BB06052481C30ED
:109F6000406A002804D02169B068814200D920618C
:109F7000B06800280DD1718800291BD0307809F015
:109F8000F7FE7068002801D0B06002E0B0680028D9
:109F900010D0708800280DD03746F668002ED6D134
:109FA000414D1C35686A00287DD000203F4A617809
:109FB00014E078E0002F06D0F068F8603046F668CC
:109FC00009F08EFDEAE73948F1680161F6E7D668E5
:109FD0004300F35A002B66D1401CC0B28142F6D830
:109FE0003149032082008A58002A5CD1401CC0B24B
:109FF0000728F7D301A8FDF781F82D4A411C25D089
:10A00000EB7C019EB3424ED221694F1C17D0287DB4
:10A01000C00702D01420414302E0292041434908EF
:10A020008B4240D28E4200D231462248CE1A816BFA
:10A030000091816B009B9942F9D198191DE09842DB
:10A0400001D3C01A1EE0C01A80181BE02069411C11
:10A0500029D0297DC90702D01421484302E02921D3
:10A0600048434008E97C81421DD2461A1148816B61
:10A070000091836B8B42FAD18819904202D30C492C
:10A0800049424018696A002800D1104688470006F6
:10A09000000E08D12089002805D0F8F7BDFFFCF795
:10A0A000EFFAF8F7ADFDFEBDB06900201C460020B8
:10A0B0000000C0A80010004010B50548C06A002884
:10A0C00000D08047034800F007F8002010BD0000D2
:10A0D000CC6900207197000010B5034948618047A2
:10A0E0000249886110BD00001C460020006A002063
:10A0F000F0B5144EFD23757A84247472124CA7684F
:10A10000002F07D0A77B002F04D0A489E71FFF3FB3
:10A11000FA3F02D07572FF20F0BD7D24E402A04218
:10A120000AD34027491E07D3706008CA33609A23B8
:10A130003372B37A7B4002D075721846F0BD001DB1
:10A14000F0E7000000180040CC6900200FB410B503
:10A1500003A9044B044A029800F03CF810BC08BC68
:10A1600004B01847651A0000E0480020F8B5040C58
:10A170008BB2264682B25E430D0C1046370C584314
:10A18000360480190021794116466E43370C360497
:10A190008019794126466E438919F8BD30B474465A
:10A1A000641E2578641CAB4200D21D46635D5B00D3
:10A1B000E31830BC184702E008C8121F08C1002A83
:10A1C000FAD170477047002001E001C1121F002A38
:10A1D000FBD17047FFB58FB00F460446002606E05E
:10A1E00025280AD0129A11999047641C761C207871
:10A1F0000028F5D1304613B0F0BD00250121A14A59
:10A20000009500E00543641C23780846203B9840F5
:10A210001042F7D120782E2815D10420054360780C
:10A22000641C2A280AD101CF641C00900BE000991D
:10A230000A22514330394018641C009020780146AE
:10A2400030390929F3D920786C280ED004DC4C2849
:10A2500013D06A2812D104E074280ED07A280DD1C8
:10A260000BE001204005054307E001210905627864
:10A270000D43824201D16D18641C641C207886460F
:10A2800069284AD008DC0028B4D058286DD063284B
:10A2900010D0642808D140E070286BD0732812D009
:10A2A000752860D0782860D0129A7046119990472E
:10A2B000761CE5E03878694608720020487202A8EA
:10A2C0000190012003E0386801900020C0433F1D49
:10A2D00069070CD5002500E06D1C00998D420FDA4E
:10A2E0008542F9DB0199495D0029F5D108E0002597
:10A2F00000E06D1C8542FCDB0199495D0029F8D125
:10A30000761907E0019801990078491C0191129A89
:10A31000119990476D1EF5D2B2E00A2002900021FB
:10A320006802400F039102280CD001CFC117844668
:10A3300000290DDA624608465242002181419446C6
:10A340002D2008E0FF1DFF08FF0003CF8446EFE744
:10A35000280504D52B206A46107401203CE0E8074C
:10A360003AD02020F7E70A2000E0102000210391D6
:10A37000029007E0102002900021042005430820ED
:10A38000039100906802400F022810D001CF0021F5
:10A39000844600200D9028071FD5704670280CD0E9
:10A3A000029A1020039B42401A430CD015E0FF1D77
:10A3B000FF08FF0003CF8446EBE740206A46107495
:10A3C00001200D900CE06046084306D030206A461C
:10A3D00010747046507402200D907046582804D0B6
:10A3E00029A001900DA80E900DE02CA0F9E7604681
:10A3F000039B029AF7F749FD019B84469B5C0E9AEA
:10A40000521E0E92137060460843F0D10E9805A9B3
:10A41000081A20300190680701D5009801E001205A
:10A4200000900199884203DD01460198081A00E076
:10A4300000200025009006E004A8129A405D1199C2
:10A4400090476D1C761C0D988542F5DB04E0129A4E
:10A45000302011999047761C0099481E00900029E1
:10A46000F5DC08E00E980E990078491C0E91129ABE
:10A4700011999047761C0199481E01900029F1DC42
:10A48000641CB4E6092801003031323334353637E4
:10A490003839616263646566000000003031323330
:10A4A00034353637383941424344454600000000D0
:10A4B000FFB583B00C9C1646002C01D0002708E0A5
:10A4C00001270398F8F796F90421FCF7CBF804006C
:10A4D00014D0267004980125002805D0049A601C29
:10A4E00006999047401C85B2300614D51021039878
:10A4F00005F0D0F8002804D0192616E0132007B084
:10A50000F0BD621929462046FFF7AAF90C35064628
:10A51000ADB2002809D104206946088001940D815C
:10A520000398FCF759F80600E9D0002F02D0204626
:10A5300009F0D6FA3046E2E7F8B5074606980090EB
:10A540001E4614463846FFF7B3FF05000BD10748F7
:10A550000268002A07D0012C02D13078401CC4B216
:10A560002146384690472846F8BD00007C48002028
:10A5700030B5437803245B1D2343C45CE50601D555
:10A58000012030BD002903D0210601D5022030BDB5
:10A59000002A03D0C0182038C07F1070002030BDC2
:10A5A00070B50D46044609F0BDFB2D1B0246002385
:10A5B000E9172846F7F70AFC081980B270BD70B594
:10A5C0000D46044609F0AEFB00232D1B024628462B
:10A5D0001946F7F7FBFB081970BD70B50D46044628
:10A5E00009F0A0FB2D1B02460023E9172846F7F7C8
:10A5F000EDFB0819C0B270BDF0B5364E9446326816
:10A6000013689B0713D0136DDB08DB001365136819
:10A6100008242343136013681B0703D500BF00BF42
:10A6200000BF00BF136DDB08DB005B1C13652A4F06
:10A630003B68DC6A07221205944301225205A218E6
:10A64000DA62DD6A072424060522A5431206AA1849
:10A65000DA62224A1368DA6A92089200921CDA627D
:10A660001D680122120715431D601A686546D2094C
:10A67000D2016D066D0E2A431A6098601861596008
:10A68000D960306841680123194341603968144D2D
:10A6900000200A4680322D890EE01769FF0108D597
:10A6A000C86A072212051043C862C86AA043C8627C
:10A6B00004E000BF00BF401C8542EEDC0948006892
:10A6C000002804D0C1680A68406902430A60306803
:10A6D0000360F0BD38460020644800205C4800203C
:10A6E000006A00203C46002010B5144A5921136826
:10A6F0001965134909680B684024DB092043DB0115
:10A700004006400E03430B600E4808610E48C860C7
:10A710000E490020487010684168490849004160AE
:10A720000B480068002804D0C1680B6840690343E7
:10A730000B6011680120086010BD00003846002041
:10A740005C4800202941767155555500206A00204B
:10A750003C46002010B514480068016889070ED0F7
:10A76000016DC908C9000165016808221143016033
:10A770000168090703D500BF00BF00BF00BF00226A
:10A7800002650A4B186800280AD041680C68806886
:10A7900004430C60186801690B68406903430B604F
:10A7A0000348C27110BD0000384600203C4600201E
:10A7B000206A0020FFB5804C064620680D460168DF
:10A7C00081B0174689071AD0016DC908C900016513
:10A7D00001680823194301607848407D002801D0B2
:10A7E000F8F796FA20680168090703D500BF00BF93
:10A7F00000BF00BF016DC908C900891C0165704A0E
:10A800001068C16A07231B05994301235B05C9181A
:10A81000C162C16A07231B06994305231B06C91899
:10A82000C1626848006801687B06C909C9015B0EFE
:10A8300019430160866006614560C560C16A890888
:10A840008900C162016801231B07994301605E4DC5
:10A850002B6898680499400B400308439860564859
:10A860000068416801242143416058488178A14330
:10A8700081701168564E00200C46803432890FE0FA
:10A880002669F60109D5CC6A072636053443CC6221
:10A89000CC6A3601B443CC620AE000BF00BF401C62
:10A8A0008242EDD804E000BF00BF00BF00BF401CE3
:10A8B0008242F8D89868474BC004C00C3A2805D9A2
:10A8C0001F6830204349C043803108604248006817
:10A8D000002804D001680A68806802430A6036488C
:10A8E00002210068016028688068C004C00C3A2812
:10A8F00060D900BF00BF00BF00BF00BF00BF00BFE6
:10A9000000BF00BF00BF00BF00BF00BF00BF00BF4F
:10A9100000BF00BF00BF00BF00BF00BF00BF00BF3F
:10A9200000BF00BF00BF00BF00BF00BF00BF00BF2F
:10A9300000BF00BF00BF00BF00BF00BF00BF00BF1F
:10A9400000BF00BF00BF00BF00BF00BF00BF00BF0F
:10A9500000BF00BF00BF00BF00BF00BF00BF00BFFF
:10A9600000BF00BF00BF00BF00BF00BF00BF00BFEF
:10A9700000BF00BF00BF00BF00BF00BF00BF00BFDF
:10A9800000BF00BF00BF00BF00BF00BF00BF00BFCF
:10A9900000BF00BF00BF00BF00BF00BF00BF00BFBF
:10A9A00000BF00BF00BF00BF00BF00BF00BF00BFAF
:10A9B00000BF1F6005B0F0BD38460020CC69002004
:10A9C000644800205C48002060480020206A002085
:10A9D000006A002000E100E03C46002010B51D495F
:10A9E00009688A68520B520302438A603A282ED9BA
:10A9F000194A1168194883689B029B0E3E2BFAD0B6
:10AA000083681B0CDB439B060CD083689B029B0E68
:10AA1000332B03D283681B0C9B06ECD1FFF79AFE05
:10AA2000002010BD30230C4CDB438034236083684E
:10AA30001B0CDB439B06FAD083689B029B0E302BDA
:10AA400004D383689B029B0E332BF0D3116001204B
:10AA500010BD00006048002000E100E000C200409E
:10AA6000F0B5614E04463068174600680D46800711
:10AA700001D0FFF76FFE31685A2008655B49002D51
:10AA80000868026809D04023D2091C43D20163063A
:10AA90005B0E1A430260564A07E0D209D2016306F0
:10AAA0005B0E1A430260524AD243826009685148E1
:10AAB0004860514A11688868400B400338438860F9
:10AAC0004E4B0020D870306843685B085B004360E1
:10AAD0004B4B00201B8904E000BF00BF00BF00BF3C
:10AAE000401C8342F8D88868464BC004C00C3A2802
:10AAF00005D91D6830204349C04380310860424871
:10AB00000068002804D001680C68806804430C6069
:10AB100031680220086010688068C004C00C3A28C0
:10AB200060D900BF00BF00BF00BF00BF00BF00BFB3
:10AB300000BF00BF00BF00BF00BF00BF00BF00BF1D
:10AB400000BF00BF00BF00BF00BF00BF00BF00BF0D
:10AB500000BF00BF00BF00BF00BF00BF00BF00BFFD
:10AB600000BF00BF00BF00BF00BF00BF00BF00BFED
:10AB700000BF00BF00BF00BF00BF00BF00BF00BFDD
:10AB800000BF00BF00BF00BF00BF00BF00BF00BFCD
:10AB900000BF00BF00BF00BF00BF00BF00BF00BFBD
:10ABA00000BF00BF00BF00BF00BF00BF00BF00BFAD
:10ABB00000BF00BF00BF00BF00BF00BF00BF00BF9D
:10ABC00000BF00BF00BF00BF00BF00BF00BF00BF8D
:10ABD00000BF00BF00BF00BF00BF00BF00BF00BF7D
:10ABE00000BF1D60F0BD0000384600205C4800201A
:10ABF000294176715555550060480020206A002093
:10AC0000006A002000E100E03C4600200249C860E4
:10AC10000249802008717047006A0020206A0020E5
:10AC200008B51148407D002801D0F8F771F80F4BA6
:10AC30001879000612D50E48816B0091816B009A3D
:10AC40009142F9D10B491046C9680122814202D8CC
:10AC5000401A02D502E0081A00D51A710648806928
:10AC6000002800D0804708BDCC690020206A002061
:10AC700000100040006A0020B069002010B50C46AA
:10AC800004F09CFB002804D040882146FAF779FFA5
:10AC900010BD122010BD002917D0002815D00128A2
:10ACA00004D0022805D0032807D00CE04879C02240
:10ACB00007E048798006800E04E048798006800E1F
:10ACC0004022104348710120704700207047000067
:10ACD00010B5054C606B002803D008F097FF0020EA
:10ACE0006063207E607610BDB4470020F0B54D4D06
:10ACF0000746686B87B00E4600281CD1002F7DD018
:10AD0000002E7BD0384600F04FFA6876297E8842C4
:10AD100011D300240AE0E96B200140180622FF212C
:10AD200008F061FE002805D1641CE4B2287E84424C
:10AD3000F1D3C4B26C76687E297E884270D2696B8A
:10AD400000290DD08A680024002A27D00621484314
:10AD50002130C0B21C2109F0BFF8686B846050E05C
:10AD6000062148432030C0B23A46102109F0B4F819
:10AD70001822FF21684608F02DFF687E6A46703071
:10AD8000C0B2182109F0A8F8687EE96B00014018EC
:10AD90001022394608F044FE6E6332E00A69002A48
:10ADA00009D0062148432230C0B21C2109F094F892
:10ADB000686B046125E04A69002A09D006214843EE
:10ADC0002330C0B2102109F087F8686B446118E0A5
:10ADD000CA68002A18D0062148432430C0B2102186
:10ADE00009F07AF8686B0621C268687E1032484321
:10ADF0002530C0B2042109F06FF800E010E0686B64
:10AE0000C460002007B0F0BD687C002801D000F0CD
:10AE100083FBA87C002801D000F046FB00F0E6FB95
:10AE20000120EFE7B4470020F7B588B004462022A0
:10AE30000021684608F0CEFE6A4614805B4804256F
:10AE4000817B1177FF2101310A9E4A008B00022489
:10AE5000002E50D087786E463771C7787771069E7E
:10AE60004079BC467608C7077600FF0F3E4306963A
:10AE70008607069E01D5264300E0A6430696C60631
:10AE80004A4F069E01D50E4300E08E43069681068A
:10AE900006993E4601D5114300E0914306914106D3
:10AEA000069901D5194300E09943400706910846E9
:10AEB00001D5284300E0A84306906046002805D04D
:10AEC00001A810223A49023008F0AAFD3179002980
:10AED00005D00998002802D00698204306906846BD
:10AEE000807D002900D0012108436946887571786A
:10AEF00050E0042150E0077A6E463771477A777147
:10AF0000069EC07ABC467608C7077600FF0F3E4310
:10AF100006968607069E01D5264300E0A6430696C0
:10AF2000C606224F069E01D50E4300E08E430696CC
:10AF3000810606993E4601D5114300E091430691F2
:10AF40004106069901D5194300E09943400706914F
:10AF5000084601D5284300E0A84306906046002833
:10AF600006D0134901A810221031023008F058FD14
:10AF7000B17A002905D00998002802D0069820430C
:10AF800006906846807D002900D00121084369466B
:10AF90008875F1790029ACD10843694688756846FF
:10AFA0000A99F9F75BF90BB0F0BD0000B447002037
:10AFB000346B0020F0B5064687B0062041430C9D57
:10AFC0001446082B1BD02131CFB21C220021684629
:10AFD00008F000FE6A461C21384608F039FF0028B8
:10AFE0000BD16846807EC01F092806D8E107C90F2B
:10AFF0002B466A463046F9F783F907B0F0BD223197
:10B00000E2E7000070B500252C460A4E0CE0F16B1B
:10B01000200140180622FF2108F0E5FC002801D19C
:10B020006D1CEDB2641CE4B2307E8442EFD328463E
:10B0300070BD0000B44700207FB50D46062148438F
:10B04000044616462034E0B26A46102108F000FF9C
:10B05000002806D10622FF21684608F0C4FC00281B
:10B0600002D0002004B070BD68468089002EC3B2B3
:10B0700002D02B43DBB200E0AB4398420AD06846D3
:10B080008381E0B26A46102108F026FF0248007D65
:10B0900008F0BEFE0120E5E7B447002070B50020AF
:10B0A0000446064D04E0204600F00AF8641CE4B2B1
:10B0B000297E8C4201D20028F5D070BDB447002013
:10B0C000F0B5384E0546707E91B0854209D1012118
:10B0D000F07D08F06DFC0221F07D08F069FCFFF7BF
:10B0E000F7FD2C460620444327462037F8B207AA2E
:10B0F000102108F0ADFE002806D10622FF2107A886
:10B1000008F071FC002803D00025284611B0F0BDDE
:10B110001022FF2107A808F05DFD1C22FF216846D0
:10B1200008F058FD1822FF210BA808F053FDF8B2D3
:10B1300007AA102108F0D0FE074620462130C0B2F1
:10B140006A461C2108F0C8FE074320462230C0B2E0
:10B150006A461C2108F0C0FE074320462330C0B2D7
:10B160006A46102108F0B8FE074320462430C0B2DA
:10B170006A46102108F0B0FE07432534E0B26A4663
:10B18000042108F0A9FE044670353C43E8B20BAA3E
:10B19000182108F0A1FE20430546307D08F038FE56
:10B1A000B3E70000B447002070B5064600240A4DFE
:10B1B0000CE0E96B200140180622314608F022FC21
:10B1C000002801D0204670BD641CE4B2287E844271
:10B1D000EFD3C0B270BD0000B4470020002293003E
:10B1E000CB5A834202D1900040187047521CD2B211
:10B1F000062AF4D3002070477FB50D460D49097E1D
:10B2000088420CD2002D0AD0062148432030C0B21B
:10B210006A46102108F01CFE040003D007E002205B
:10B2200004B070BD06226946284608F0F9FB2046A6
:10B23000F6E70000B44700201FB506214843203040
:10B24000C0B26A46102108F003FE002802D0002098
:10B2500004B010BD68468089C0B2F9E700218A00B9
:10B26000835A491CDB43835212189378C9B2DB43DB
:10B2700093700629F3D3704770B500241E4E1FE06B
:10B28000F06B25012A182046062148432030C0B221
:10B29000102108F0DDFD002810D0F06B06222818E0
:10B2A000FF2108F097FCF06B06222818FF21801D73
:10B2B00008F090FCF16B002069188881641CE4B2EE
:10B2C000307E8442DCD3FFF79DFE317E8842B07E23
:10B2D00002D10121084301E040084000B076707CB3
:10B2E000002801D000F018F9B07C002801D000F04F
:10B2F000DBF800F07BF970BDB447002010B50349BE
:10B300004088C97DF9F734FF10BD0000B447002024
:10B3100070B50E460546062148438AB014462030D3
:10B32000C0B206AA102108F093FD002846D10622DB
:10B33000FF2106A808F057FB00283FD17035E8B27E
:10B340006A46182108F084FD002834D16846FFF7CA
:10B3500085FF002E06D069463046FFF73FFF0028E4
:10B360000DD015E018220021684608F03CFB0028AB
:10B3700021D118220021684608F02CFC10E0002C96
:10B380001CD069460020FFF729FF002816D0068050
:10B390008178A1420FD08470002C01D1002101805E
:10B3A00007490120C8736846FFF758FFE8B26A46AC
:10B3B000182108F091FD01200AB070BD0020FBE7C4
:10B3C000B447002070B501780125B02907D0B12914
:10B3D00013D0D02923D1F8F7A9F805461FE0044679
:10B3E00000791E2803D160880021F8F705FA20466D
:10B3F00021790830FAF7BCFA11E0017900290ED161
:10B40000084C0026E6730289C1884088F8F7F0FBF3
:10B41000E07B002803D0E673207D08F0F9FC284685
:10B4200070BD0000B447002070B51C4C0646A06BF0
:10B430001B4D86B000280BD120461C300090022303
:10B44000184A29460120F9F73DFFA063002823D0C0
:10B45000FF2303930222002105A86B4607C304AB18
:10B46000A28B3046A16BF9F715FD002808D168467C
:10B47000028A002A04D0A06B41893046F8F7B8FB55
:10B480000023A28B2946A06BF9F756FFA063002882
:10B4900002D0002006B070BD0120FBE7B4470020B9
:10B4A000FFFF000040430100F0B589B0FAF786FBCA
:10B4B0000024184F26E0F86B260130180622FF21E1
:10B4C00008F091FA00281BD1F86B301840798009F8
:10B4D00002281CD001252046062148432330C0B253
:10B4E0006A46102108F0B4FC04AA1021022008F0DA
:10B4F000AFFCF86B04AB31186A462846FAF756FBE6
:10B50000641CE4B2387E8442D5D309B0F0BD002576
:10B51000E1E70000B447002070B5FAF753FB0024C0
:10B520000A4E0FE0F06B250128180622FF2108F0D3
:10B530005AFA002804D1F06B29180020FAF73AFBD8
:10B54000641CE4B2307E8442ECD370BDB44700206A
:10B5500070B514460D46064603F018FF00280DD0BE
:10B56000017B084808290AD0C06A002806D0436831
:10B57000002B03D0224629463046984770BD006B09
:10B58000F3E70000B4470020FFB581B01D46164622
:10B590000C46084603F0FAFE00280ED0007B124A43
:10B5A00008280CD0D06A002817D00768002F14D0C4
:10B5B0002B46324621460198B84705B0F0BD106BC6
:10B5C000002802D00768002FF2D12146506A06E019
:10B5D00001212046F9F7CAFAEFE72146106AF9F788
:10B5E0001BF90028F4D1E8E7B447002008B5FFF7BD
:10B5F00009FD012801D9022000E00A2069460870EF
:10B600006A4601210520FAF765FA08BD10B50C4A13
:10B610000A4B1268994206D1002A0DD01178814256
:10B6200007D0032010BD0548401C814204D1002AE8
:10B6300002D0FAF7E6FA10BD122010BDFEFF00009E
:10B640005846002030B587B0032817D0344A00256B
:10B6500090421BD1887800285CD032490B68002BBF
:10B6600058D0059502950395049500950195DA78D3
:10B6700019781B1D01F0FEF801200CE048890090AC
:10B680008C880B89CA88C878214612E0244A521C4B
:10B69000904203D1022000F0BDF83BE0204A921D09
:10B6A000904209D18878002834D000231A461946E0
:10B6B000009501F00FF92DE0194A0C32904229D083
:10B6C000194A904229D148790C46122822D1E3899F
:10B6D000A28961892089FAF727FB002804D0172066
:10B6E000F8F7AAFF002800D00120694608832179D5
:10B6F000608806AAFAF736FE6846008B002809D152
:10B70000E089019502950090A3896289218960886A
:10B71000FAF75CFA012007B030BD0020FBE700001B
:10B720000D20000058460020FFFF00000A4A10B517
:10B73000904202D18868007807E0074A521C904284
:10B7400008D188680078002802D001F09FF910BD68
:10B75000012010BD002010BD0B20000000290ED0DC
:10B7600000280CD0487980098001C02803D04028E7
:10B7700003D002207047012070470320704700204B
:10B780007047FFB5002008701F2A1BD2904219D2C3
:10B790001C5C401CC5B2002C14D06619964211D80E
:10B7A0005F5D384601F0BDF900280BD0641E0C70B7
:10B7B0000098874203D15819401C04B0F0BD761E92
:10B7C000F0B2E3E70020F8E710B5044C2068002849
:10B7D00003D008F085F90020206010BD54460020F9
:10B7E00070B5846B0546002C13D0206A002801D068
:10B7F00008F076F9606A002801D008F071F9A06AB3
:10B80000002801D008F06CF9204608F069F9002002
:10B81000A86370BD10B5044CA069002803D008F0DF
:10B820005FF90020A06110BD40460020F3B51E4E18
:10B830000546706881B0002824D0002418E07068A4
:10B84000270138188068002805D008F049F9716888
:10B8500000207918886070683818C068002805D002
:10B8600008F03EF9716800207918C860641CE4B2E1
:10B87000AC42E4D302980028706804D008F030F994
:10B8800000207060FEBD0028FCD02A01002108F0D5
:10B89000A1F90021FF22706803E00B01491CC2548A
:10B8A000C9B2A942F9D3FEBD84480020002805D1C1
:10B8B00004488078002801D00348704701481830B8
:10B8C00070470000546A00205C46002001488078E0
:10B8D00070470000546A00200148C06870470000AB
:10B8E000546A00200148006970470000546A002033
:10B8F0000148406900687047546A002010B5064A44
:10B9000050690168491C0160D078FF2803D00121EB
:10B91000890308F02DFA10BD546A002070B5064D59
:10B92000064CE888A04205D005490A780549FAF78F
:10B930000BFDEC8070BD0000546A0020FFFF00008A
:10B940007248002062460020FFB581B00B9F0A9E1E
:10B950000D9D039803F01AFD04007AD00198002889
:10B960002ED104984007207902D51221084303E024
:10B9700010210843FD210840207130460C993843BE
:10B9800008432843207924D0042108432071002D46
:10B9900007D02869A062204610222946183008F0F6
:10B9A0003FF80298002818D0002F09D0E06A00283C
:10B9B00001D008F095F81C21384608F03DF8E06207
:10B9C000A46B002C45D0002E1CD0206A00280ED07D
:10B9D00014E0FB2108402071F2E7002EF0D0E06A6D
:10B9E000002801D008F07CF81C213046E5E747210B
:10B9F0001C2008F031F82062002803D01C223146B8
:10BA000008F00EF80C9800280DD0606A002806D1C6
:10BA10004721162008F020F86062002803D0162283
:10BA20000C9907F0FDFF002D0DD0A06A002806D16B
:10BA30004721142008F010F8A062002803D0142237
:10BA4000294607F0EDFF3B46049A0399019806F05A
:10BA5000ADFA05B0F0BDF3B581B0019803F096FCE6
:10BA600005002AD00E2008F0BDF8040025D01820CB
:10BA7000F8F7E2FD0606360E00D12E78D0202070B1
:10BA8000002767700B20A0700622A91DE01C07F09C
:10BA9000C7FF0298C1070120002901D0207300E0F0
:10BAA0002773019961810299890701D5607300E0CC
:10BAB00067732146304608F009F9FEBDFEB5012640
:10BAC0001F4D032809D01F4A904227D188780C289F
:10BAD00021D011281FD03046FEBDC8781A4F0C4621
:10BAE0001A2803D1A088F988884214D0A08803F0CE
:10BAF0004DFC002801D0E188C18160890090238934
:10BB0000E288A188E07800F0E5FEA088F988884204
:10BB1000E1D1FD80DFE7FFF701FFDCE7A8420DD1AF
:10BB20000C46497900201229D6D1694688802179AE
:10BB3000608801AAFAF7FCFB0120FEBD0020FEBDD3
:10BB4000FFFF000013200000546A002070B58188B8
:10BB50001F4A914213D11F49806809680078002963
:10BB60000BD0002805D101204870FAF796F800287C
:10BB700001D000F0D5FE012070BD002070BD144A38
:10BB8000D21C91421AD8521E914201D1012400E0E8
:10BB900000248068104E05783078FF28EBD0042010
:10BBA00008F020F80100E6D0D02008704D70022087
:10BBB0008870CC70307808F089F8DCE7044A121DF0
:10BBC0009142DAD18068007800F0B6FF70BD0000C5
:10BBD00006200000544600206C46002070B5024646
:10BBE0001B481C4C01680026184D2078012A0BD0F8
:10BBF000002908D0E178490705D5022108F068FA44
:10BC00006E80FFF7E1FD70BD6A88002A03D0124BF9
:10BC10001B79002B05D00029F5D00878F8F7E2FC55
:10BC200070BD3C2A0FD2022108F052FA68880B49F5
:10BC300048430B49F6F7B6F802462078022108F08F
:10BC4000E9F96E8070BD3C3A6A8070BD6C46002098
:10BC50005446002072480020546A002040420F00E1
:10BC60007102000070B514460D4603F00CFD0C493E
:10BC7000042809D08868002810D04268002A0DD016
:10BC800021462846904770BD0969002906D00B68F7
:10BC9000002B03D021462846984770BD012070BD77
:10BCA00040460020F0B587B004005AD02E48A17954
:10BCB000C6782E4F002924D0F8680425002804D027
:10BCC0004168002901D0002088472146E0790831E9
:10BCD0000691FFF743FDE0718446237D628A218A45
:10BCE000E089029003A80EC0A08801950090E0783A
:10BCF00062463146069B00F0BDFDE078002806D084
:10BD000016E0B86908250028DFD00678DDE7628AEA
:10BD1000218AE0890290172303A80EC0069800909C
:10BD20000195E379A1880122304603F0CBFAE07057
:10BD3000B869002802D00420FFF76CFD787800284D
:10BD40000FD03978FEF79AFF00280AD0E078312822
:10BD500005D00095A2880346797806F08FF9002077
:10BD6000787007B0F0BD0000546A00204046002003
:10BD7000F8B50446FF26808803F008FB050009D0CB
:10BD80002E782F7BFFF72CFD284606F0E9F9A088D6
:10BD900003F05EFC114D6878002808D0864206D179
:10BDA0002978FEF76BFF00280AD1687008E0FF2EA3
:10BDB00006D00097A379A288A078314606F05EF9F4
:10BDC000A08803F060FC042807D10548A188C28838
:10BDD000914202D10021C943C180F8BD40460020F4
:10BDE000546A0020F0B587B004005BD02E48A179DA
:10BDF000C6782E4F002925D0F8680425002804D0E5
:10BE00004168002901D0002088472146E07914319B
:10BE10000691FFF7A3FCE071844620231B5DE28BB3
:10BE2000A18B608B029003A80EC0A08801950090A2
:10BE3000E07862463146069B00F01CFDE078002861
:10BE400006D016E0B86908250028DED00678DCE7C1
:10BE5000E28BA18B608B0290172303A80EC006987B
:10BE600000900195E379A1880122304603F02AFA77
:10BE7000E070B869002802D00420FFF7CBFC787886
:10BE800000280FD03978FEF7F9FE00280AD0E078B4
:10BE9000312805D00095A2880346797806F0EEF89F
:10BEA0000020787007B0F0BD546A002040460020A2
:10BEB00010B5094CA278002A0CD00146062207488A
:10BEC00007F0AEFDA0780549FEF7E5FE0348F9F757
:10BED000F3FE10BD002010BD546A00205C46002017
:10BEE00070B5164D0646E878FF2814D00A2007F0F2
:10BEF00079FE04000FD0D020207066700820A0705A
:10BF0000A878E07006220E49201D07F089FDE87828
:10BF1000214607F0DBFE287901280ED108481C389D
:10BF2000C068002803D08068002800D080470548FA
:10BF3000054A0078042108F05BF870BD546A0020BF
:10BF40005C460020724800200077010010B586B0E2
:10BF5000044603A91448F7F77DFE134804A9401CC2
:10BF6000F7F778FE6846E388018A8B4203D8228976
:10BF70008089824205D2A0882021F9F774FE06B09C
:10BF800010BD834200D2E0808A4200D92181A1897C
:10BF9000002001900091029063892289E188A088A5
:10BFA000F9F765FEEBE7000011030000F8B50700A4
:10BFB00041D0F87800283DD07D68002D3AD0162079
:10BFC000F8F73AFB40B20026009030E00F216956A6
:10BFD0000098814228DB1D488068002824D0142066
:10BFE00007F000FE04001FD0D020207000206070F9
:10BFF0001020A0702878E070E87BA0746878207129
:10C000000622A91C601D07F00BFD287AE072294664
:10C010002046062209310C3007F002FD0B4821466C
:10C020008068007807F052FE761CF6B21035F8787A
:10C03000B042CBD8F8BD054880680028FAD000206F
:10C0400000F08EFB002000F0B5FCF8BD8448002015
:10C05000F1B584B0049800287ED0C07800287CD048
:10C0600004984468002C78D01620F8F7E5FA40B21E
:10C07000002702901BE12046203008210190415604
:10C08000029881426ADB9349002589682846002985
:10C090007ED0217801290CD02346227A093303A9C6
:10C0A0000120FFF76EFB002800D0057821780429D5
:10C0B00014D088498968497803290FD0002D0DD004
:10C0C00000290BD0002863D0012902D002295FD1BA
:10C0D00001E0A80700E0E807002859D06078A11C1B
:10C0E000FFF73CFB009060707A480025406800280C
:10C0F00057D0002617E0496830010A5CFF2A10D0AB
:10C100004018427800998A420BD10622A11C801C5B
:10C1100007F078FC002804D06E48310140680D1803
:10C1200005E0761CF6B26B4908788642E3D3002D11
:10C1300037D02078042871D0A868002818D001785A
:10C14000227A914206D121460931401C07F05AFC5F
:10C15000012870D0207802E0B0E0ADE0A4E004282F
:10C160005ED0A868002803D007F0BAFC0020A860C1
:10C17000207A0421401C07F06FFC00280DD02178A4
:10C18000042955D0A860217A0170227A214600E066
:10C1900042E00931401C07F043FC207A00284FD1CF
:10C1A00052E02678042E4FD04A4A516800294BD0DD
:10C1B0000020137805E002018A5CFF2A24D0401C8D
:10C1C000C0B29842F7D3002D3ED02E7060786870D0
:10C1D0000622A11CA81C07F023FC207A0321401C86
:10C1E00007F03AFC00280BD0217804290FD0A86072
:10C1F000217A01702146227A0931401C07F010FC97
:10C20000207A00281CD104E000014518DBE7E86033
:10C21000EEE72078012813D016E0FFE7E8688CE706
:10C22000E8680028A4D007F05BFC0020E8609FE7E6
:10C23000E860A8E7FFE71520F8F7FEF9002803D12A
:10C2400024488068002803D12248406800282BD168
:10C25000207A143007F0C6FC050025D0D0202870C5
:10C2600000266E700D20A8702078E87001980622D4
:10C27000007AE87260782871A11C681D07F0D0FB75
:10C28000227A2A73207A002807D0284614302146C3
:10C290000931286107F0C4FB00E02E610D482946F2
:10C2A0008068007807F012FD7F1CFFB229340498E3
:10C2B000C078B84200D9DEE605B0F0BD0548806818
:10C2C0000028F9D0002000F04BFA002000F072FBAB
:10C2D000F2E700008448002070B50178744D912980
:10C2E00002D0A22973D04FE04178052908D0714CC3
:10C2F000714B0E2907D00F296AD03E2969D043E03F
:10C30000FFF736FD1CE082886C4900258A4219D16E
:10C3100081680E78491C002E06D1002904D065489A
:10C320000622183007F07CFB207801282CD1002E43
:10C3300002D02570304624E002202070F9F78BFCF3
:10C34000012070BD5E498A4220D18668002E1BD034
:10C350003078002806D1B178727808021043208125
:10C36000F0786070207802280ED13078002801D053
:10C37000257005E00320207061782089FAF76AF9BA
:10C38000307800F055FADBE7002070BD4C49C91C3D
:10C390008A4204D180680078FFF7A2FDD0E74949BE
:10C3A0005118042907D8D9680029C9D0096800297B
:10C3B000C6D0884770BD424909318A420AD15968BE
:10C3C0000029BDD00B68002BBAD0014634E067E0ED
:10C3D00016E034E03A490A318A4203D1816809788B
:10C3E0000029ADD0364C0C34A242CDD19968002939
:10C3F000A6D04A68002AA3D001462046904770BDC7
:10C40000014682882E480B30824203D02C481730D8
:10C41000824204D19868002892D043680AE02848F4
:10C4200011308242B0D1E088A842F3D018690028C8
:10C4300086D00368002B83D01046984770BD817862
:10C44000012914D00A2915D0022916D00B2919D098
:10C4500003291FD0062920D0072995D181880829D2
:10C4600092D2C0884900184A001F50528CE7FFF74B
:10C4700019FC65E7FFF7B6FC62E7596800298DD023
:10C48000496803E05968002988D08968002985D067
:10C49000884755E70246808806E0FFF757FD4FE7DB
:10C4A0004388024629461846FFF7DCFB70BD0000B2
:10C4B000FFFF0000546A00204046002009100000E1
:10C4C00002200000FADFFFFFC06B00200149486036
:10C4D0007047000040460020014988607047000016
:10C4E000404600200149C8607047000040460020D7
:10C4F000014908617047000040460020F8B5054634
:10C500008078624C00220626032721780300FDF77D
:10C5100045FE0805AF375A5A6E99A1AF68780028D2
:10C520006AD110225A495B4807F06CFA002807D0FC
:10C53000574910221031584807F064FA00280DD1ED
:10C54000544A1021022007F0C7FC534A102103204F
:10C5500007F0C2FC5148007807F05AFC0622E91C9B
:10C560004F4807F05DFA012020704F484D4B02788C
:10C570004E4801210078F8F74DFB00283CD179E0C6
:10C580006878002838D14948EA780078002A07D02E
:10C590004849474B0A780021F8F73CFB68700EE0E9
:10C5A00002290FD00121414F07F014FA002806D1CB
:10C5B0002078052803D00121387807F0D9FB687866
:10C5C000002819D1F8BD6A78002A15D1032805D0B2
:10C5D0000020394A0529107005D006E0042937D11A
:10C5E0000520207046E00420FBE7277042E06878D1
:10C5F000002803D0312821D026703BE00420207091
:10C600006A89E8780423291DF6F7D6FD2B4E307889
:10C6100000280DD02A49E8780A78904206D10622EF
:10C62000281D491C07F0EEF9012805D001203070C3
:10C630002149002008701DE00220F8E71E49002073
:10C640000870D2E72846F6F771FF20780528CCD18C
:10C650000220C6E768780028B4D11A4800688468C8
:10C66000002CAFD06B892A89E988A888A047F8BD3B
:10C67000002AFCD0134800680028F8D00268002A7D
:10C68000F5D0294620789047F8BD000010480020DA
:10C69000546B0020936B0020A36B0020C847002040
:10C6A000264800202C4800200A4800200848002086
:10C6B000746B00200C4800200B480020CF4700205E
:10C6C000F44700200448002010B50178912906D0D5
:10C6D000A22903D0D02901D1FFF710FF10BD417866
:10C6E0000E29FBD181880A4A9142F7D18068032143
:10C6F000827841564378100218437F29EED0054ACC
:10C700001268002AEAD05268002AE7D0904710BD8C
:10C710000514000004480020F8B507460E460846F8
:10C7200002F034FE020019D01820F7F785FF050645
:10C730002D0E00D11578062007F054FA04000DD014
:10C740000622002107F046FAD020207067700E20E4
:10C75000A070A6802146284607F0B8FAF8BD000070
:10C76000F8B5054631480024806800285CD0002DCB
:10C7700010D12E494A68002A0CD00020097807E021
:10C780000301D35CFF2B01D0641CE4B2401CC0B297
:10C790008842F5D3E000083007F024FA060007D1FC
:10C7A000082007F01FFA002413250646002831D080
:10C7B000D020307001207570B070F470002C21D042
:10C7C000354608350027756015E051683801095C69
:10C7D000FF290ED029705168641E4118497869708C
:10C7E0005168E4B241180622A81C891C07F018F908
:10C7F00008357F1CFFB20D4A1078874204D2002C06
:10C80000E3D101E00020706008483146806800787C
:10C8100007F05CFA054C00212078FFF707F8A068C4
:10C8200007F05EF90020A060F8BD000084480020F9
:10C8300070B50F4D0646E878FF2817D00E2007F098
:10C84000D1F9040012D0D020207066700020A070B2
:10C85000294606221831E01C07F0E2F82889608199
:10C8600068782073E878214607F030FA70BD000040
:10C87000546A0020FFB5074681B01D4616461620B3
:10C8800007F0B0F9040022D0D02020700520677096
:10C89000A070E670002D05D006222946201D07F065
:10C8A000BFF804E006220021201D07F093F90A9842
:10C8B00060810B9820730C98E0810D9820820E986F
:10C8C00060820F9820752146029807F0FFF905B0A5
:10C8D000F0BD0000FFB581B01E4617460D460C2086
:10C8E00007F080F9040016D0284602F04FFD00281A
:10C8F00001D0007801E00948C078D0212170019969
:10C9000061700721A170A580E78026810A99618165
:10C91000214607F0DBF905B0F0BD0000546A0020A5
:10C9200070B50C4D04462868002811D0032007F08C
:10C9300059F9010008D0D02008704C70032088708D
:10C940002868007807F0C2F9002C01D0FEF73CFF00
:10C9500070BD000054460020FFB581B01F460E4652
:10C96000084602F013FD050022D0102007F03AF926
:10C9700004001DD01022002107F02CF91820F7F731
:10C980005BFE0006000E00D12878D02121700199AD
:10C9900061700F21A170A6800399217267720A99B4
:10C9A000A1720B99E1720C99E160214607F08EF9B2
:10C9B00005B0F0BD10B504461520F7F73DFE002880
:10C9C00001D0012100E000212046F9F77DF910BDDA
:10C9D000FFB5074681B01D460E460E2007F002F94E
:10C9E000040010D0D0202070002060700C20A070B7
:10C9F000A6800622A01D039907F012F82573F8B24D
:10CA0000214607F063F905B0F0BD0000F0B51C4FFA
:10CA100085B03868002831D00320F7F70DFE0646B0
:10CA20000420F7F709FE054604A91648F6F756FB59
:10CA30006846017C14480029807806D0032802D07B
:10CA4000002806D003E0022404E0002801D00124DD
:10CA500000E000243968C878091DFEF71CF93A681F
:10CA6000D77A937A0090111D01A88AC09278234644
:10CA700029463046F9F715F905B0F0BD0120FBE76E
:10CA8000544600201F040000546A002070B504467C
:10CA90000E488068002817D00D4D002C0CD10220C4
:10CAA000F7F7CAFD02462878012107F0B3FA012002
:10CAB000FFF780FF040006D02878012107F008FB6B
:10CAC0002046FFF74DFE012070BD00008448002085
:10CAD0007248002070B50C4602F058FC05001FD0CB
:10CAE0001820AC62F7F7A8FD0606360E00D12E78A6
:10CAF000102007F077F8040012D0D020207000201A
:10CB000060700920A0706879E0700622A91D201DC0
:10CB100006F086FFA86AE0602146304607F0D6F8A6
:10CB200070BD002803D0172803D3FF2801D00020B0
:10CB30007047012070470000F1B52D4E82B030687B
:10CB4000002842D040782B4D012814D028790028A5
:10CB50003AD1032007F046F8010009D0D020087030
:10CB600002984870042088703068007807F0AEF8AA
:10CB7000FEF72AFE28E02048204F4368002B19D0FA
:10CB80001A78694601205B1CFEF7FBFD002811D0D6
:10CB90000078C0070ED00120F7F74EFD04463C2870
:10CBA00014D33878164A022107F022FA12483C3C86
:10CBB000448016E00020F7F73FFD0CE000202871CC
:10CBC00002E00298FFF7ACFE0120FEBD0D480E49C1
:10CBD0006043F5F7E7F8020003D03878022107F048
:10CBE00019FA31680220487028790028E9D0E5E771
:10CBF00054460020546A00206C46002072480020F1
:10CC00000077010040420F0071020000074A002136
:10CC100006234B43D35A834203D10620414388184D
:10CC20007047491C0329F3DB00207047E46A0020A9
:10CC300001460648406906E0826852898A4201D16D
:10CC4000001D704700680028F6D170473C4700205F
:10CC500000B50F292ED00BDC0B00FDF79FFA0F2338
:10CC6000232323232B252B232B232B232B27230089
:10CC7000182917D008DC10390B00FDF78FFA0813BC
:10CC80001B1B1313131919131E290BD006DC1929AA
:10CC900008D01B290ED01D2904D10BE0522909D040
:10CCA000D22907D0002000BDC06800BD006800BDCB
:10CCB000806800BD406800BD10B50C46FFF7A6FFB8
:10CCC00000280DD0002C00D020608078FE2803D0F2
:10CCD000FF2803D0162010BD172010BD002010BD66
:10CCE000022010BDFFB581B001980A9D1E4617466F
:10CCF000FF2813D0202006F075FF04001DD0B020BF
:10CD000020706770029860802671002D09D020463F
:10CD100018222946083006F083FE08E0022005B0FC
:10CD2000F0BD204618220021083006F053FF2146AE
:10CD3000019806F0CBFF0020F1E71320EFE7002079
:10CD400070470020704738B54C88088884420ED35D
:10CD500000280CD0002200920B794A1D2146F8F7DA
:10CD6000B1FA002801D0002038BD0A2038BD0120CA
:10CD700038BD0000F3B585B00698002607884088C6
:10CD8000B8421ED3002F1CD0002069468880029034
:10CD900000206946888100900698002341881A4641
:10CDA0003846F8F78FFA040057D068468088002884
:10CDB00033D0684680790128207812D0102850D1CD
:10CDC00002E0012007B0F0BDA07A2870608910222F
:10CDD000000A6870AD1C2846616806F021FE103517
:10CDE0000DE002283DD1A07A287060890222000A55
:10CDF0006870AD1C2846616806F012FEAD1C6946DD
:10CE00008888401C80B28880B04226D261891F4841
:10CE1000814222D07F1CBFB2BAE72220009003AB30
:10CE20001A4A05210598F8F75DFD05000CD002951A
:10CE3000207802280AD002206A4690711221908937
:10CE4000F4F79AFFC6B2BFE71120BBE7012069469D
:10CE5000887188898005060EC5E7684680880028A5
:10CE600012D001A90598F5F7A7FC00280AD001AB5C
:10CE7000052216210598F8F747FB002802D00298F2
:10CE800006F02EFE00209DE70A209BE7FFFF000032
:10CE900038B505460C4608886946F8F7EFF90028CA
:10CEA00007D0017A6846028823462846F8F794FCA2
:10CEB00038BD012038BD000038B50C4649882088AF
:10CEC000814219D3002817D02379621D02210B4813
:10CED000F5F7FAFB00280DD0002000902379618837
:10CEE0002088621DF8F7EEF9002801D0002038BD37
:10CEF0000A2038BD102038BD012038BD3443010060
:10CF000038B54C88088884420ED300280CD0002203
:10CF100000920B794A1D2146F8F7D4F9002801D078
:10CF2000002038BD0A2038BD012038BDF8B50D46B7
:10CF30000646002428E028686100401841780278FD
:10CF4000080210436946F8F799F9002810D0017AD1
:10CF5000684602883046F8F768FC002812D02A6834
:10CF60006100535C13702A68491C515C5170F8BD14
:10CF7000296860000A5C0A702968401C085C4870D7
:10CF80000120F8BD641CA4B2A888A042D3D8002018
:10CF9000F8BD38B5044608886946F8F76FF90028E7
:10CFA00006D0017A684602882046F8F73EFC38BD74
:10CFB000012038BD38B505460C4608886946F8F7A3
:10CFC0005DF9002807D0017A684602882346284682
:10CFD000F8F756FC38BD012038BD000001498860D3
:10CFE000704700003047002010B50446801C00F058
:10CFF0000BFFFF20E07010BD1CB5044668460171B0
:10D000004271204602F0C2F900280BD0027B01A930
:10D010000748082A009106D07E2300222146007886
:10D02000FFF760FE1CBD7E23002221464078F7E713
:10D0300030470020F8B50024064627460C20604300
:10D040008519A8882D1D00280ED0A868002801D0B9
:10D0500006F046FD0C220021284606F0BBFD641CAC
:10D06000E4B22F80052CE9D30020C0433080F8BD06
:10D0700000B500F023F8002800D0806800BD002231
:10D080009300CB5A834202D1900040187047521C43
:10D09000032AF5DB00207047074A002192698B01C3
:10D0A000D35A834202D1880180187047491CC9B203
:10D0B0000329F4D3002070473C4700200649096942
:10D0C000002906D08A88824201D1886870470968A1
:10D0D000F6E70020704700003C4700207CB506467C
:10D0E000012906D0022922D1012102F0D3FA002819
:10D0F0001DD13046FFF7D0FF002801D0FFF79AFF7F
:10D1000001A80C4D00900223094A29460120F8F796
:10D11000D9F80AE03046E168F7F70CFE68468288E5
:10D12000002329462046F8F707F90400F2D17CBD18
:10D1300040430100FFFF0000F3B5002083B002462A
:10D14000054604460C21049B6143C9188B88091DC0
:10D15000002B0ED0002A1BD093421ED14B88834255
:10D160001BD189884B199DB20818641C80B2052C0C
:10D17000E8DB022C39DB00200190002D0DD0472187
:10D18000284606F069FC0090002807D0002625E01C
:10D190008D8848881A464019E7E7002005B0F0BDA1
:10D1A0000C20049970434718F9683F1D00290DD0E1
:10D1B000019B0098BA88C01806F032FCB988019823
:10D1C000081880B20190B86806F08AFC002E04D0DE
:10D1D0000C220021384606F0FDFC761CA642DFDB5F
:10D1E00004990098C860049805810120D6E7F3B53A
:10D1F000074683B000254088FFF74EFF02900028C5
:10D2000003D0387A012807D047E07888F5F7B4FAD8
:10D21000002856D105B0F0BD384608300299FFF716
:10D220008BFF002817D0029C1821E0880191009004
:10D230002389A188E2687888241DF7F7B7FF05469F
:10D24000162805D0002D28D004982188018024E0DC
:10D250000020A06021E000260C20029970434018B5
:10D260008188041D002918D0042E1ED0008A0028B1
:10D270001BD01620628800920190A3887888A2684B
:10D28000F7F794FF0546162811D0002D02D0049818
:10D2900021880180761C052EDEDB0298FFF7CAFE8E
:10D2A000002D09D0162D05D00DE01820E2E7002052
:10D2B000A060EFE7002506E07888F5F75DFA002822
:10D2C00001D01620A6E72846A4E70000F3B50446DF
:10D2D000074689B008344088F5F78CFA079004A80F
:10D2E00000900025237961882088621DF7F7EAFF06
:10D2F000059000286FD00798401F08900898854235
:10D3000069DA397907983D4BC01F80B2002203913A
:10D310000093019202901E466946083E0A8A788868
:10D32000F3680599F7F7B6FD002821D120893289E5
:10D3300090421DD1E068F16806F064FB002817D028
:10D340002F4E706800280AD11120009078880023A1
:10D350002C4A0721F8F7C6FA002803D07060059818
:10D36000468906E00A982188018011200BB0F0BDA3
:10D3700000266846028A618806AB0598F7F7DCFF4D
:10D380000590002E1AD01E49320A486846556D1C79
:10D390004B68A8B21A54401C059A80B2002A10D0DB
:10D3A0006A464B68128B1A546A46128B401C4968B5
:10D3B00080B2120A0A54401C85B29FE700289DD112
:10D3C00009E00F4AFF2153681954401C526880B28B
:10D3D0001154401C85B2002D0AD00948A9080180CB
:10D3E00078880749F5F7D0F90028BFD01620BDE7A7
:10D3F0000A98218801800A20B8E7000044470020ED
:10D40000CC6A0020FFFF0000F0B589B00446002779
:10D4100069468F820120884D0874E868002807D18A
:10D42000F8F7C0FF472106F017FBE86000281ED080
:10D4300018220021814806F0CDFB20797F4E411C47
:10D44000C9B20691022816D0062835D0082838D04F
:10D450000A283BD00C2867D00E287DD010287CD01D
:10D4600012287BD016287AD0182879D0D5E06846C3
:10D47000007C09B0F0BD6088082803D270494000E4
:10D48000085A00E01720308060886C49F5F764F98D
:10D4900000282189308805D0814200D3208120894D
:10D4A0003080BEE0814200D3208121896088F8F776
:10D4B0006DF9B2E00699ADE005A92046FFF706FF39
:10D4C0008BE005A9204600F0F9F986E0208907A93C
:10D4D000F7F7D4FE05005ED015200090608808ABF9
:10D4E000584A0B21F8F7FEF97060031E47D06946D1
:10D4F0002079098C029101970096039069468A8BE6
:10D5000060882946F7F7C6FC050034D160884B498E
:10D51000F5F71CFB3CE0706806F0E2FA002D7CD0C9
:10D520002089694688825AE0208907A9F7F7A6FE74
:10D53000050030D016200090608808AB414A0D21CC
:10D54000F8F7D0F97060031E19D069460A8C20796B
:10D5500061890096029204E022E026E02AE02FE0B2
:10D5600037E00191039069468A8B60882946F7F776
:10D5700091FC050008D0162DCDD10025CBE72089E0
:10D580006946888211252CE060882C49F5F784FAD9
:10D59000002846D141E0208969460125888220E0A3
:10D5A00005A9204600F02AFA17E005A9204600F058
:10D5B000BBF812E004AA05A9204600F0A7FA0CE087
:10D5C00005A9204600F040F8050008D16846077418
:10D5D00023E005A92046FFF70AFE05001DD0162D01
:10D5E0001FD06078142818D0207930706846808A5F
:10D5F0007080357160881149F5F7A2F800280CD0C9
:10D60000012560880D4B2A461621F7F77DFF00287B
:10D6100003D029460948F8F7ABF92046F7F718FE7A
:10D6200025E76088054B1621069AF7F76DFF00285D
:10D6300000D03FE7F1E700003C470020CC6A002023
:10D64000C06B0020FFFF0000F0B5044685B00E4619
:10D65000054608340027008904A9F7F70FFE0300E8
:10D660005BD0187A800613D56846008AFFF700FD64
:10D67000070008D0688812221946B847070007D06B
:10D680002088308047E0208830800E2005B0F0BD33
:10D690006888FFF701FD010006D12248FFF7FCFC76
:10D6A00001000DD06888088000200C2242435218E7
:10D6B0009288002A08D0401C0528F6DB09202DE0BE
:10D6C000208830800920E1E70C2250434018214691
:10D6D000001D06F0A5F90C22214601A806F0A0F9CC
:10D6E00010200090A288688800231721F8F7FAF824
:10D6F000039000280BD0A288A16806F091F96888F1
:10D7000001A9F5F7B5F9002805D01620BEE7208855
:10D7100030801120BAE73846B8E7012021883180EF
:10D72000B4E70000FFFF0000F3B5024689B00832FD
:10D73000064604924088F5F75DF8079005A8049A1C
:10D740000090137951881088521DF7F7BBFD002512
:10D7500004462F46002C20D06A46217A7088928A8F
:10D76000F8F763F8070015D131790798504B801FFF
:10D770000890039180B20022009301920290194612
:10D780000839CB6869468A8A70882146F7F782FB98
:10D79000070005D00A9861890180002D70D079E0DA
:10D7A000002D0DD043484188414808380089021DAA
:10D7B00091426FD140190899001D88426ADC10E03F
:10D7C00012200090708800233B4A1121F8F78AF854
:10D7D00038490028486036D0354808380089001D8F
:10D7E00048803449A07A4A6806AB505562896D1C5E
:10D7F0004968A8B2120A0A54401C85B204984188AC
:10D800006846828A2046F7F797FD040021D06A46D1
:10D810002849108B4A6850556A46128B6D1C4B681C
:10D82000A8B2120A1A54401C85B24868204940190F
:10D8300008390A89C96806F0F3F81D4808380089D4
:10D84000281885B286E70A986189018011200BB0FB
:10D85000F0BD1849FF22486842556D1CA8B24B68BC
:10D86000134D1A54401C84B24868083D00192A8997
:10D87000E96806F0D5F82889201885B28DE7FFE71A
:10D880000498002F01880A98018000D10A273846A1
:10D89000DDE7FFE7074C28466188F4F76DFA208042
:10D8A00070882146F5F70CF90028D0D01620CEE775
:10D8B00044470020CC6A0020FFFF0000F3B5054676
:10D8C00087B0083005902F896888F4F793FF00240B
:10D8D000001F019404900498A0426FDB06A80090FA
:10D8E000059803794188421D3846F7F7EBFC06009E
:10D8F00064D06A467789317A6888128BF7F795FF8A
:10D90000019000285AD128790499394B89B20291A3
:10D91000002200930192039019460839CB686946AA
:10D920000A8B68883146F7F7B5FA0190002845D18F
:10D93000002C08D02F4841882D4808380089801CC9
:10D9400081423DD110E013200090688800232A4ACC
:10D950000921F7F7C7FF27490028486028D0244845
:10D9600008380089801C488021480838008901193E
:10D970000498814222DC1F49B07A4A6810557289A6
:10D98000641C4B68A0B2120A1A54401C184E84B290
:10D990004868083E00193289F16806F041F830897C
:10D9A000201884B21448874295D07F1CBFB292E7FA
:10D9B00008980780112009B0F0BDFFE7002C0DD0BA
:10D9C0000C4E20467188F4F7D7F9308068883146CC
:10D9D000F5F78EF80028EED01620ECE70198002825
:10D9E00001D10A200190089807800198E3E7000020
:10D9F00044470020CC6A0020FFFF0000F3B5044636
:10DA000087B0083005906088F4F7F4FE06460025DC
:10DA100060E00598690000684018417802780802C3
:10DA2000104306A90490F7F729FC01001DD02079C6
:10DA3000BAB2334F029200230097019303903A4603
:10DA4000083AD3686A466088128BF7F723FA070012
:10DA500016D00898049901802A484068002801D00F
:10DA600006F03EF8384609B0F0BD089904980880E1
:10DA700024484068002801D006F032F80120F2E77F
:10DA8000204F786800280AD1142000906088002375
:10DA90001D4A0F21F7F726FF786000282BD0184980
:10DAA000388808390A89521C8218B24202D9321ABF
:10DAB000521E0A81134A0F46526810180A89C96813
:10DAC00005F0AEFF0F483989008840180D496D1CDC
:10DAD0000880ADB205988088A84204D90948771E0D
:10DAE0000088B84295DB60880649F5F719F80028E8
:10DAF000B9D01620B7E70899049808801120B2E73A
:10DB000044470020CC6A0020FFFF0000F7B5044620
:10DB100084B0054617460834008902A9F7F7AEFB22
:10DB2000030032D0187A80060ED568460089FFF7C8
:10DB30009FFA060006D0688812221946B0470028CE
:10DB400002D023E00E2021E0607A002801D052208C
:10DB500000E0287900260096019063882188688873
:10DB60006268F7F723FB002802D016280BD00DE0DF
:10DB7000607A002810D16888F5F71AF8002800D0DC
:10DB8000162007B0F0BD3E7006E0012005992288FE
:10DB90000A80617A0029F4D00020F2E7FEB54C68D3
:10DBA000089D6678277834020E783C43022E02D115
:10DBB000054EB44201D00120FEBD0224009501941F
:10DBC000F7F71EF9FEBD000002290000F8B5054672
:10DBD0001D48854224D0461C002922D001292CD082
:10DBE00002291DD10121284601F054FD002817D13A
:10DBF0002846FFF70BF8040012D0A0780026FF2873
:10DC00000DD0FE2806D00096E0781E231422294667
:10DC1000FFF768F82046FFF7E7F9FF20A0702671AC
:10DC2000F8BD2846FEF7F2FF0028F9D13046FEF78E
:10DC3000EDFF0028F4D00580F8BD2846FEF7E6FF8A
:10DC40000400F9D02680D8E7FEFF000038B50400B4
:10DC500010D0A078FF280DD0FE280BD00020009017
:10DC60002188E0781E231722FFF73CF8FE20A070E1
:10DC7000FF20E07038BD10B50C46FEF7C7FF002846
:10DC800006D00279511CA14202D1D109C90101710A
:10DC900010BD0000F7B5887800258AB00C461E2814
:10DCA00002D0122819D115E00A98FEF7AFFF05003F
:10DCB00025D0A878FE2822D0FF2820D00020009070
:10DCC000A378E87800220A99FFF70CF82846FFF7B6
:10DCD0008BF914E06078012814D00A98FEF796FFBB
:10DCE00005000FD02A79002A0CD0100607D4A1789D
:10DCF0000A98FFF781F928798021084328710020CC
:10DD00000DB0F0BDA1784808C20034481018803822
:10DD1000876FC66F32484078FF280DD019290BD283
:10DD2000002F09D0002E07D02078002802D1627879
:10DD3000002A03D0122901D006274CE003A9009144
:10DD4000A3886178A268B847070044D103A90A985C
:10DD5000B047070020D0607800283CD1A078694601
:10DD600008710F72A0780E280FD08889C88001A989
:10DD70000A98F4F7E5FC07002DD001AB012216212B
:10DD80000A98F7F7C1FB074625E003984178027827
:10DD9000080210436946E9E7A378042B1BD003A8C7
:10DDA00000900F48002240780A99FEF79BFF070079
:10DDB00011D1A17803A8FEF74BFF002802D00C99DF
:10DDC00000200870A078122802D16178012902D0C1
:10DDD000002D00D02871384692E70000D0420100A3
:10DDE0003C47002000B50346F7F7C9FC002802D0E5
:10DDF0001818401E83B2184600BD10B51924A4019E
:10DE0000624306F0BFF810BD10B5040008D02078BA
:10DE1000FF2805D0FE2803D006F036F9FF20207039
:10DE200010BD0000F7B50F4604465321102005F041
:10DE300013FE06465321102005F00EFE0546002E67
:10DE400034D0002D2DD01022002105F0C3FE324623
:10DE500029462046F9F730F9040023D1307800062E
:10DE600009D52946304601F01FFA3A46134928469B
:10DE700006F07CF903E03946304601F015FA3878AF
:10DE8000000609D52946384601F00EFA0B49284606
:10DE9000029A06F06BF905E03846029901F004FA9F
:10DEA00000E01324304605F01BFE00E01324002D93
:10DEB00002D0284605F014FE2046FEBD8543010031
:10DEC000F8B5069800261D4614460F46002801D0D6
:10DED0000B20F8BD38780021022801D0198016E007
:10DEE00078684278037810021843294BC21A984286
:10DEF00025D007DC274A801A0BD0012817D002282A
:10DF000004D13DE0012A1FD0A32A39D0298001265F
:10DF10003BE0F86806F0EFF882B20798824200D939
:10DF200002462A80F968204605F07AFD2DE0F8685F
:10DF30000221008829802070000A607025E00620F8
:10DF400028800246F968EEE7F868002816D0082114
:10DF50002980017821700188090A61708178A17097
:10DF60004188090AE170017921718188090A61718A
:10DF70008179A171C088000AE07106E0298004E07F
:10DF800001202880F868007820703046F8BD000035
:10DF9000032A0000002A000010B50B78840702D580
:10DFA0000224234301E0FD2423400B7003060B7879
:10DFB00002D58024234301E05B065B0E0B70030750
:10DFC0000B7802D50824234301E0F72423400B708B
:10DFD00083060B7802D52024234301E0DF2423406D
:10DFE0000B708221084203D1010701D4810603D5B9
:10DFF00010780C21084304E0002803D11078F321A5
:10E000000840107010BD0000FFB581B008780024F2
:10E010000A9E1F460D46022813D16868417802788F
:10E0200008021043394A811A90425ED005DC384913
:10E03000401A0AD0012804D12DE0012943D0A42997
:10E0400062D00124204605B0F0BDE86806F053F820
:10E0500080B2864205D8F0190090152803D90D2406
:10E06000F0E70724EEE7E8683A468019039905F0DF
:10E07000D7FC0098162180B20A1AE9680818002116
:10E0800005F0A8FD234880680028DBD00268002A3C
:10E09000D8D0002112E0002E13D1022BDFD103983B
:10E0A000E9684278037810021843088019488068AC
:10E0B0000028C7D00268002AC4D0012101989047E7
:10E0C000C0E70B24BEE7002EFBD1062BC7D10622EA
:10E0D000E868039905F0A4FC0E4880680028B1D0D8
:10E0E0000268002AAED00321E8E7002EE9D1012B17
:10E0F000B5D103980078002803D0012801D08024EE
:10E10000A0E7E96808709DE703249BE7022A000066
:10E11000002A000080460020FFB581B00498164612
:10E1200000280CD00121019801F0B4FA002809D090
:10E13000214F00253878002E06D0F87805E0012020
:10E1400005B0F0BD1420FBE7FD7885421AD2FA68CD
:10E1500029018C186188002902D06D1CEDB2F4E70A
:10E16000002C0FD0002E0FD04C21202005F074FC85
:10E17000E060002806D02022002105F02BFD40356C
:10E18000658003E01520DBE70020E06000202070C0
:10E190000198E080002E08D0707A2072388AE168F9
:10E1A000301A00110009087701E0029820720498E3
:10E1B00004600020C4E70000984800200A7802703C
:10E1C0000A88120A42700B880222012B02D0022B0D
:10E1D00007D011E08A7882704988090AC170042248
:10E1E0000AE08A7882704A88120AC2700A7902713B
:10E1F0008988090A41710622104670470A78027020
:10E200000A88120A42708A7882704A88120AC2709A
:10E210000A7902718A88120A42718A798271CA88DF
:10E22000120AC2710A7A02720989090A41720A2025
:10E2300070470A7802700A88120A42708A788270DF
:10E240004988090AC170042070470A7802700A8858
:10E25000120A42708A7882704988090AC1700420C3
:10E2600070470A7802700A88120A42708A788270AF
:10E270004A88120AC2700A7902718A88120A4271A7
:10E280008A798271C988090AC171082070470A78A1
:10E2900002700988090A417002207047F8B50D46DE
:10E2A0000646002417E0F96820014718387800284E
:10E2B0000FD0F888B0420CD1072D02D17888F8F73A
:10E2C0005DF82A460021384600F0EDF9384600F0A6
:10E2D000FFF8641CE4B2164FF8788442E3D3002DB3
:10E2E00018D0F8BDF96820014518287800280FD00B
:10E2F000687AFF280CD0E888B04209D1284600F09F
:10E30000B7FF1421284600F04EFA284600F0E0F846
:10E31000641CE4B238788442E4D304242046641CAC
:10E32000E4B2FF22314600F0EDF8082CF6D3F8BD38
:10E330009848002070B504460D464088F8F71EF84E
:10E340002A460021204600F0AEF9204600F0C0F831
:10E3500070BD0000F3B5088981B00D46002803D0D8
:10E3600025490988884201D91B20FEBD042168681F
:10E3700005F004FB297A0446017028891F4E010A22
:10E3800061702978A17028880227010AE170288924
:10E39000001D85B20198B04211D10C2005F022FC7D
:10E3A00001000AD0902008704E800F71CD80144873
:10E3B0008C60007805F08AFC16E01320FEBD234631
:10E3C0002A460021F7F7ACFC0E49002807D00228A6
:10E3D0000CD007280CD012280CD01F28EED10878BA
:10E3E000002801D0401E08700020FEBD1420FEBD94
:10E3F0000420FEBD0220FEBDA0480020FEFF00005C
:10E400009F4800209948002030B5094C054600215E
:10E41000237809E0E268080180184288002A01D0C8
:10E42000AA4204D0491CC9B29942F3D3002030BD9E
:10E430009848002030B50A4A0446002113780AE0C3
:10E44000D568080140194588002D02D00579A542FC
:10E4500004D0491CC9B29942F2D3002030BD00005B
:10E460009848002030B50A4B00219C780BE01D69CC
:10E470000A01AA5A002A04D0824202D10801401996
:10E4800030BD491CC9B2A142F1D3002030BD00000B
:10E490009848002070B50D4D06460022EC7810E03B
:10E4A000EB681001C0184388002B08D0C388B34222
:10E4B00005D1C368002B02D05B888B4204D0521C6C
:10E4C000D2B2A242ECD3002070BD000098480020D8
:10E4D00070B5C4680546002C0CD0E068002801D057
:10E4E00005F0FEFA6069002801D005F0F9FA20462F
:10E4F00005F0F6FA10220021284605F06BFBFF20FC
:10E50000687270BD0C23584310B5094BC418303CD9
:10E51000608988420BD16068002808D0FF2A02D0A9
:10E520000178914203D105F0DBFA0020606010BD54
:10E53000D06B0020F3B5C46889B00026054602AF51
:10E54000002C20D0E068002802D005F0C9FAE6606F
:10E55000208869464881608888812089C881608ACE
:10E560004882208A08826888088100960197E98895
:10E57000287A64230A9A00F03DF90A986077668247
:10E5800026820BB0F0BD0C220021384605F022FB9C
:10E5900068886946088100960197E988287A64238B
:10E5A0000A9A00F027F9ECE770B50C4605461222EE
:10E5B0000021204605F00EFB002D1DD0287F010113
:10E5C0000E480269515A2180297F02690901891880
:10E5D000498861800189A1802988E1806988218139
:10E5E000A9886181E988A1812989E181297F006960
:10E5F00009010818C088208270BD000098480020DA
:10E6000010B50446084884420DD0012907D00229DC
:10E6100009D10121204601F03DF8002803D1002155
:10E620002046FFF73BFE10BDFEFF000010B507219E
:10E63000FFF734FE10BD10B5040009D06088002833
:10E6400006D01721204600F0AEF82046FFF740FF25
:10E6500010BDF0B5002689B015460446002907D044
:10E6600000960196E5880A46007A6023294616E05E
:10E670001622002102A805F0ADFA6846058102AF16
:10E68000002D06D1608869464881391DE068FFF792
:10E690008BFF019700963246E188207A602300F0D4
:10E6A000A9F809B0F0BD10B588B0002901D0002349
:10E6B0000AE06B469A8142881A81C368002B02D017
:10E6C0005A886B465A8102AB002201930092C4889B
:10E6D0000A46007A6023214600F08CF808B010BD8D
:10E6E0007FB5C2680D460446002A21D0508869468D
:10E6F0004881622D06D01849107F09680001401832
:10E70000C08812E01548D1880088814200D20846AE
:10E71000C1B2107C528A801AC0B2002A01D1801C7A
:10E72000C0B24018401EF3F73DFB6946888104E003
:10E730000622002102A805F04DFA6088694608818A
:10E7400002A9002001910090E188207A2B46002246
:10E7500000F050F87FBD0000A8480020A04800202D
:10E76000F8B5074615460E46102005F03BFA0400A2
:10E7700017D0A0202070002066806070002D05D08A
:10E780000C222946201D05F04BF904E00C22002143
:10E79000201D05F01FFA2146384605F097FA0020A3
:10E7A000F8BD0120F8BD7CB50446007804280AD0E5
:10E7B000022815D0062813D0032803D100222046B2
:10E7C000FFF771FF7CBD002000900190E5880A46AC
:10E7D000207A1323294600F00DF8E188122205E083
:10E7E00000222046FFF735FFE18814220520FFF7BD
:10E7F00089FE7CBDFFB581B01E46174620200B9DCB
:10E8000005F0F0F904001AD0A22020706770029879
:10E8100060800A9820716671002D06D0204618226B
:10E820002946083005F0FCF805E0204618220021B2
:10E83000083005F0CFF92146019805F047FA05B0F8
:10E84000F0BD0000F0B507460D4C002001462578CC
:10E8500012E0E3680A019E5C002E0BD0D218D26849
:10E86000002A07D0127F23691201D218BA4201D1BF
:10E87000401CC0B2491CC9B2A942EAD3F0BD000095
:10E8800098480020022A01D2012070474A780B786C
:10E8900012021A430280012A02D0022A06D00FE097
:10E8A000CA788B7811021943418009E0CA788B78C5
:10E8B00012021A4342804A790B791102194381806E
:10E8C000002070470A2A01D0012070474A780B784F
:10E8D00012021A430280CA788B7812021A434280CD
:10E8E0004A790B7912021A438280CA798B79120213
:10E8F0001A43C2804A7A0B7A11021943018100201F
:10E900007047042A01D0012070474A780B78120220
:10E910001A430280CA788B78110219434180002083
:10E920007047042A01D0012070474A780B78120200
:10E930001A430280CA788B78110219434180002063
:10E940007047F8B506460020706008790D46022829
:10E9500025D1E988042922D3A868427803781702D0
:10E96000C278807814021F430443381D814216D1B7
:10E97000042C0AD0052C08D0062C06D0072C04D075
:10E980002046FFF741FD002809D03781348003215C
:10E99000C943A86804F0F2FF70600020F8BD0120B0
:10E9A000F8BD022A01D0012070474A780B78110285
:10E9B00019430180002070470A7802704A7842703B
:10E9C000CA788B781102194341807047FEB506461C
:10E9D0001446508800220D467F2808D90220694637
:10E9E00008804A8060888880E9B26A460BE0A18886
:10E9F000172904D3E088172801D3814207D268463B
:10EA00000280E9B26A463046F7F792FCFEBD0292F8
:10EA10002088FFF727FD07002FD0FFF713FF397A73
:10EA2000884207D202AB3A46FF213046FFF774FB1B
:10EA3000002801D0042221E002982189C0680180C9
:10EA400061884180A1888180E188C180B988018185
:10EA5000FB68002B0FD0E9B22246304698470A499E
:10EA6000024688420AD102980621017005711E21D2
:10EA700000F0E8FBFEBD002200E0022229463046FD
:10EA8000029B00F059FAFEBDFFFF0000F7B50878C1
:10EA900002278AB013460C4606280AD0122832D024
:10EAA000142846D00026162850D068460684497897
:10EAB00078E0A278194602A8FFF723FF050069D184
:10EAC00068460089FFF7A0FC060010D03848009087
:10EAD000627802AB07210A9800F0FAF902220021BD
:10EAE0003046FFF7E0FD3046FFF7F2FC51E06946A3
:10EAF0000F840889488448898884617808AA0A981C
:10EB0000F7F716FC45E06288194602A8F7F7EBFC18
:10EB100005003ED12748818900293AD0617802AAB0
:10EB2000019200912378807B00220A99FFF762FE10
:10EB30002FE06288194602A8F7F7A6FC050028D145
:10EB4000617802AA0A98FFF741FF22E0628819461D
:10EB500002A8F7F7B8FC05001BD1684601890A989E
:10EB6000FFF798FC002817D0C068694602884989D9
:10EB700089180904090C01800BD0C068002808D04E
:10EB80000D480078002804D00C480121007805F0D9
:10EB9000EFF828460DB0F0BD69460F844E84088911
:10EBA0008884617808AA0A98F7F7C2FB3046F1E733
:10EBB0004BE20000D06B0020994800209F480020C5
:10EBC000F7B588B00D464878FFF734FC01270446B6
:10EBD00000282FD00020207160802E78012E06D0D2
:10EBE000072E0AD0132E18D0152E20D022E0AA7896
:10EBF00002A80A99FFF746FE17E02078032819D1EA
:10EC0000AA7802A80A99FFF78CFE05004BD10122D1
:10EC100000212046FFF747FD45E02078042809D170
:10EC2000AA7802A80A99FFF7BCFE05463BE02078C7
:10EC3000022802D000200BB0F0BDAA7802A80A99E1
:10EC4000FFF740FE05002ED16846008A002100280B
:10EC500024D1684600890246403A402A07D26A46D3
:10EC60005289172A03D36A469289172A06D2E16885
:10EC700048806088F7F782FB02210FE06A46E0686F
:10EC8000D28902806A46128942806A46528982800D
:10EC90006A469289C2800120207000276846028A55
:10ECA0002046FFF7D6FC204600F0E2FA02A9002039
:10ECB00001910090207A33462A460899FFF79AFD81
:10ECC000002F02D02046FFF703FC2846B3E70000E0
:10ECD00030B587B004464588014602A8FFF731FEEB
:10ECE000039900291AD068460089052819D00428FC
:10ECF00049D0062847D0072845D002A9284600F069
:10ED000059F8002808D0A068002801D004F0E8FED7
:10ED100001212846F7F74CFB07B030BD0028F7D09B
:10ED2000F1E76846008A0428EDD301A8FFF744FE06
:10ED30006846C088182809D30120694688821720B0
:10ED4000C882497905AA2846F7F7F2FA6846018A87
:10ED5000C088001D814202D02846FFF767FC684644
:10ED60000079039AC00701A9284603D0121DFFF7B6
:10ED700027FF02E0121DFFF789FE0028C3D02846B6
:10ED8000FFF754FCBFE70C214843094940183038CD
:10ED900001880029B7D0807802AA2946FFF7E0FC55
:10EDA0000028B0D1684600890428B1D1B4E700003A
:10EDB000D06B0020F3B583B00D460888FFF724FB25
:10EDC000060076D0F468002C73D0F1880398814255
:10EDD0006FD12089002874D0401E80B22081217F0D
:10EDE0000A013A4909685118C988884203D1632148
:10EDF0003046FFF775FC6069002828D168684178C3
:10EE000002780F0217432A89B91C8A420DD10121C9
:10EE1000C94304F0B3FD68602F81307A2A46039914
:10EE2000FFF79EFC002845D00EE04C21384604F048
:10EE300013FE606127830121C943686804F09EFDC9
:10EE400068602889801E28816069002837D02A8957
:10EE5000608B238B1118994201D9042132E0237F62
:10EE60001F011A4B1B68FB185B88994225D8616902
:10EE70000818696804F0D4FD2889618B401880B2B5
:10EE80006083218B884214D170886946088060694C
:10EE90000190208B0881307A6A460399FFF760FC65
:10EEA000002802D0606904F01BFE002060616083CE
:10EEB0002083012005B0F0BD03E0052102E0092117
:10EEC00000E006213046FFF735FAF2E7A8480020B7
:10EED000FFB583B00E461546022117200C9FF7F7A9
:10EEE000C1FB040023D0002F03D0201D0699B84792
:10EEF00000E0002026706570A070010AE17069468C
:10EF0000001D0881052008800A4801940078002827
:10EF1000039802D0FFF71EFA01E000F0B1F90500F6
:10EF200002D0204604F0DCFD284607B0F0BD1320D7
:10EF3000FBE7000099480020F0B585B015460E4665
:10EF400007461C460A22002101A804F043FE684639
:10EF50008581002D12D16088694688801548008817
:10EF60000881E068002809D0134A017F126809016E
:10EF7000891849886A46D180008950810F480090DD
:10EF8000F2B201AB15213846FFF7A2FF060007D009
:10EF9000002D05D02046FFF79BFA304605B0F0BDA6
:10EFA0000120207000202071024601462046FFF714
:10EFB00050FBF2E7A0480020A8480020FDE1000037
:10EFC0003EB504281DD30C210F4A41438C18303C18
:10EFD0006168002915D00D4A1278002A0FD06A46C0
:10EFE000108001912089108160896946FFF7B2F98C
:10EFF000002802D0606804F073FD002060600120EA
:10F000003EBD00203EBD0000D06B0020994800208E
:10F01000F8B5214F3E7834462048210100680D188C
:10F02000287801282DD1E96800292AD0C86800284D
:10F0300027D0088800281AD019480078002814D052
:10F04000164821010068081800F09CF8010003D060
:10F050002846FFF76FFA1DE01248641C00788442CE
:10F0600001D23C7001E0002038700120F8BD487FDB
:10F07000FF2806D128466221FFF732FBE96800200D
:10F0800048770848641C0078E4B2844200D3002426
:10F09000B442C1D10020F8BD9E480020A448002001
:10F0A000994800209B48002010B50520FFF788FFF5
:10F0B00000280ED10620FFF783FF002809D1042085
:10F0C000FFF77EFF002804D10720FFF779FF002813
:10F0D00001D0012010BD034800780028FAD0FFF7C6
:10F0E00097FF10BD9B480020FFB583B014460D4626
:10F0F0000C9F0E9A0D991E46062D13D001AB039856
:10F10000FFF70AF800281BD10198052207701C4B55
:10F1100042801978FF2915D00171491C1970142DEE
:10F1200014D018E06088FFF76FF90190002806D02E
:10F13000C068408820800198C0880390E4E70220DE
:10F1400007B0F0BD012119700171E8E762800198F4
:10F150002189C068018101980096027923462946D9
:10F160000398FFF7B5FE040003D00198FFF7B0F94C
:10F1700003E01E21019800F065F82046E0E700005A
:10F180009D480020F1B584B00498C4682C48E688F6
:10F190000088B04200D20646608A002804D0218A46
:10F1A000081AB04204DB05E0208A801CB04201D27C
:10F1B00085B200E0354602212846F7F753FA0700EA
:10F1C0003AD060886946088001970D81608A0028DE
:10F1D0000BD1207C3870208A000A7870BF1CB542A1
:10F1E00001D2258A01E0AD1EADB2618AE0682A46EF
:10F1F0004118384604F014FC04986946C088FFF7AB
:10F20000A9F8060003D0384604F06AFC15E020880F
:10F21000401E80B22080618A491989B26182228AA7
:10F22000914204D2002808D1FF20607705E0002138
:10F230000498FFF77FF900E01326304605B0F0BDD3
:10F24000A048002010B50446064848430649F2F796
:10F2500093FD0246234609332146044804F092FEFA
:10F2600010BD000040420F007102000037E60000B0
:10F2700010B50446407A04F007FFFF20607210BD0D
:10F280000A880C235A43074BD218303A5368002B94
:10F2900001D0162070474B68536050810889108157
:10F2A00000207047D06B002010B500230F22845C33
:10F2B00064001C438C54835C521EDB09D2B20F2ABB
:10F2C000F5D910BDFFB581B01D4617460E4608465C
:10F2D00000F05CF8002802D0112005B0F0BD144801
:10F2E00000F054F8040020D065710622A01D0A9990
:10F2F00004F096FB66802771019820700025E56276
:10F300000B9820730C98E0810D9820820E986082F3
:10F310000F98A08200F0B8F820866563002130467F
:10F32000A56302F031FE0020D7E71520D5E70000E5
:10F33000FFFF000070B514460D46064600F026F8A3
:10F34000002808D00379C06A00280CD01221194087
:10F35000102905D00BE00C48864213D0142070BD54
:10F36000002C02D103E0D8060CD4052070BDD906CC
:10F3700001D40F2070BD002804D0807EA84201D2A5
:10F380000C2070BD002070BDFEFF000030B50A4AA1
:10F39000002113780CE03C2455684C4364196488C0
:10F3A000844203D13C204143481930BD491CC9B2B5
:10F3B0009942F0D3002030BDAC470020F0B50C4D91
:10F3C00000210C4E2C780FE03C226B684A43D71882
:10F3D0007F88B74206D09A5C824203D13C204143E9
:10F3E000C818F0BD491CC9B2A142EDD30020F0BD40
:10F3F000AC470020FFFF000030B50B4A0021147815
:10F400000DE03C2355684B435B191B8E834204D1AE
:10F410003C2041434819408830BD491CC9B2A14233
:10F42000EFD3024830BD0000AC470020FFFF0000D2
:10F4300030B5134B0020134D1C781DE03C215A6859
:10F44000414389184A88AA4214D0496B002911D037
:10F450000A78012A02D0002A04D00BE049780C294E
:10F4600003D807E049780C2904D23C214843596865
:10F47000401830BD401CC0B2A042DFD3002030BDD8
:10F48000AC470020FFFF000030B5114C00210846BA
:10F4900023780AE03C226568424352191579002D11
:10F4A00001D0128E1143401CC0B29842F2D34808DA
:10F4B000C04381B2012004E0CA0704D14908401CBE
:10F4C000C0B29842F8D30121814088B230BD00001B
:10F4D000AC47002070B51348134C007F8107890F9B
:10F4E0008008081820701BD03C214843902104F06C
:10F4F000B3FA6060002002460C4B07E03C216568CF
:10F50000414349194B800A71401CCA6221788842E4
:10F51000F4DB074900208300401CCA500C28FADBAA
:10F5200070BD0000CC690020AC470020FFFF000048
:10F53000046B002000B5FFF729FF002800D0808A67
:10F5400000BD000030B50F4B00200F4C1A7814E0BE
:10F550003C215D68414349194D88A5420BD0496B58
:10F56000002908D04978C91F092904D83C214843FB
:10F570005968401830BD401CC0B29042E8D300200A
:10F5800030BD0000AC470020FFFF000030B5094A45
:10F590000020014614780AE03C2355684B435B1970
:10F5A0001B79002B01D0401CC0B2491CC9B2A1423A
:10F5B000F2D330BDAC47002001480078704700000E
:10F5C000AC470020F8B505000FD00024074E084FC7
:10F5D00008E03C207168604340184188B94200D07F
:10F5E000A847641C30788442F3DBF8BDAC470020A8
:10F5F000FFFF000070B50B4B002001460A4D1C7840
:10F600000DE03C225E684A4392195688AE4204D00F
:10F61000127B042A01D1401CC0B2491CC9B2A142CC
:10F62000EFD370BDAC470020FFFF0000074A002168
:10F630008B00D358002B05D0491CC9B20C29F7D335
:10F64000132070478900505000207047046B002041
:10F6500010B5FFF79BFE040013D06088012102F073
:10F6600093FCE06A002801D004F03AFA3C22002121
:10F67000204604F0AFFA0020C043608000202071D3
:10F6800010BD022010BD00B5FFF780FE002800D09D
:10F69000007B00BD10B50C460549884206D0FFF737
:10F6A00075FE002803D00079204000D0012010BD55
:10F6B000FEFF000010B50C46FFF768FE002802D0E0
:10F6C000818AA14201D1012010BD8482002010BD99
:10F6D00010B51248846B207B012817D1607927214F
:10F6E000252803D0262811D1E07E10E0E07E820795
:10F6F0000DD526206071204600F0EAFBE07E400731
:10F7000004D507480221C07804F032FB10BD400741
:10F71000FCD56171204600F0DBFB10BD006C0020C1
:10F72000006A002070B51121942004F095F90400BE
:10F7300044D02348942284630021204604F04AFAEE
:10F74000012222719020A07200231E4923732046BB
:10F750008030CD6885600969C1600321A1731A4DAD
:10F76000E5671A4D05601A4D45601A48807C1528DA
:10F770001DD008DC01280DD003280ED0072810D09A
:10F780000F281BD110E01D2813D0232813D03F28A9
:10F7900014D112E01320C04301E00D20C043607378
:10F7A0000CE00720C043FAE70220C043F7E7637389
:10F7B00004E0627302E00220F1E76173204670BD4D
:10F7C000006C0020206A0020D9F70000D9F8000062
:10F7D000D1F60000CC690020FEB53D4E0127B46B88
:10F7E000324625466035114668799C310191936B0C
:10F7F000663300280AD0891D0091012809D0002114
:10F8000002280ED003282CD01220FEBD0622184656
:10F8100048E0B0780028F9D12D490622A8311846D1
:10F8200040E02971287B002817D020466C30F8F77B
:10F8300045FB206600280DD001F0C4F9216E887ABE
:10F84000002807D0022028712046062266300C319D
:10F8500004F0E6F82879022826D02F7106220199B3
:10F860001EE02971287B002817D020466C30F8F75D
:10F8700025FB206600280DD001F0A4F9216E887ABE
:10F88000002807D0022028712046062266300C315D
:10F8900004F0C6F82879022806D02F7100990622B4
:10F8A0002046663004F0BCF87078002808D0E87C68
:10F8B0008009012804D120466C30F8F71BFB206634
:10F8C00004482773C078012104F052FA0020FEBDDD
:10F8D000006C0020006A002070B51948846B207B02
:10F8E00001282CD101F0FCF8E07E164DC10705D0AF
:10F8F000252140076171800F06D10EE0810708D5F0
:10F9000026216171400708D5E878022104F030FA19
:10F9100003E0400701D527206071A07E012804D0B4
:10F9200010210120FAF759FEE082E08AA18A4218EC
:10F93000E878012104F06EFB204600F0C9FA70BDA2
:10F94000006C0020006A002070B5F7F71DFB050071
:10F9500042D0F7F7E3FA040040D01020A071012054
:10F96000E071B021217360731D4801692046803029
:10F97000C16606461721202004F06EF8194B0021BD
:10F98000B06658186030027F6018D8263254E030D4
:10F99000491CC9B202700829F3D30021C943218749
:10F9A0002046FF212030417001708170E07E80216F
:10F9B0000843E0760C494420015320460C22FF21E5
:10F9C000623004F007F9204600F05AFE204600F0AD
:10F9D000EBFD2046F7F72CFC284670BD012070BDDA
:10F9E000206A0020006C0020B80B000070B5394B75
:10F9F0000446418D187DC20702D02822514305E0FC
:10FA0000354A5143FF31FF310231890A22468032A3
:10FA10001161002802D07F31090A02E02F4D4919F7
:10FA2000490B5B7FC91CC9188BB2A386218D9568D1
:10FA3000491CC60702D02826714305E0264E7143B3
:10FA4000FF31FF310231890A5B00C91A6918244D60
:10FA5000A94201D36D42491951612146FF31443118
:10FA60004A7B0D7B11022943C20702D01F3149098D
:10FA700002E01C4A5143490CC9188AB22346E28667
:10FA80002033D979C00702D02820414305E012482D
:10FA90004143FF31FF310231890A8818E086042092
:10FAA0002077002525861D71204600F027FEE08D79
:10FAB0000005010C204600F00DFFA08801228021E6
:10FAC000F8F72AF902210848FAF7DCF90748058116
:10FAD00070BD0000CC690020D7A30000FF07000024
:10FAE0000000C0A8C7100000451D0100006C0020E8
:10FAF000F0B5ED480022846BEC49A07A85B09528DA
:10FB00002BD094287ED0962825D18878C3079120C1
:10FB1000002B78D0A072FAF71DFE00210846FAF7F4
:10FB2000B1F9E34D2868002815D04068002812D0AC
:10FB30000220694608707520005D4870E07B0872FD
:10FB4000214600A806227631023003F069FF2868BA
:10FB500041686846884705B0F0BDC878C0077DD0C9
:10FB6000D24DEA702646803622460F320021F068D8
:10FB7000FAF7FEFCA871002871D1F0684078800681
:10FB8000800E2072801F1F2869D8F0680078000757
:10FB9000000F6072052801D00328EDD12046F168DE
:10FBA000663006220831019003F02CFF002856D061
:10FBB000F0682746007860374006C00F7875204609
:10FBC000F16876300622891C009003F029FFB648C0
:10FBD00025464078002830D0787D00282DD0F87E4A
:10FBE0008009012829D1286E002815D0817C0029A0
:10FBF00012D0C078022108437875216E082202A82D
:10FC0000891C01E01EE142E1F2F72DF9009A039907
:10FC10000298F8F70FF92EE0A8790007000F0128E5
:10FC20001ED028467430F8F765F92866002804D0FD
:10FC3000C0780221084378751FE0A8790007000FFB
:10FC400001280DD0E87AC10702D0697A03290ED0C5
:10FC5000800712D5687A052809D00EE0EDE0EAE0C9
:10FC6000284606226E30009903F0CCFE03E0A96F0F
:10FC7000686FF8F78FFE002899D0607A0528A07980
:10FC800006D0010779D00007000F06287ED0D2E009
:10FC9000010703D00007000F0128F8D1824D686EDC
:10FCA000002870D0FAF756FD2846406E8047F7F7D7
:10FCB00035F9050067D07F48816B0091816B009A10
:10FCC0009142F9D188204251F0682F46C27B817B56
:10FCD00012028918027C407C1204000610180818D1
:10FCE000A867F0682037C17C0A02017D807C090486
:10FCF00051180818E867F068407DF871F068C17D18
:10FD0000827D080210432885F068417E027E080249
:10FD100010436885F068C17E827E08021043A88582
:10FD2000F068417F027F08021043E885F168E81D12
:10FD30000522F9301E3103F073FEF0685E49203071
:10FD4000C078C006C00E7871F0682030C0784009D5
:10FD5000B871688D801F884209D2A88DFF21F431C7
:10FD6000884204D8E88D1921C901884207D9FF3596
:10FD70004135288BF7F74CF85DE007E003E04A488F
:10FD8000816E28468847F6F70FFE87E00420A071B1
:10FD9000617F891DE171B1680870E079B168800602
:10FDA000800E48707879C00702D13879022804D1D2
:10FDB000B0684022017811430170B0680622801CAF
:10FDC000019903F02DFEB0682146627F3E31083074
:10FDD00003F026FEE079394D401D8008B268A97C09
:10FDE00080001154E079FAF7F9FD35495A20096885
:10FDF0000865E0792D49C00080220A71297DFF3015
:10FE00001930C90702D01F30430902E02D49484389
:10FE1000430C2848816B0091816B009A9142F9D183
:10FE20002949D018884201D3494240182749C8605F
:10FE30009620A0728FE692202DE008790128F9D152
:10FE40000A71F8E78878C0071DD0A079020705D0AD
:10FE50000007000F012801D00628ECD19520A072E0
:10FE60008020087113481223816B0091816B009AE6
:10FE70009142F9D11449D018884201D3494240181F
:10FE80001249C86067E608790128D4D063E60B7987
:10FE9000012BCFD10A71A072FAF75CFC0021084651
:10FEA000F9F7F0FF57E60000006C0020206A002000
:10FEB000D0480020001000407B0C0000CC690020DE
:10FEC00038460020C71000000000C0A8006A0020CB
:10FED000F8B504465648C06D00287DD1A07E264660
:10FEE0000007000F254660368035A071012826D016
:10FEF000207F801D8106890EE171A968A0790870B4
:10FF0000227F2146A8681E31083003F089FD7079F0
:10FF100027468007663700280DDA206E00280AD0B1
:10FF2000807A002807D002203071216E06223846E0
:10FF30000C3103F075FD7079C00728D124E00C2145
:10FF4000E171A968012008707079274680076E3733
:10FF500000280DDA206E00280AD0817C002907D005
:10FF6000C07C7073216E06223846143103F058FDB0
:10FF7000707B002804D0A8688022017811430170AA
:10FF800006223946A868BFE73079022804D1A8685C
:10FF90004022017811430170A968E0794870A8688F
:10FFA00006223946801C03F03BFDE079214E401DBE
:10FFB0008008AA68B17C8000115492211E4DA17264
:10FFC000E879002801D0FAF7C5FB1C495A200968D6
:10FFD0000865E079C00000E029E080212971317DC9
:10FFE000FF301930C90702D01F30430902E014491D
:10FFF0004843430C1348816B0091816B009A9142F6
:020000040001F9
:10000000F9D11149D018884201D3494240180F490B
:10001000C86000210E48F9F735FF0120E8719420EF
:10002000A072E37962790B490B48FAF7C3FBF8BD7C
:10003000006C0020CC690020206A00203846002097
:10004000C7100000001000400000C0A8006A002097
:10005000F1FA000055555500D6BE898EF8B5044614
:10006000807900280ED0208F2546401C80B2208742
:10007000618E8035491C61860021A177E379002BD0
:1000800002D013E00120F8BD217F00290ED04207E5
:100090000CD16A6904291FD30826711A8A4201D338
:1000A000511A02E0521A8D49511869612246E17BCA
:1000B00020320092002916D0894F4A064FD5BF2220
:1000C0001140E173009A002111712A6804210A434A
:1000D0002A60012B11D042E05118804A9142E4D3AA
:1000E00052428918E1E706287ED33E212046F6F7E2
:1000F000CDFD009908710220F8BD21773A7D29696C
:10010000002A02D07F31090A02E0764BC918490B58
:100110007B7FC91CC91826468BB2FF36A38644369E
:10012000717B367B09023143D60702D01F31490962
:1001300002E06D4E7143490C5B00C9188BB2E38637
:100140000099D207C97902D02822514305E0674AB5
:100150005143FF31FF310231890AC918E186A17B81
:100160002646CA074036002A78D0318B814276D1A4
:10017000A08D70830098F17BC171308A2085B08A90
:10018000A085F08AE08501010098807803F0BCFF2B
:1001900000206086E079002809D0208D002855D005
:1001A0003A7D6969D20744D02822504347E03A7D1E
:1001B000208D6969D20702D02822504305E04B4ABE
:1001C0005043FF30FF300230800A14300818434992
:1001D000884201D3494240186861708A60853A7D3F
:1001E000D107014604D000E076E02823594302E01D
:1001F0003E4B5943890A2961D10701D000200AE00A
:100200003A494143CF093949F9F7B0FF8905800AD6
:100210000843C000381AC0B22077042802D32869E6
:10022000401C2861A07E002821D0204600F0E4F97F
:100230001DE02E4A5043FF30FF300230800A08187C
:100240002649884201D3494240186861708A608516
:10025000397DC90704D02821484307E013E00EE0A8
:1002600022494843FF30FF300230800A2861E07B9A
:1002700040210843E073A07B400840001EE0081ABC
:10028000000408D41BE0890719D5E31DF933598907
:100290000A1A120407D528212046F6F7F7FC009920
:1002A00008712820F8BD884209D1E11D0522FE31E0
:1002B000184603F0B5FBA07BFD210840A073009811
:1002C000C078400608D53088218F884204D10121AA
:1002D00068688902084368600020F8BD0000C0A873
:1002E000CC690020FF070000C7100000D7A3000062
:1002F000002809D00146803101230A689B021A4375
:100300000A60FF2120300170704770B50646FF3645
:100310002436717D337D0A0231461A431D31CB8864
:100320009A4200D31A460446FF3442342273120A1A
:1003300025466273203D6A7E2B7E12021A430B898A
:100340009A4200D31A460346FF3344331A73120A03
:100350005A73727E367E120232434E88B24200D306
:1003600032462274120A62746A7F2C7F12028988D4
:1003700022438A4200D211461974090A597400F0C6
:10038000DDFB70BDFEB506466648016E01297DD9CC
:10039000046D6548C07B22304508304680300B35FF
:1003A0000290BBE0B44202D12468002C6ED0A07E43
:1003B00000286CD1471E02980169204680300190C8
:1003C0000069009081421FD30298019940694A69EF
:1003D000904219D35449097DC90702D07D21890271
:1003E00001E001214904801A81420DD9009981421E
:1003F00002D2F1F7C1FC0846A84205D2009949088B
:10040000A94200D929460F18781C40D046493846E1
:10041000097DC90705D04549F9F7A8FE8904800B75
:1004200004E01921F9F7A2FEC905400A0843401C5F
:10043000410872D0E079002811D0708D618D88421A
:100440004ED2F1F799FC0F4637492846097DC90776
:1004500020D03649F9F78AFE8904800B1FE0204638
:10046000628D40304282A28D8282E28DC28202225F
:10047000C2730182318F0A3101830198019A416868
:100480000420014351600121617601E049E044E02C
:10049000A07642E01921F9F769FEC905400A084330
:1004A000401C400887421BD3618D708DF1F764FCBE
:1004B0000F461D492846097DC90705D01B49F9F794
:1004C00055FE8904800B04E01921F9F74FFEC90598
:1004D000400A0843401C618D4008081A87421CD915
:1004E000608D4108C81C062801D9C91C00E00621FE
:1004F00020464030C18519228900D201914200D99D
:1005000011460186A18D8182E18DC1821420A076E1
:10051000A08886228021F7F7FFFB2468002C00D0FA
:1005200040E7FEBD006C0020CC69002033030000D2
:1005300018B5817F490830D1C17F00292DD1184BD2
:10054000418F5A7C914228D20246047CFF3200211E
:100550004432002C03D0517B147B09022143007AE2
:10056000C00604D5507C127C0002104341180029BB
:1005700013D0187DFF312D31C00702D01F314C0937
:1005800002E0084841434C0C68461434F6F7B6FDC7
:100590000098A04201D3012018BD002018BD000022
:1005A000CC690020C7100000017AF32211400172CB
:1005B000704700000148006E70470000006C00208A
:1005C0000548016D002004E0CA79002A00D1401CD2
:1005D00009680029F8D17047006C00200548016DBA
:1005E000002004E0CA79012A00D1401C09680029D2
:1005F000F8D17047006C0020FCB584461E48006EA0
:10060000012835D91D480124C07B654622304008A9
:100610000B308646604640300090C07B401E8035DF
:10062000019023E0002328206969DB4360430A1816
:100630001148016D13E0614502D10968002918D005
:100640000E46803637692869874205D17069904225
:1006500001D8131A00E0831A734503D309680029EF
:10066000E9D106E0002904D00198641CA042D9D841
:10067000FCBD00980482FCBD006C0020CC69002009
:1006800030B501461B4CFF312431238C0B761B0AFD
:100690004B760A46638C891E0B771B0A4B77A38C1B
:1006A00013751B0A5375E28C0A76120A4A761B23CD
:1006B0001F31FF24CB8049340C814B808C80491C36
:1006C0000B7300254D730A46891C0C73250A4D7364
:1006D00013741B0A53740C74220A4A740649097D68
:1006E000C90701D00B2100E00A21828E520089182F
:1006F000C18630BD006C0020CC69002070B5044676
:100700004034A288C38D91005518EE08418DB34244
:1007100004D2D01AC000F1F745FB02E02846F1F7F9
:100720002BFB608070BDEC2109580A789207920F6C
:100730008272032A08D0FF2242750A7810231A40D9
:1007400002744978C17270478A78F5E710B50400E1
:100750000AD02221F6F79AFA01462046203001718C
:1007600000216173FF21417010BD000070B52C495C
:100770000446808F097C04260025884205D3207A10
:10078000704020722574012070BD26480068002842
:1007900040D12548F6F7D2FB01003BD0887A48814A
:1007A00020468030826F002A30D0C26FD160C1678E
:1007B000A18F491CA187C16FCD60C26FE17AD18042
:1007C000C26FA17A11711949C06F0A690168E07A94
:1007D0002130400913680B6053684B6093688B604D
:1007E000D368CB6013690B6153694B6193698B616B
:1007F000D369401ECB61203120320006000EE9D1C2
:100800000B490889401C0881002070BD8167C167C1
:100810000121CFE7207A704020722574022070BD3C
:10082000CC6900206848002052FF0000206A0020A8
:10083000006C002030B5014680310B46096F00295D
:1008400002D00A89012A01D0012030BD027A012498
:100850009208920002720D79002D01D0224301E02E
:1008600002252A4302728A79427203220A81196F91
:10087000C968002908D0064A418F527C914203D2B0
:10088000017A102211430172C475002030BD0000AE
:10089000CC69002070B504460546203420780E4609
:1008A000FF2803D003F0F0FBFF202070E0786021E8
:1008B0000843E07028464030298F42882346891833
:1008C000018032462946024803F05CFB70BD0000FF
:1008D000F102010070B5044605462034A0780E46AA
:1008E000FF2803D003F0D0FBFF20A0702B4622335B
:1008F00032462946014803F045FB70BD3509010029
:10090000F8B5074604462037787815460E46FF2886
:1009100003D003F0B9FBFF20787023462133324621
:100920002146034803F02EFB40342572F8BD000039
:100930004D07010070B505000CD0E97B2C46203432
:10094000002908D00821F6F7A1F92071002068736A
:10095000FF20A07070BD3E21F5E70000F0B506460F
:1009600085B004210020F9F738FE014630464030BA
:10097000009001822248006E01283CD90098318FF6
:10098000008B0125401A00994F8A94218959784398
:10099000401804901B48C07B223040080B30039065
:1009A000781E029025E016482821046D2846484309
:1009B00000220499D2434018019013E0B44202D1BE
:1009C0002468002C19D0204680300169B94205D135
:1009D000019A4069101AF1F7CFF90A46039882424A
:1009E00003D32468002CE9D107E0002C05D002983D
:1009F000AD1CA842D7D805B0F0BD00980582FAE733
:100A0000006C0020CC69002030B50022074C07E0C4
:100A10000D889D4202D8D8B2088030BD521CD2B297
:100A2000A35C8342F9D8FF2BF2D130BD954301007E
:100A300010B5F1F7F9FA002010BD000010B5154906
:100A40000968CA68520B52030243CA603A281FD988
:100A5000114B1A68114881688902890E16290CD039
:100A600081688902890E1A2903D28168090C8906D6
:100A7000F1D1F9F76FFE002010BD3021064CC943BB
:100A80008034216081688902890E1A29FAD31A609C
:100A9000012010BD6048002000E100E000C20040DD
:100AA00010B5F1F76BFB002801D0012010BD034900
:100AB000792009680865002010BD00003846002034
:100AC00010B5F1F7B5FB002801D0012010BD034996
:100AD0007A2009680865002010BD00003846002013
:100AE00070B50E4DA86A002817D080470C4E0446FA
:100AF0007089002811D0A04201D2214600E00146B1
:100B0000A04200D32046081A3C2806DDE86A0028E7
:100B100000D08047F2F712FA748170BDCC690020D2
:100B2000006A002010B5418E032900D90321828E6E
:100B30004A430286FFF7D4FF10BD00000146FF3193
:100B400044314A7B0B7B1102074A1943127DD207BD
:100B500002D01F31490902E0044A5143490C828EF8
:100B600052008918C1867047CC690020C710000068
:100B700010B588B00C4600210091019102910391BB
:100B80000491059106910791E1786A46D173217924
:100B900091736179517304AA6946FFF749FF6A4668
:100BA000D07F217888420AD1907F6178884206D12F
:100BB000507FA178884202D1012008B010BD0020EA
:100BC000FBE7000010B504460F48806F02E0A0422A
:100BD00003D0C06B0028FAD110BD0028FCD0002C37
:100BE000FAD0A07A002805D0214620460C311A30D0
:100BF000F5F7EAFDA07C0028EED02146204614310E
:100C00002A30F5F7E1FD10BD006C0020034610B559
:100C10000A461946014803F0B5F910BD210C010040
:100C200070B5124D0446A86F02E0A04203D0C06B1D
:100C30000028FAD170BD0028FCD0002CFAD0A07A90
:100C4000002805D0214620460C311A30F5F7BCFDAE
:100C5000A07C002805D02146204614312A30F5F723
:100C6000B3FD2046296BFFF7D1FF70BD006C00205B
:100C7000F0B50646654885B0016E01297ED9E021B0
:100C8000895D89077AD500210291006D0D460446E1
:100C900003E0817E002977D100680028F9D1471E42
:100CA0005B480097C07B223040080B3001903046F3
:100CB0008030039031E0B44202D12468002C2ED061
:100CC00022460398803251694069814210D3081A44
:100CD00003990969814202D2F1F74EF8084600995A
:100CE000884219D201990090884215D2029413E0EB
:100CF000884201D3401A02E0401A4649401811695F
:100D0000814202D2F1F738F80846B84204D201997C
:100D10000746884200D225462468002CCBD11924EE
:100D2000E401002D47D0E879698D00280BD00F46EB
:100D3000708DF1F721F8002926D17908C81C062802
:100D400024D9C91C23E02846403041820221C173C6
:100D50002A8F418B52184907490F511A10310183CC
:100D6000A98D8182E98DC1822846FFF7F7FD2846CB
:100D70008030416804221143416001E042E003E019
:100D8000012068760320A87605B0F0BD062128462C
:100D90004030C1858900A14200D80C460486A98D47
:100DA0008182E98DC1821220A876A88886228021BE
:100DB000F6F7B2FFE8E70298002823D0718D408D46
:100DC0000D46F0F7D9FF00291CD1307E000619D559
:100DD0006908C81C062801D9C91C00E00621304654
:100DE0004030C1858900A14200D80C460486B18DEF
:100DF0008182F18DC1821320B076B0888622802155
:100E0000F6F78AFF00203076BEE70000006C002075
:100E1000CC6900200000C0A8F0B5FF4887B0856D00
:100E2000F9F7FEFE287BD02826D0D1287BD0D22807
:100E3000F6D1FA4C6078002873D02846FFF778FB8B
:100E400001286FD0F9F786FCE87F002810D0F4491C
:100E50000968000905D03D212846F5F717FF242130
:100E60004855F048026B002A02D0052185209047A2
:100E7000284600F019FEFFE3E84C2079C007CFD0E8
:100E8000687B01280ED128468030016F002909D1E6
:100E90004068002806D1E87B802803D1A88D698EA0
:100EA0008842E8D24620405DC00709D0294601208B
:100EB000FFF7F6FD002807D02846FFF733FEDBE3F7
:100EC000D949592009680865C02020701020E071B8
:100ED000D1202873AA7CE96FA86FF9F78DFB298EC2
:100EE000E88E49004018400180212171CD49097DDB
:100EF000C90702D01F30400902E0CC494843400CEA
:100F0000CB498A6B00928A6B009B9A42F9D1C949FE
:100F10001818884201D349424018C749C8607FE782
:100F200001E0E9E3E9E3BD4F3878C00771D02A4614
:100F300040320192029290792E46C10780362C46AB
:100F4000C90F2C3AF06EF9F713FB01003846817196
:100F50000CD0012972D002988079C00702D0E07FBE
:100F6000401CE077E07B002869D0A6E200272046FD
:100F7000E77720300090C17802221143C170E07BF6
:100F800000282ED02046F5F7E7FD002829D1677408
:100F9000306F00280DD0018901290AD04189FF2234
:100FA000120211434181306FC0683067E08F401CEE
:100FB000E087607A002806D002988079800702D501
:100FC0002046F5F7A1FE607B44280AD1009808214D
:100FD0000771306808433060A07B0843A073462047
:100FE00060732046F5F7A7FD0028BBD12046FFF728
:100FF0009AFBA07B00070DD5E07A00280AD0607D1F
:10100000062807D0022805D0207A04214840207203
:10101000A8E7F3E3A07A032812D0E07A002802D0F0
:101020002046FFF7A3FBE07A00289BD00198807947
:10103000C00797D02046F5F7C7FD93E714E217E203
:10104000607D0F2822D000283BD001284ED00228F6
:1010500065D00A286CD00B287ED0032871D00628D2
:1010600070D008286FD009286ED00C286DD01228B7
:101070006CD013286BD014286AD0152869D00728A3
:1010800068D00D2867D0112876D0DCE1E07A1828E6
:10109000FBD1E020005D8007F7D5607B012801D0FF
:1010A0009228F2D12046F6F73BFF014600980171E5
:1010B000617B922903D1C17801221143C170932130
:1010C0004CE1E07A0C28E0D1607B012809D092281D
:1010D00002D0972805D0B6E100980122C1781143CB
:1010E000C170132161730521A1769FE7E07A08287A
:1010F000CBD1607B012802D0922802D0A3E123212A
:101100008AE100982A21017131680422114331607B
:1011100024216173C17801221143C17086E7E07A0E
:101120000228B2D1F06EC17802988173332173E145
:10113000E07A0128A9D1607B0128A6D173216BE157
:101140000AE01AE0BEE0C5E0DFE0F9E008E122E1F4
:1011500029E134E13EE161E1E07A012895D1607B4B
:10116000742892D1029887710098C178490601D5F8
:101170001021C17075214FE154E1E07A172884D124
:101180000396F16E2046FF3000912746082210306A
:10119000C91C02F045FC0099087BC97A000208438B
:1011A000F91DFC310875000A487502F0BBFDFF37D8
:1011B00021373872010A7972010CB972000EF87287
:1011C00002F0B0FD01040A0E3873010205927A7331
:1011D000090E84460491B973000EF873009986468F
:1011E0000A7CC97B090252180099897B0B0400997B
:1011F000497B090659185118039A516200990A7DD2
:10120000C97C090252180099897C0B040099497C19
:1012100009065918511811E0006C0020206A0020BE
:1012200080C30040CC69002038460020C710000071
:10123000001000400000C0A8006A0020039A604629
:101240001162BA7AF97A120289187A7A3B7A120410
:101250001B06D2188918039A0006D161059A0499D1
:101260001204090210187144039A0918916102F0DE
:1012700059FDC2B284460104080E04923A7478748F
:10128000614686460B021B0E6046BB74020EFA7462
:1012900000991B04887D4F7D00023F18C87D097EA0
:1012A0000004090640183F180398714687630498A4
:1012B0000902401811065918039A4018D0634322B6
:1012C0006273B0E6E07A012878D1607B522875D14C
:1012D0005521A1E0E07A092870D1607B01286DD109
:1012E00000232046803084466046C06ED91CE71833
:1012F000415C3846C0300174007EE03701405B1C21
:101300003970082BF0D3632128E0E07A092855D101
:10131000607B622852D1002320468030844660469C
:10132000C06ED91CE718415C3846C0300174007E9D
:10133000E03701405B1C3970082BF0D365210DE0CC
:10134000E07A06287FD12046F6F774FE607B82287B
:1013500003D00122520271687CE08521617362E64C
:10136000E07A01286FD1E020005DC0066BD5607B7C
:10137000012802D0A22802D007E0A3214CE0009867
:101380000122C1781143C170627301227168D202D7
:10139000114371604AE6E07A012854D1607BA228AB
:1013A00051D1A42138E0E07A09284CD1607B012892
:1013B00049D12046F6F71EFEB321CFE719E0E07AC7
:1013C000092840D1607BB2283DD12046F6F712FEB5
:1013D000B421C3E7E07A022835D100991A200871B8
:1013E000607BA22806D0622806D0922806D0B228B8
:1013F00011D028E0A5210FE067210DE0992060734E
:101400002046E0300278FD231A400270C87801229D
:101410001043C8700AE6B521617307E6E07A022836
:1014200006D010E0E07A03280DD1F06E017901E0DA
:10143000F06EC17800980171607B92280DD09728DA
:1014400010D001288BD02046617DF7F725FA0122C4
:101450007168D20311437160E5E500980122C178FB
:101460001143C170982179E7A07F401CA07779E5EE
:101470008020E073F74A2076117D3069002902D080
:101480007F30000A02E0F44BC018400B527FC01CB2
:10149000801882B22046FF30A2864430437B077B0F
:1014A00018023843C90702D01F30400902E0EB4957
:1014B0004843400C51004018E086688F401C688704
:1014C000687C00283BD1287A032108430024EC756E
:1014D0004027C0B2EF216F7408402872687B012852
:1014E00011D0002872D0672871D071DC472870D0E5
:1014F00070DC31286FD078DC13286ED0232801D01F
:10150000242863D113E17068002868D081050ED5C6
:10151000E87E000607D52846F7F7CCF9E87EC00735
:1015200001D0822169730120400271684BE00106FD
:1015300006D58021884370602846F7F743F887E096
:10154000810706D50221884370602846F5F7FAFB2B
:101550007EE0410507D50121890288437060284655
:10156000F5F7EFFF74E0C10407D5012109038843B3
:1015700070602846F5F706FF6AE0010404D50121F2
:10158000C9038843706063E0810407D501214903E2
:10159000884370602846F5F70BFC59E041040AD5F2
:1015A00001218903884370606FE00F2117E128460D
:1015B000F6F7F4FA7CE100054AD52846F5F7D4FFA2
:1015C00001207168C0028143716041E03DE04DE15E
:1015D0001DE014E10EE0C8E007E069E0FFE72846FF
:1015E000FFF728F9002830D132E033287ED0432895
:1015F0002BD1E3E055287AD004DC492876D0502856
:1016000023D1F0E0632873D065281ED128E1A328F8
:101610006FD00EDC932834D006DC73286AD075288E
:1016200069D0852811D12AE1982839D099280CD180
:1016300036E0B32871D004DCA42801D0A52804D159
:1016400039E1B4286AD0B52869D02846F6F728FDD4
:101650002846F6F78DFD687A00287DD002988079BB
:10166000800779D529460020FFF72AFA002874D090
:1016700000E001E0F9F76EF82846F5F77FFA07B0C9
:10168000F0BD2420405D002804D0E020405D4007EC
:101690008DD58AE72846F6F703FD02213068D1E0B0
:1016A0002846F6F7FDFC012068730421306826E126
:1016B000F16E0298CA78C2734A790B7912021A4302
:1016C0000282CA798B7912021A4342824A7A0B7AD1
:1016D00012021A438282CA7A8B7A12021A43C28297
:1016E0004A7B0B7B11021943018307E047E097E037
:1016F000ABE0DAE04CE05CE0BDE18FE1698D428A6D
:1017000091420DD1A98D828A914209D1E98DC28A77
:10171000914205D10121818303E0D7E0DFE0E6E0DB
:101720008483A87B01242043A873284642E0F16EFD
:1017300000200A18D3782A18FF320132401CC0B2A8
:1017400053710528F5D3487A0A7A01021143FF2024
:101750000B304153A87B01E0D4E0D7E002210843DD
:10176000A8732846F6F79CFCA2E02846F7F709F88C
:10177000029816218173012109033068BFE02846D1
:10178000F6F78EFC0121306809030843306013E04E
:101790002846FFF74FF8002800D159E7029C0120A6
:1017A000E0712846F5F7BFFEA07940084000A0711F
:1017B0004EE72846F6F774FC6C7349E72846E0309C
:1017C0000178C90703D02846F5F756FC40E71A22EE
:1017D00024214A550078400700D4E8E60321284632
:1017E000F6F7EEF964E02846F6F709FF02980122C1
:1017F000817911438171B464F46429E7FFE0E0204A
:10180000405D400704D503212846F6F7D9F902E0E8
:101810002846F6F7C3F9A87BF7210840A87347E0EC
:1018200002980222817911438171346428467464DC
:10183000F6F7F3FE24204455A87BF7210840A8734F
:10184000306810210843306032E02846F5F73CFC50
:1018500009E00000CC690020FF070000C71000006D
:101860002846F6F71DFC2420445505E02846F6F7E7
:1018700017FC1A212420415530683843E3E72846F5
:10188000F6F70EFCE87EC00707D02420445501215E
:101890003068490208433060EC7628462030C27830
:1018A00001210A43C2706973D2E62846F5F75CFE4F
:1018B00001206873CCE62846F6F7F2FB01212846A2
:1018C00069732030C2780A43C270C1E62846F5F732
:1018D00093FD242044550121C9023068B2E728460F
:1018E000F6F7DEFB012068732420445504E0284607
:1018F000F6F7D6FB0120687301213068C90208435E
:101900003060A5E660485A21006801655F4CA07907
:1019100000282ED1207800062BD5288E5C4B40085D
:10192000288600206886F06E197D4078C00050300F
:10193000CA0702D01F30400902E0564A5043400C0B
:10194000A268101AF060E87B40060CD530690029C7
:1019500002D07F30000A02E04F494018400B597F07
:10196000C01C4018A886F16830690918A88E091AA9
:101970007161687AFFF762F8002802D12846F5F70E
:10198000FDF8D2202873687AC00080212171404977
:10199000FF30097D3930C90702D01F30400902E00D
:1019A0003C494843400C3D498A6B00928A6B009B3E
:1019B0009A42F9D13A491818884201D3494240184D
:1019C0003849C860B06F002801D1FFF729FA0368D1
:1019D00082790179A8889B1CF4F79EF90028F4D13C
:1019E000B06FFF224189120211434181B06FC0687C
:1019F000B067A88F0028E8D0401EA887E5E73879AF
:101A00000128E2D1214C00202071F8F7A3FE2078B4
:101A1000000601D5FFF750FAFFF72AFA4620405D8D
:101A2000C00704D029460120FFF73AF803E0164921
:101A3000592009680865D12028732846FF304430B2
:101A4000417B027B08021043802121711049FF3045
:101A5000097D2D30C90702D01F30400902E00D4931
:101A60004843400C0D498A6B00928A6B009B9A4256
:101A7000F9D1FFF74CFA20790128A6D103490020BB
:101A80000871F8F767FEC7E738460020206A002093
:101A9000CC690020C7100000FF07000000100040C4
:101AA0000000C0A8006A0020F8B50546064680364A
:101AB0002F462C46306840372034002875D08107E7
:101AC00007D5022188433060A88806228021F6F7D6
:101AD00023F9306841074BD504218843964A30608A
:101AE000137D3069002B02D07F30000A02E0934959
:101AF0004018400B517FC01C401881B22846FF306F
:101B0000A9864430427B007B12020243D80702D0F0
:101B10001F32500902E08A484243500C49004018E5
:101B2000E886E078400607D50121706889020843FD
:101B300070602846FEF7E2FD2079002808D0402199
:101B40002976697E002905D0B98B002907D00DE0E0
:101B50008021F5E7E07801210843E07001E00028EA
:101B600004D1A88803228021F6F7D6F80020A876B1
:101B7000306801070BD5082188433060A88805220A
:101B80008021F6F7C9F8E07804210843E070306856
:101B9000C1061FD5102188433060F879002805D090
:101BA0000020F871A888302202E057E0A8880822B7
:101BB0008121F6F7B1F8E020405DC00605D5B88870
:101BC0000005010C2846FEF765FEE178012001437F
:101BD000E17068733068810508D5012149028843A6
:101BE0003060A8880C228121F6F796F8306841060B
:101BF0000CD5402188433060A88804228021F6F764
